******************************************************************************
             TMS320C2000 Linker PC v15.12.5                    
******************************************************************************
>> Linked Thu May 25 17:11:02 2017

OUTPUT FILE NAME:   <Test2_PMSM_Porting_F28377D_CPU1.out>
ENTRY POINT SYMBOL: "_c_int00"  address: 0008648d


MEMORY CONFIGURATION

         name            origin    length      used     unused   attr    fill
----------------------  --------  ---------  --------  --------  ----  --------
PAGE 0:
  D01SARAM              0000b000   00001000  00000027  00000fd9  RWIX
  BEGIN                 00080000   00000002  00000002  00000000  RWIX
  MYFLASH               00080004   0000007c  00000027  00000055  RWIX
  FLASHA                00080080   00001f80  00001f7f  00000001  RWIX
  FLASHB                00082000   00002000  00002000  00000000  RWIX
  FLASHC                00084000   00002000  00002000  00000000  RWIX
  FLASHD                00086000   00002000  00001d96  0000026a  RWIX
  FLASHE                00088000   00008000  000040c2  00003f3e  RWIX
  FLASHF                00090000   00008000  00000000  00008000  RWIX
  FLASHG                00098000   00008000  00000000  00008000  RWIX
  FLASHH                000a0000   00008000  00000000  00008000  RWIX
  FLASHI                000a8000   00008000  00000000  00008000  RWIX
  FLASHJ                000b0000   00008000  00000000  00008000  RWIX
  FLASHK                000b8000   00002000  00000000  00002000  RWIX
  FLASHL                000ba000   00002000  00000000  00002000  RWIX
  FLASHM                000bc000   00002000  00000000  00002000  RWIX
  FLASHN                000be000   00002000  00000000  00002000  RWIX
  RESET                 003fffc0   00000002  00000000  00000002  RWIX

PAGE 1:
  BOOT_RSVD             00000002   00000120  00000000  00000120  RWIX
  M01SARAM              00000122   000006de  00000200  000004de  RWIX
  ADCA_RESULT           00000b00   00000020  00000018  00000008  RWIX
  ADCB_RESULT           00000b20   00000020  00000018  00000008  RWIX
  ADCC_RESULT           00000b40   00000020  00000018  00000008  RWIX
  ADCD_RESULT           00000b60   00000020  00000018  00000008  RWIX
  CPU_TIMER0            00000c00   00000008  00000008  00000000  RWIX
  CPU_TIMER1            00000c08   00000008  00000008  00000000  RWIX
  CPU_TIMER2            00000c10   00000008  00000008  00000000  RWIX
  PIE_CTRL              00000ce0   00000020  0000001a  00000006  RWIX
  PIE_VECT              00000d00   00000200  00000000  00000200  RWIX
  DMA                   00001000   00000200  000000e0  00000120  RWIX
  CLA1                  00001400   00000040  0000003e  00000002  RWIX
  EPWM1                 00004000   00000100  00000100  00000000  RWIX
  EPWM2                 00004100   00000100  00000100  00000000  RWIX
  EPWM3                 00004200   00000100  00000100  00000000  RWIX
  EPWM4                 00004300   00000100  00000100  00000000  RWIX
  EPWM5                 00004400   00000100  00000100  00000000  RWIX
  EPWM6                 00004500   00000100  00000100  00000000  RWIX
  EPWM7                 00004600   00000100  00000100  00000000  RWIX
  EPWM8                 00004700   00000100  00000100  00000000  RWIX
  EPWM9                 00004800   00000100  00000100  00000000  RWIX
  EPWM10                00004900   00000100  00000100  00000000  RWIX
  EPWM11                00004a00   00000100  00000100  00000000  RWIX
  EPWM12                00004b00   00000100  00000100  00000000  RWIX
  ECAP1                 00005000   00000020  00000020  00000000  RWIX
  ECAP2                 00005020   00000020  00000020  00000000  RWIX
  ECAP3                 00005040   00000020  00000020  00000000  RWIX
  ECAP4                 00005060   00000020  00000020  00000000  RWIX
  ECAP5                 00005080   00000020  00000020  00000000  RWIX
  ECAP6                 000050a0   00000020  00000020  00000000  RWIX
  EQEP1                 00005100   00000040  00000022  0000001e  RWIX
  EQEP2                 00005140   00000040  00000022  0000001e  RWIX
  EQEP3                 00005180   00000040  00000022  0000001e  RWIX
  DACA                  00005c00   00000010  00000008  00000008  RWIX
  DACB                  00005c10   00000010  00000008  00000008  RWIX
  DACC                  00005c20   00000010  00000008  00000008  RWIX
  CMPSS1                00005c80   00000020  00000020  00000000  RWIX
  CMPSS2                00005ca0   00000020  00000020  00000000  RWIX
  CMPSS3                00005cc0   00000020  00000020  00000000  RWIX
  CMPSS4                00005ce0   00000020  00000020  00000000  RWIX
  CMPSS5                00005d00   00000020  00000020  00000000  RWIX
  CMPSS6                00005d20   00000020  00000020  00000000  RWIX
  CMPSS7                00005d40   00000020  00000020  00000000  RWIX
  CMPSS8                00005d60   00000020  00000020  00000000  RWIX
  SDFM1                 00005e00   00000080  00000080  00000000  RWIX
  SDFM2                 00005e80   00000080  00000080  00000000  RWIX
  MCBSPA                00006000   00000040  00000024  0000001c  RWIX
  MCBSPB                00006040   00000040  00000024  0000001c  RWIX
  SPIA                  00006100   00000010  00000010  00000000  RWIX
  SPIB                  00006110   00000010  00000010  00000000  RWIX
  SPIC                  00006120   00000010  00000010  00000000  RWIX
  SPID                  00006130   00000010  00000000  00000010  RWIX
  UPP                   00006200   00000100  00000048  000000b8  RWIX
  WD                    00007000   00000040  0000002b  00000015  RWIX
  NMIINTRUPT            00007060   00000010  00000007  00000009  RWIX
  XINT                  00007070   00000010  0000000b  00000005  RWIX
  SCIA                  00007200   00000010  00000010  00000000  RWIX
  SCIB                  00007210   00000010  00000010  00000000  RWIX
  SCIC                  00007220   00000010  00000010  00000000  RWIX
  SCID                  00007230   00000010  00000010  00000000  RWIX
  I2CA                  00007300   00000040  00000022  0000001e  RWIX
  I2CB                  00007340   00000040  00000022  0000001e  RWIX
  ADCA                  00007400   00000080  00000080  00000000  RWIX
  ADCB                  00007480   00000080  00000080  00000000  RWIX
  ADCC                  00007500   00000080  00000080  00000000  RWIX
  ADCD                  00007580   00000080  00000080  00000000  RWIX
  INPUT_XBAR            00007900   00000020  00000020  00000000  RWIX
  XBAR                  00007920   00000020  00000020  00000000  RWIX
  SYNC_SOC              00007940   00000010  00000006  0000000a  RWIX
  DMACLASRCSEL          00007980   00000040  0000001a  00000026  RWIX
  EPWM_XBAR             00007a00   00000040  00000040  00000000  RWIX
  CLB_XBAR              00007a40   00000040  00000000  00000040  RWIX
  OUTPUT_XBAR           00007a80   00000040  00000040  00000000  RWIX
  GPIOCTRL              00007c00   00000180  00000180  00000000  RWIX
  GPIODAT               00007f00   00000030  00000030  00000000  RWIX
  LS05SARAM             00008000   00003000  0000015f  00002ea1  RWIX
  RAMGS06               0000c000   00007000  0000587e  00001782  RWIX
  RAMGS7                00013000   00001000  00000000  00001000  RWIX
  RAMGS8                00014000   00001000  00000000  00001000  RWIX
  RAMGS9                00015000   00001000  00000000  00001000  RWIX
  RAMGS10               00016000   00001000  00000000  00001000  RWIX
  RAMGS11               00017000   00001000  00000000  00001000  RWIX
  RAMGS12               00018000   00001000  00000000  00001000  RWIX
  RAMGS13               00019000   00001000  00000000  00001000  RWIX
  RAMGS14               0001a000   00001000  00000000  00001000  RWIX
  RAMGS15               0001b000   00001000  00000000  00001000  RWIX
  CPU2TOCPU1RAM         0003f800   00000400  00000000  00000400  RWIX
  CPU1TOCPU2RAM         0003fc00   00000400  00000000  00000400  RWIX
  EMIF1                 00047000   00000800  00000070  00000790  RWIX
  EMIF2                 00047800   00000800  00000070  00000790  RWIX
  CANA                  00048000   00000800  00000000  00000800  RWIX
  CANB                  0004a000   00000800  00000000  00000800  RWIX
  IPC                   00050000   00000024  00000024  00000000  RWIX
  FLASHPUMPSEMAPHORE    00050024   00000002  00000002  00000000  RWIX
  DEV_CFG               0005d000   00000180  0000012e  00000052  RWIX
  ANALOG_SUBSYS         0005d180   00000080  00000048  00000038  RWIX
  CLK_CFG               0005d200   00000100  00000032  000000ce  RWIX
  CPU_SYS               0005d300   00000100  00000082  0000007e  RWIX
  ROMPREFETCH           0005e608   00000002  00000002  00000000  RWIX
  DCSM_Z1               0005f000   00000030  00000024  0000000c  RWIX
  DCSM_Z2               0005f040   00000030  00000024  0000000c  RWIX
  DCSM_COMMON           0005f070   00000010  00000008  00000008  RWIX
  MEMCFG                0005f400   00000080  00000080  00000000  RWIX
  EMIF1CONFIG           0005f480   00000020  00000020  00000000  RWIX
  EMIF2CONFIG           0005f4a0   00000020  00000020  00000000  RWIX
  ACCESSPROTECTION      0005f4c0   00000040  00000040  00000000  RWIX
  MEMORYERROR           0005f500   00000040  00000040  00000000  RWIX
  ROMWAITSTATE          0005f540   00000002  00000002  00000000  RWIX
  FLASH0_CTRL           0005f800   00000300  00000182  0000017e  RWIX
  FLASH0_ECC            0005fb00   00000040  00000028  00000018  RWIX
  DCSM_Z1_OTP           00078000   00000020  00000020  00000000  RWIX
  DCSM_Z2_OTP           00078200   00000020  00000020  00000000  RWIX


SECTION ALLOCATION MAP

 output                                  attributes/
section   page    origin      length       input sections
--------  ----  ----------  ----------   ----------------
.TI.ramfunc 
*          0    00080080    0000003f     RUN ADDR = 00008000
                  00080080    00000037     F2837xD_SysCtrl.obj (.TI.ramfunc)
                  000800b7    00000004     F2837xD_usDelay.obj (.TI.ramfunc)
                  000800bb    00000004     sysctl.obj (.TI.ramfunc)

.binit     0    00087d8c    0000000a     
                  00087d8c    0000000a     (.binit)

.cinit     0    0008b674    00000a51     
                  0008b674    0000083a     PMCU_BIOS_cpu1_p28FP.o28FP (.cinit)
                  0008beae    000000e4     Cmd_Task.obj (.cinit)
                  0008bf92    00000075     PMCU_GpioXint.obj (.cinit)
                  0008c007    00000055     EQEP_PMSM_Control.obj (.cinit)
                  0008c05c    0000002a     Can_Task.obj (.cinit)
                  0008c086    00000010     PMCU_PI_Task.obj (.cinit)
                  0008c096    0000000e     rts2800_fpu32.lib : exit.obj (.cinit)
                  0008c0a4    00000009     uartstdio.obj (.cinit)
                  0008c0ad    00000005     rts2800_fpu32.lib : _lock.obj (.cinit:__lock)
                  0008c0b2    00000005                       : _lock.obj (.cinit:__unlock)
                  0008c0b7    00000004     PMCU_Emif.obj (.cinit)
                  0008c0bb    00000004     rts2800_fpu32.lib : errno.obj (.cinit)
                  0008c0bf    00000004     ustdlib.obj (.cinit)
                  0008c0c3    00000002     --HOLE-- [fill = 0]

.pinit     0    00080080    00000000     UNINITIALIZED

.ti_catalog_c2800_initF2837x_begin 
*          0    00080000    00000002     
                  00080000    00000002     Boot.a28FP : Boot_asm.o28FP (.ti_catalog_c2800_initF2837x_begin)

.text:ti_catalog_c2800_initF2837x_flashfuncs 
*          0    00080004    00000027     RUN ADDR = 0000b000
                  00080004    00000027     Boot.a28FP : Boot.o28FP (.text:ti_catalog_c2800_initF2837x_flashfuncs:_ti_catalog_c2800_initF2837x_Boot_initFlash)

.text.1    0    000800c0    00001f40     
                  000800c0    00000bd9     rts2800_fpu32.lib : _printfi.obj (.text)
                  00080c99    000007d5     Can_Task.obj (.text)
                  0008146e    000006ba     Cmd_Task.obj (.text)
                  00081b28    00000347     F2837xD_SysCtrl.obj (.text)
                  00081e6f    00000181     sysbios.a28FP : BIOS.obj (.text:_ti_sysbios_heaps_HeapMem_allocUnprotected__E)
                  00081ff0    00000010     PMCU_BIOS_cpu1_p28FP.o28FP (.text:_ti_sysbios_BIOS_rtsLock__I)

.text.2    0    00082000    00002000     
                  00082000    000005da     ustdlib.obj (.text)
                  000825da    0000052e     can.obj (.text)
                  00082b08    000002e9     uart.obj (.text)
                  00082df1    0000027c     rts2800_fpu32.lib : trgdrv.obj (.text)
                  0008306d    00000267     uartstdio.obj (.text)
                  000832d4    0000025f     ti.targets.rts2800.a28FP : System.o28FP (.text:_xdc_runtime_System_doPrint__I)
                  00083533    00000244     F2837xD_Gpio.obj (.text)
                  00083777    00000243     sysctl.obj (.text)
                  000839ba    00000232     sysbios.a28FP : BIOS.obj (.text:_ti_sysbios_knl_Event_pend__E)
                  00083bec    000001eb                   : BIOS.obj (.text:_ti_sysbios_knl_Semaphore_pend__E)
                  00083dd7    000001ca     interrupt.obj (.text)
                  00083fa1    0000005e     SpiA_ExtTemp_Task.obj (.text)
                  00083fff    00000001     sysbios.a28FP : BIOS.obj (.text:_ti_sysbios_BIOS_linkedWithIncorrectBootLibrary__E)

.text.3    0    00084000    00002000     
                  00084000    000001a1     sysbios.a28FP : BIOS.obj (.text:_ti_sysbios_heaps_HeapMem_freeUnprotected__E)
                  000841a1    00000145     PMCU_PI_Task.obj (.text)
                  000842e6    00000135     sysbios.a28FP : BIOS.obj (.text:_ti_sysbios_knl_Task_sleep__E)
                  0008441b    0000010a     PMCU_BIOS_cpu1_p28FP.o28FP (.text:_xdc_runtime_System_printfExtend__I)
                  00084525    00000108     PMCU_GpioXint.obj (.text)
                  0008462d    00000107     rts2800_fpu32.lib : ll_div.obj (.text)
                  00084734    000000fd     F2837xD_EPwm.obj (.text)
                  00084831    000000ed     sysbios.a28FP : BIOS.obj (.text:_ti_sysbios_heaps_HeapMem_Instance_init__E)
                  0008491e    000000e1     AD7689_ExtADC.obj (.text)
                  000849ff    000000e0     sysbios.a28FP : BIOS.obj (.text:_ti_sysbios_family_c28_Hwi_clearInterrupt__E)
                  00084adf    000000df     ti.targets.rts2800.a28FP : LoggerBuf.o28FP (.text:_xdc_runtime_LoggerBuf_write8__E)
                  00084bbe    000000dd     F2837xD_Adc.obj (.text)
                  00084c9b    000000d8     AdcC_Handler.obj (.text)
                  00084d73    000000d7     ti.targets.rts2800.a28FP : Core-mem.o28FP (.text:_xdc_runtime_Core_createObject__I)
                  00084e4a    000000ce     AdcD_Handler.obj (.text)
                  00084f18    000000ca     SpiB_LowDriver.obj (.text)
                  00084fe2    000000ca     sysbios.a28FP : BIOS.obj (.text:_ti_sysbios_knl_Event_post__E)
                  000850ac    000000c0                   : BIOS.obj (.text:_ti_sysbios_knl_Semaphore_post__E)
                  0008516c    000000be     SpiC_LowDriver.obj (.text)
                  0008522a    000000bc     rts2800_fpu32.lib : s_scalbn.obj (.text)
                  000852e6    000000b8     PMCU_Emif.obj (.text)
                  0008539e    000000b6     sysbios.a28FP : BIOS.obj (.text:_ti_sysbios_knl_Clock_workFunc__E)
                  00085454    000000b5     AdcA_Handler.obj (.text)
                  00085509    000000b5     AdcB_Handler.obj (.text)
                  000855be    000000af     sysbios.a28FP : BIOS.obj (.text:_ti_sysbios_knl_Swi_run__I)
                  0008566d    000000ae                   : BIOS.obj (.text:_ti_sysbios_family_c28_Hwi_dispatchCore__I)
                  0008571b    000000a5     ti.targets.rts2800.a28FP : Error.o28FP (.text:_xdc_runtime_Error_policyDefault__E)
                  000857c0    000000a2                              : Core-smem.o28FP (.text:_xdc_runtime_Core_constructObject__I)
                  00085862    0000009d     F2837xD_Spi.obj (.text)
                  000858ff    0000009c     rts2800_fpu32.lib : fd_add.obj (.text)
                  0008599b    0000009b     sysbios.a28FP : c28_Hwi_disp_asm.obj (.text:_ti_sysbios_family_c28_Hwi_dispatch)
                  00085a36    00000095     ti.targets.rts2800.a28FP : LoggerBuf.o28FP (.text:_xdc_runtime_LoggerBuf_write4__E)
                  00085acb    00000094     Ipc_Handler.obj (.text)
                  00085b5f    00000001     PMCU_BIOS_cpu1_p28FP.o28FP (.text:_ti_sysbios_BIOS_nullFunc__I)
                  00085b60    00000094     rts2800_fpu32.lib : trgmsg.obj (.text)
                  00085bf4    0000008e     sysbios.a28FP : BIOS.obj (.text:_ti_sysbios_family_c28_Hwi_enableInterrupt__E)
                  00085c82    0000008b     rts2800_fpu32.lib : fd_div.obj (.text)
                  00085d0d    00000084     SpiB_ExtADC_Task.obj (.text)
                  00085d91    00000083     SpiA_LowDriver.obj (.text)
                  00085e14    00000083     rts2800_fpu32.lib : fd_mpy.obj (.text)
                  00085e97    00000081     sysbios.a28FP : BIOS.obj (.text:_ti_sysbios_family_c28_Hwi_disableInterrupt__E)
                  00085f18    0000007e                   : BIOS.obj (.text:_ti_sysbios_family_c28_Hwi_disablePIEIER__E)
                  00085f96    00000066                   : BIOS.obj (.text:_ti_sysbios_family_c28_Timer_stopAndClear__I)
                  00085ffc    00000004     PMCU_BIOS_cpu1_p28FP.o28FP (.text:.bootCodeSection:_ti_catalog_c2800_initF2837x_Boot_init)

.text.4    0    00086000    00001d70     
                  00086000    0000007d     sysbios.a28FP : BIOS.obj (.text:_ti_sysbios_family_c28_Hwi_enablePIEIER__E)
                  0008607d    0000007d     ti.targets.rts2800.a28FP : Startup.o28FP (.text:_xdc_runtime_Startup_startMods__I)
                  000860fa    0000007b                              : Text.o28FP (.text:_xdc_runtime_Text_putSite__E)
                  00086175    00000076     PMCU_Main.obj (.text)
                  000861eb    00000073     EPwm_Handler.obj (.text)
                  0008625e    00000073     sysbios.a28FP : BIOS.obj (.text:_ti_sysbios_knl_Task_checkStacks__E)
                  000862d1    00000071                   : BIOS.obj (.text:_ti_sysbios_knl_Task_startCore__E)
                  00086342    00000070                   : BIOS.obj (.text:_ti_sysbios_gates_GateMutex_enter__E)
                  000863b2    0000006e                   : BIOS.obj (.text:_ti_sysbios_knl_Task_schedule__I)
                  00086420    0000006d     AD5764_ExtDAC.obj (.text)
                  0008648d    00000063     boot.a28FP : boot_cg.o28FP (.text)
                  000864f0    00000060     sysbios.a28FP : BIOS.obj (.text:_ti_sysbios_knl_Swi_post__E)
                  00086550    00000060                   : BIOS.obj (.text:_ti_sysbios_knl_Task_blockI__E)
                  000865b0    0000005a     rts2800_fpu32.lib : s_frexp.obj (.text)
                  0008660a    00000057     sysbios.a28FP : BIOS.obj (.text:_ti_sysbios_knl_Task_exit__E)
                  00086661    00000054                   : BIOS.obj (.text:_ti_sysbios_family_c28_Timer_setPeriodMicroSecs__E)
                  000866b5    00000051                   : BIOS.obj (.text:_ti_sysbios_knl_Task_unblockI__E)
                  00086706    00000051     ti.targets.rts2800.a28FP : Core-mem.o28FP (.text:_xdc_runtime_Core_deleteObject__I)
                  00086757    0000004e                              : Memory.o28FP (.text:_xdc_runtime_Memory_alloc__E)
                  000867a5    0000004c                              : Text.o28FP (.text:_xdc_runtime_Text_putLab__E)
                  000867f1    0000004b     sysbios.a28FP : BIOS.obj (.text:_ti_sysbios_heaps_HeapMem_alloc__E)
                  0008683c    0000004b                   : BIOS.obj (.text:_ti_sysbios_knl_Task_postInit__I)
                  00086887    00000049                   : BIOS.obj (.text:_ti_sysbios_knl_Mailbox_post__E)
                  000868d0    00000049     cmdline.obj (.text)
                  00086919    00000047     sysbios.a28FP : BIOS.obj (.text:_ti_sysbios_family_c28_Hwi_Module_startup__E)
                  00086960    00000046     SpiC_ExtDAC_Task.obj (.text)
                  000869a6    00000046     rts2800_fpu32.lib : cpy_tbl.obj (.text)
                  000869ec    00000043     sysbios.a28FP : BIOS.obj (.text:_ti_sysbios_family_c28_Timer_postInit__I)
                  00086a2f    00000043     ti.targets.rts2800.a28FP : Error.o28FP (.text:_xdc_runtime_Error_setX__E)
                  00086a72    00000042     sysbios.a28FP : BIOS.obj (.text:_ti_sysbios_family_c28_Hwi_unPluggedInterrupt__I)
                  00086ab4    00000042     ti.targets.rts2800.a28FP : Core-params.o28FP (.text:_xdc_runtime_Core_assignParams__I)
                  00086af6    00000040                              : System.o28FP (.text:_xdc_runtime_System_formatNum__I)
                  00086b36    0000003f                              : LoggerBuf.o28FP (.text:_xdc_runtime_LoggerBuf_setFilterLevel__E)
                  00086b75    0000003e     sysbios.a28FP : BIOS.obj (.text:_ti_sysbios_knl_Mailbox_pend__E)
                  00086bb3    0000003e                   : BIOS.obj (.text:_ti_sysbios_knl_Swi_restoreHwi__E)
                  00086bf1    0000003c     ti.targets.rts2800.a28FP : LoggerBuf.o28FP (.text:_xdc_runtime_LoggerBuf_getFilterLevel__E)
                  00086c2d    0000003a     sysbios.a28FP : BIOS.obj (.text:_ti_sysbios_family_c28_TaskSupport_start__E)
                  00086c67    0000003a     ti.targets.rts2800.a28FP : Text.o28FP (.text:_xdc_runtime_Text_putMod__E)
                  00086ca1    00000039     sysbios.a28FP : BIOS.obj (.text:_ti_sysbios_knl_Semaphore_Instance_init__E)
                  00086cda    00000039     ti.targets.rts2800.a28FP : Text.o28FP (.text:_xdc_runtime_Text_visitRope2__I)
                  00086d13    00000038     PMCU_BIOS_cpu1_p28FP.o28FP (.text:_xdc_runtime_LoggerBuf_Object__create__S)
                  00086d4b    00000036     PMCU_Mgmt_Task.obj (.text)
                  00086d81    00000036     sysbios.a28FP : BIOS.obj (.text:_ti_sysbios_knl_Clock_logTick__E)
                  00086db7    00000036     ti.targets.rts2800.a28FP : Error.o28FP (.text:_xdc_runtime_Error_print__E)
                  00086ded    00000035                              : Startup.o28FP (.text:_xdc_runtime_Startup_exec__E)
                  00086e22    00000034     PMCU_BIOS_cpu1_p28FP.o28FP (.text:_ti_sysbios_BIOS_rtsUnlock__I)
                  00086e56    00000032     sysbios.a28FP : BIOS.obj (.text:_ti_sysbios_knl_Task_Module_startup__E)
                  00086e88    00000032     ti.targets.rts2800.a28FP : Assert.o28FP (.text:_xdc_runtime_Assert_raise__I)
                  00086eba    00000032                              : LoggerBuf.o28FP (.text:_xdc_runtime_LoggerBuf_Instance_init__E)
                  00086eec    00000032     rts2800_fpu32.lib : sprintf.obj (.text)
                  00086f1e    00000031     sysbios.a28FP : BIOS.obj (.text:_ti_sysbios_family_c28_Timer_getFreq__E)
                  00086f4f    00000031     rts2800_fpu32.lib : atoi.obj (.text)
                  00086f80    0000002e     sysbios.a28FP : BIOS.obj (.text:_ti_sysbios_knl_Swi_runLoop__I)
                  00086fae    0000002e                   : BIOS.obj (.text:_ti_sysbios_knl_Swi_schedule__I)
                  00086fdc    0000002e     rts2800_fpu32.lib : ltoa.obj (.text)
                  0008700a    0000002d     sysbios.a28FP : BIOS.obj (.text:_ti_sysbios_heaps_HeapMem_getStats__E)
                  00087037    0000002c                   : BIOS.obj (.text:_ti_sysbios_family_c28_Hwi_getStackInfo__E)
                  00087063    0000002c                   : BIOS.obj (.text:_ti_sysbios_family_c28_Timer_start__E)
                  0008708f    0000002b                   : BIOS.obj (.text:_ti_sysbios_knl_Mailbox_Module_startup__E)
                  000870ba    0000002a     ti.targets.rts2800.a28FP : Text.o28FP (.text:_xdc_runtime_Text_xprintf__I)
                  000870e4    0000002a     rts2800_fpu32.lib : fd_cmp.obj (.text)
                  0008710e    0000002a                       : l_div.obj (.text)
                  00087138    00000029                       : exit.obj (.text)
                  00087161    00000028     ti.targets.rts2800.a28FP : SysMin.o28FP (.text:_xdc_runtime_SysMin_flush__E)
                  00087189    00000027     sysbios.a28FP : BIOS.obj (.text:_ti_sysbios_heaps_HeapMem_free__E)
                  000871b0    00000027                   : BIOS.obj (.text:_ti_sysbios_heaps_HeapMem_init__I)
                  000871d7    00000025                   : c28_TaskSupport_asm.obj (.text:_ti_sysbios_family_c28_TaskSupport_buildTaskStack)
                  000871fc    00000024     rts2800_fpu32.lib : s_copysign.obj (.text)
                  00087220    00000023     ti.targets.rts2800.a28FP : System.o28FP (.text:_xdc_runtime_System_processAtExit__E)
                  00087243    00000022     rts2800_fpu32.lib : i_div.obj (.text)
                  00087265    00000021     sysbios.a28FP : BIOS.obj (.text:_ti_sysbios_knl_Task_allBlockedFunction__I)
                  00087286    00000021     ti.targets.rts2800.a28FP : System.o28FP (.text:_xdc_runtime_System_atexit__E)
                  000872a7    00000021     rts2800_fpu32.lib : fd_toi.obj (.text)
                  000872c8    00000020     sysbios.a28FP : BIOS.obj (.text:_ti_sysbios_family_c28_Timer_setPrescale__E)
                  000872e8    0000001f     PMCU_BIOS_cpu1_p28FP.o28FP (.text:_ti_sysbios_gates_GateHwi_Object__create__S)
                  00087307    0000001f     PMCU_BIOS_cpu1_p28FP.o28FP (.text:_ti_sysbios_gates_GateMutex_Object__create__S)
                  00087326    0000001f     PMCU_BIOS_cpu1_p28FP.o28FP (.text:_ti_sysbios_heaps_HeapMem_Object__create__S)
                  00087345    0000001f     rts2800_fpu32.lib : fd_tol.obj (.text)
                  00087364    0000001e     ti.targets.rts2800.a28FP : SysMin.o28FP (.text:_xdc_runtime_SysMin_putch__E)
                  00087382    0000001e     rts2800_fpu32.lib : ll_cmp.obj (.text)
                  000873a0    0000001e                       : memcpy.obj (.text)
                  000873be    0000001d     sysbios.a28FP : c28_TaskSupport_asm.obj (.text:_ti_sysbios_family_c28_TaskSupport_swap__E)
                  000873db    0000001d     ti.targets.rts2800.a28FP : LoggerBuf.o28FP (.text:_xdc_runtime_LoggerBuf_filterOutEvent__I)
                  000873f8    0000001d     rts2800_fpu32.lib : i_tofd.obj (.text)
                  00087415    0000001c     sysbios.a28FP : BIOS.obj (.text:_ti_sysbios_hal_Hwi_checkStack)
                  00087431    0000001c     Ipc_Handler.obj (.text:retain)
                  0008744d    0000001c     rts2800_fpu32.lib : fs_tofd.obj (.text)
                  00087469    0000001c                       : l_tofd.obj (.text)
                  00087485    0000001b     sysbios.a28FP : c28_Hwi_asm.obj (.text:_ti_sysbios_family_c28_Hwi_switchAndDispatch__I)
                  000874a0    0000001b                   : BIOS.obj (.text:_ti_sysbios_hal_Hwi_initStack)
                  000874bb    0000001b     PMCU_BIOS_cpu1_p28FP.o28FP (.text:_ti_sysbios_knl_Semaphore_construct)
                  000874d6    0000001b     sysbios.a28FP : BIOS.obj (.text:_ti_sysbios_knl_Task_processVitalTaskFlag__I)
                  000874f1    0000001b     PMCU_BIOS_cpu1_p28FP.o28FP (.text:_xdc_runtime_SysMin_output__I)
                  0008750c    0000001a     sysbios.a28FP : BIOS.obj (.text:_ti_sysbios_knl_Clock_addI__E)
                  00087526    0000001a     ti.targets.rts2800.a28FP : Core-label.o28FP (.text:_xdc_runtime_Core_assignLabel__I)
                  00087540    0000001a                              : LoggerBuf.o28FP (.text:_xdc_runtime_LoggerBuf_Module_startup__E)
                  0008755a    0000001a     rts2800_fpu32.lib : cpy_utils.obj (.text)
                  00087574    00000019     PMCU_BIOS_cpu1_p28FP.o28FP (.text:_ti_sysbios_family_c28_Hwi_Object__get__S)
                  0008758d    00000019     sysbios.a28FP : BIOS.obj (.text:_ti_sysbios_knl_Event_pendTimeout__I)
                  000875a6    00000019                   : BIOS.obj (.text:_ti_sysbios_knl_Mailbox_postInit__I)
                  000875bf    00000019     PMCU_BIOS_cpu1_p28FP.o28FP (.text:_ti_sysbios_knl_Queue_Object__get__S)
                  000875d8    00000019     PMCU_BIOS_cpu1_p28FP.o28FP (.text:_ti_sysbios_knl_Queue_construct)
                  000875f1    00000019     sysbios.a28FP : BIOS.obj (.text:_ti_sysbios_knl_Semaphore_pendTimeout__I)
                  0008760a    00000019                   : BIOS.obj (.text:_ti_sysbios_knl_Swi_restore__E)
                  00087623    00000019     ti.targets.rts2800.a28FP : Memory.o28FP (.text:_xdc_runtime_Memory_valloc__E)
                  0008763c    00000019                              : System.o28FP (.text:_xdc_runtime_System_avprintf__E)
                  00087655    00000019                              : System.o28FP (.text:_xdc_runtime_System_putchar__I)
                  0008766e    00000019     rts2800_fpu32.lib : args_main.obj (.text)
                  00087687    00000018     sysbios.a28FP : c28_Hwi_asm.obj (.text:_ti_sysbios_family_xxx_Hwi_switchAndRunFunc)
                  0008769f    00000018     ti.targets.rts2800.a28FP : LoggerBuf.o28FP (.text:_xdc_runtime_LoggerBuf_reset__E)
                  000876b7    00000018                              : System.o28FP (.text:_xdc_runtime_System_vprintf__E)
                  000876cf    00000018                              : Text.o28FP (.text:_xdc_runtime_Text_printVisFxn__I)
                  000876e7    00000018     rts2800_fpu32.lib : ll_aox.obj (.text)
                  000876ff    00000017     PMCU_BIOS_cpu1_p28FP.o28FP (.text:_ti_sysbios_BIOS_atExitFunc__I)
                  00087716    00000017     sysbios.a28FP : BIOS.obj (.text:_ti_sysbios_family_c28_Timer_startup__E)
                  0008772d    00000017     PMCU_BIOS_cpu1_p28FP.o28FP (.text:_ti_sysbios_heaps_HeapMem_Object__get__S)
                  00087744    00000017     PMCU_BIOS_cpu1_p28FP.o28FP (.text:_ti_sysbios_knl_Clock_doTick__I)
                  0008775b    00000017     PMCU_BIOS_cpu1_p28FP.o28FP (.text:_ti_sysbios_knl_Mailbox_Object__get__S)
                  00087772    00000017     PMCU_BIOS_cpu1_p28FP.o28FP (.text:_ti_sysbios_knl_Swi_Object__get__S)
                  00087789    00000017     PMCU_BIOS_cpu1_p28FP.o28FP (.text:_ti_sysbios_knl_Task_Object__get__S)
                  000877a0    00000017     PMCU_BIOS_cpu1_p28FP.o28FP (.text:_xdc_runtime_LoggerBuf_Object__get__S)
                  000877b7    00000017     ti.targets.rts2800.a28FP : SysMin.o28FP (.text:_xdc_runtime_SysMin_abort__E)
                  000877ce    00000016     sysbios.a28FP : BIOS.obj (.text:_ti_sysbios_family_c28_Timer_Module_startup__E)
                  000877e4    00000016                   : BIOS.obj (.text:_ti_sysbios_knl_Task_restore__E)
                  000877fa    00000015     PMCU_BIOS_cpu1_p28FP.o28FP (.text:_ti_sysbios_BIOS_startFunc__I)
                  0008780f    00000015     sysbios.a28FP : BIOS.obj (.text:_ti_sysbios_knl_Swi_Module_startup__E)
                  00087824    00000015     ti.targets.rts2800.a28FP : Text.o28FP (.text:_xdc_runtime_Text_cordText__E)
                  00087839    00000014     sysbios.a28FP : BIOS.obj (.text:_ti_sysbios_knl_Idle_run__E)
                  0008784d    00000014                   : BIOS.obj (.text:_ti_sysbios_knl_Semaphore_Instance_finalize__E)
                  00087861    00000013     PMCU_BIOS_cpu1_p28FP.o28FP (.text:_ti_sysbios_BIOS_errorRaiseHook__I)
                  00087874    00000013     sysbios.a28FP : BIOS.obj (.text:_ti_sysbios_family_c28_Timer_checkOverflow__I)
                  00087887    00000013     PMCU_BIOS_cpu1_p28FP.o28FP (.text:_ti_sysbios_gates_GateMutex_Object__delete__S)
                  0008789a    00000013     sysbios.a28FP : BIOS.obj (.text:_ti_sysbios_knl_Event_checkEvents__I)
                  000878ad    00000012     PMCU_BIOS_cpu1_p28FP.o28FP (.text:_ti_sysbios_family_c28_Hwi_disableIER__E)
                  000878bf    00000012     PMCU_BIOS_cpu1_p28FP.o28FP (.text:_ti_sysbios_gates_GateHwi_Object__delete__S)
                  000878d1    00000012     PMCU_BIOS_cpu1_p28FP.o28FP (.text:_ti_sysbios_heaps_HeapMem_Object__delete__S)
                  000878e3    00000012     sysbios.a28FP : BIOS.obj (.text:_ti_sysbios_knl_Clock_Module_startup__E)
                  000878f5    00000012     PMCU_BIOS_cpu1_p28FP.o28FP (.text:_xdc_runtime_LoggerBuf_Object__delete__S)
                  00087907    00000011     PMCU_BIOS_cpu1_p28FP.o28FP (.text:_ti_sysbios_gates_GateHwi_Handle__label__S)
                  00087918    00000011     PMCU_BIOS_cpu1_p28FP.o28FP (.text:_ti_sysbios_gates_GateMutex_Handle__label__S)
                  00087929    00000011     PMCU_BIOS_cpu1_p28FP.o28FP (.text:_ti_sysbios_heaps_HeapMem_Handle__label__S)
                  0008793a    00000011     ti.targets.rts2800.a28FP : Error.o28FP (.text:_xdc_runtime_Error_raiseX__E)
                  0008794b    00000011     PMCU_BIOS_cpu1_p28FP.o28FP (.text:_xdc_runtime_LoggerBuf_Handle__label__S)
                  0008795c    00000010     PMCU_BIOS_cpu1_p28FP.o28FP (.text:_ti_sysbios_family_c28_Hwi_enableIER__E)
                  0008796c    00000010     sysbios.a28FP : BIOS.obj (.text:_ti_sysbios_family_c28_Timer_stop__E)
                  0008797c    00000010                   : BIOS.obj (.text:_ti_sysbios_knl_Task_restoreHwi__E)
                  0008798c    0000000f                   : BIOS.obj (.text:_ti_sysbios_gates_GateMutex_Instance_init__E)
                  0008799b    0000000f     PMCU_BIOS_cpu1_p28FP.o28FP (.text:_ti_sysbios_knl_Semaphore_Object__destruct__S)
                  000879aa    0000000f     ti.targets.rts2800.a28FP : LoggerBuf.o28FP (.text:_xdc_runtime_LoggerBuf_write2__E)
                  000879b9    0000000f     PMCU_BIOS_cpu1_p28FP.o28FP (.text:_xdc_runtime_Text_visitRope__I)
                  000879c8    0000000f     interrupt.obj (.text:retain)
                  000879d7    0000000e     sysbios.a28FP : BIOS.obj (.text:_ti_sysbios_family_c28_f2837x_TimestampProvider_get64__E)
                  000879e5    0000000e     PMCU_BIOS_cpu1_p28FP.o28FP (.text:_ti_sysbios_knl_Queue_Object__destruct__S)
                  000879f3    0000000e     PMCU_BIOS_cpu1_p28FP.o28FP (.text:_xdc_runtime_IHeap_alloc)
                  00087a01    0000000e     ti.targets.rts2800.a28FP : Registry.o28FP (.text:_xdc_runtime_Registry_findById__E)
                  00087a0f    0000000e                              : SysMin.o28FP (.text:_xdc_runtime_SysMin_Module_startup__E)
                  00087a1d    0000000e     rts2800_fpu32.lib : fd_sub.obj (.text)
                  00087a2b    0000000d     PMCU_BIOS_cpu1_p28FP.o28FP (.text:_ti_sysbios_BIOS_registerRTSLock__I)
                  00087a38    0000000d     PMCU_BIOS_cpu1_p28FP.o28FP (.text:_ti_sysbios_BIOS_removeRTSLock__I)
                  00087a45    0000000d     sysbios.a28FP : BIOS.obj (.text:_ti_sysbios_family_c28_Hwi_dispatchC__I)
                  00087a52    0000000d     PMCU_BIOS_cpu1_p28FP.o28FP (.text:_ti_sysbios_family_c28_Hwi_restoreIER__E)
                  00087a5f    0000000d     PMCU_BIOS_cpu1_p28FP.o28FP (.text:_ti_sysbios_knl_Task_SupportProxy_start__E)
                  00087a6c    0000000d     sysbios.a28FP : BIOS.obj (.text:_ti_sysbios_knl_Task_enter__I)
                  00087a79    0000000d                   : BIOS.obj (.text:_ti_sysbios_knl_Task_sleepTimeout__I)
                  00087a86    0000000d     ti.targets.rts2800.a28FP : Error.o28FP (.text:_xdc_runtime_Error_check__E)
                  00087a93    0000000d                              : LoggerBuf.o28FP (.text:_xdc_runtime_LoggerBuf_write1__E)
                  00087aa0    0000000d     PMCU_BIOS_cpu1_p28FP.o28FP (.text:_xdc_runtime_Memory_HeapProxy_alloc__E)
                  00087aad    0000000d     ti.targets.rts2800.a28FP : System.o28FP (.text:_xdc_runtime_System_abort__E)
                  00087aba    0000000d     rts2800_fpu32.lib : memccpy.obj (.text)
                  00087ac7    0000000c     PMCU_BIOS_cpu1_p28FP.o28FP (.text:_ti_sysbios_BIOS_exitFunc__I)
                  00087ad3    0000000c     sysbios.a28FP : BIOS.obj (.text:_ti_sysbios_gates_GateMutex_leave__E)
                  00087adf    0000000c                   : BIOS.obj (.text:_ti_sysbios_knl_Queue_get__E)
                  00087aeb    0000000c                   : BIOS.obj (.text:_ti_sysbios_knl_Queue_put__E)
                  00087af7    0000000c                   : BIOS.obj (.text:_ti_sysbios_knl_Task_enabled__E)
                  00087b03    0000000c     ti.targets.rts2800.a28FP : Memory.o28FP (.text:_xdc_runtime_Memory_free__E)
                  00087b0f    0000000c     PMCU_BIOS_cpu1_p28FP.o28FP (.text:_xdc_runtime_System_aprintf__E)
                  00087b1b    0000000c     PMCU_BIOS_cpu1_p28FP.o28FP (.text:_xdc_runtime_System_printf__E)
                  00087b27    0000000c     ti.targets.rts2800.a28FP : Text.o28FP (.text:_xdc_runtime_Text_ropeText__E)
                  00087b33    0000000c     rts2800_fpu32.lib : memset.obj (.text)
                  00087b3f    0000000c                       : strchr.obj (.text)
                  00087b4b    0000000b     PMCU_BIOS_cpu1_p28FP.o28FP (.text:_ti_sysbios_family_c28_Hwi_Module__startupDone__F)
                  00087b56    0000000b     PMCU_BIOS_cpu1_p28FP.o28FP (.text:_ti_sysbios_family_c28_Timer_Module__startupDone__F)
                  00087b61    0000000b     sysbios.a28FP : BIOS.obj (.text:_ti_sysbios_knl_Task_unblock__E)
                  00087b6c    0000000b     ti.targets.rts2800.a28FP : LoggerBuf.o28FP (.text:_xdc_runtime_LoggerBuf_Instance_finalize__E)
                  00087b77    0000000b                              : LoggerBuf.o28FP (.text:_xdc_runtime_LoggerBuf_write0__E)
                  00087b82    0000000b     PMCU_BIOS_cpu1_p28FP.o28FP (.text:_xdc_runtime_Startup_exec__I)
                  00087b8d    0000000b     ti.targets.rts2800.a28FP : SysMin.o28FP (.text:_xdc_runtime_SysMin_exit__E)
                  00087b98    0000000b                              : System.o28FP (.text:_xdc_runtime_System_exit__E)
                  00087ba3    0000000b     rts2800_fpu32.lib : u_div.obj (.text)
                  00087bae    0000000a     PMCU_BIOS_cpu1_p28FP.o28FP (.text:_xdc_runtime_IHeap_free)
                  00087bb8    0000000a     rts2800_fpu32.lib : strcmp.obj (.text)
                  00087bc2    00000009     sysbios.a28FP : BIOS.obj (.text:_ti_sysbios_family_c28_TaskSupport_checkStack__E)
                  00087bcb    00000009                   : c28_TaskSupport_asm.obj (.text:_ti_sysbios_family_c28_TaskSupport_glue)
                  00087bd4    00000009                   : BIOS.obj (.text:_ti_sysbios_hal_Hwi_Module_startup__E)
                  00087bdd    00000009                   : BIOS.obj (.text:_ti_sysbios_hal_Timer_Module_startup__E)
                  00087be6    00000009     ti.targets.rts2800.a28FP : System.o28FP (.text:_xdc_runtime_System_vsnprintf__E)
                  00087bef    00000009     rts2800_fpu32.lib : _lock.obj (.text)
                  00087bf8    00000009                       : fd_neg.obj (.text)
                  00087c01    00000008     Boot.a28FP : Boot.o28FP (.text:.bootCodeSection:_ti_catalog_c2800_initF2837x_Boot_initSharedRAMs)
                  00087c09    00000008     sysbios.a28FP : BIOS.obj (.text:_ti_sysbios_BIOS_setThreadType__E)
                  00087c11    00000008                   : BIOS.obj (.text:_ti_sysbios_gates_GateMutex_Instance_finalize__E)
                  00087c19    00000008     PMCU_BIOS_cpu1_p28FP.o28FP (.text:_ti_sysbios_knl_Clock_Module_State_clockQ)
                  00087c21    00000008     PMCU_BIOS_cpu1_p28FP.o28FP (.text:_xdc_runtime_Memory_HeapProxy_free__E)
                  00087c29    00000008     ti.targets.rts2800.a28FP : Memory.o28FP (.text:_xdc_runtime_Memory_calloc__E)
                  00087c31    00000008                              : SysMin.o28FP (.text:_xdc_runtime_SysMin_ready__E)
                  00087c39    00000008     rts2800_fpu32.lib : strlen.obj (.text)
                  00087c41    00000007     PMCU_BIOS_cpu1_p28FP.o28FP (.text:.bootCodeSection:_ti_catalog_c2800_initF2837x_Boot_initStartup)
                  00087c48    00000007     PMCU_BIOS_cpu1_p28FP.o28FP (.text:_ti_sysbios_BIOS_RtsGateProxy_leave__E)
                  00087c4f    00000007     PMCU_BIOS_cpu1_p28FP.o28FP (.text:_ti_sysbios_hal_Hwi_HwiProxy_getStackInfo__E)
                  00087c56    00000007     PMCU_BIOS_cpu1_p28FP.o28FP (.text:_ti_sysbios_heaps_HeapMem_Module_GateProxy_leave__E)
                  00087c5d    00000007     sysbios.a28FP : BIOS.obj (.text:_ti_sysbios_knl_Event_sync__E)
                  00087c64    00000007                   : BIOS.obj (.text:_ti_sysbios_knl_Queue_empty__E)
                  00087c6b    00000007     PMCU_BIOS_cpu1_p28FP.o28FP (.text:_ti_sysbios_knl_Task_SupportProxy_checkStack__E)
                  00087c72    00000007     PMCU_BIOS_cpu1_p28FP.o28FP (.text:_ti_sysbios_knl_Task_SupportProxy_swap__E)
                  00087c79    00000007     ti.targets.rts2800.a28FP : Error.o28FP (.text:_xdc_runtime_Error_init__E)
                  00087c80    00000007     PMCU_BIOS_cpu1_p28FP.o28FP (.text:_xdc_runtime_LoggerBuf_Module_GateProxy_leave__E)
                  00087c87    00000007     PMCU_BIOS_cpu1_p28FP.o28FP (.text:_xdc_runtime_System_Module_GateProxy_leave__E)
                  00087c8e    00000006     PMCU_BIOS_cpu1_p28FP.o28FP (.text:_ti_sysbios_BIOS_RtsGateProxy_enter__E)
                  00087c94    00000006     sysbios.a28FP : BIOS.obj (.text:_ti_sysbios_BIOS_start__E)
                  00087c9a    00000006                   : c28_IntrinsicsSupport_asm.obj (.text:_ti_sysbios_family_c28_IntrinsicsSupport_maxbit__E)
                  00087ca0    00000006     PMCU_BIOS_cpu1_p28FP.o28FP (.text:_ti_sysbios_heaps_HeapMem_Module_GateProxy_enter__E)
                  00087ca6    00000006     PMCU_BIOS_cpu1_p28FP.o28FP (.text:_ti_sysbios_heaps_HeapMem_Module_GateProxy_query__E)
                  00087cac    00000006     PMCU_BIOS_cpu1_p28FP.o28FP (.text:_ti_sysbios_knl_Clock_TimerProxy_getMaxTicks__E)
                  00087cb2    00000006     PMCU_BIOS_cpu1_p28FP.o28FP (.text:_ti_sysbios_knl_Queue_destruct)
                  00087cb8    00000006     PMCU_BIOS_cpu1_p28FP.o28FP (.text:_ti_sysbios_knl_Semaphore_destruct)
                  00087cbe    00000006     sysbios.a28FP : BIOS.obj (.text:_ti_sysbios_knl_Swi_disable__E)
                  00087cc4    00000006                   : BIOS.obj (.text:_ti_sysbios_knl_Task_disable__E)
                  00087cca    00000006     ti.targets.rts2800.a28FP : Gate.o28FP (.text:_xdc_runtime_Gate_enterSystem__E)
                  00087cd0    00000006                              : Gate.o28FP (.text:_xdc_runtime_Gate_leaveSystem__E)
                  00087cd6    00000006     PMCU_BIOS_cpu1_p28FP.o28FP (.text:_xdc_runtime_LoggerBuf_Module_GateProxy_enter__E)
                  00087cdc    00000006     PMCU_BIOS_cpu1_p28FP.o28FP (.text:_xdc_runtime_LoggerBuf_TimestampProxy_get64__E)
                  00087ce2    00000006     PMCU_BIOS_cpu1_p28FP.o28FP (.text:_xdc_runtime_System_Module_GateProxy_enter__E)
                  00087ce8    00000006     PMCU_BIOS_cpu1_p28FP.o28FP (.text:_xdc_runtime_System_SupportProxy_abort__E)
                  00087cee    00000006     PMCU_BIOS_cpu1_p28FP.o28FP (.text:_xdc_runtime_System_SupportProxy_exit__E)
                  00087cf4    00000006     PMCU_BIOS_cpu1_p28FP.o28FP (.text:_xdc_runtime_System_SupportProxy_putch__E)
                  00087cfa    00000005     sysbios.a28FP : BIOS.obj (.text:_ti_sysbios_family_c28_Hwi_switchFromBootStack__E)
                  00087cff    00000005                   : BIOS.obj (.text:_ti_sysbios_gates_GateHwi_enter__E)
                  00087d04    00000005     PMCU_BIOS_cpu1_p28FP.o28FP (.text:_xdc_iargToPtr)
                  00087d09    00000005     ti.targets.rts2800.a28FP : LoggerBuf.o28FP (.text:_xdc_runtime_LoggerBuf_enable__E)
                  00087d0e    00000005     rts2800_fpu32.lib : strcpy.obj (.text)
                  00087d13    00000004     PMCU_BIOS_cpu1_p28FP.o28FP (.text:_ti_sysbios_family_c28_Hwi_startup__E)
                  00087d17    00000004     sysbios.a28FP : BIOS.obj (.text:_ti_sysbios_heaps_HeapMem_isBlocking__E)
                  00087d1b    00000004                   : BIOS.obj (.text:_ti_sysbios_knl_Swi_startup__E)
                  00087d1f    00000004     ti.targets.rts2800.a28FP : LoggerBuf.o28FP (.text:_xdc_runtime_LoggerBuf_disable__E)
                  00087d23    00000004                              : Memory.o28FP (.text:_xdc_runtime_Memory_getMaxDefaultTypeAlign__E)
                  00087d27    00000004                              : Startup.o28FP (.text:_xdc_runtime_Startup_rtsDone__E)
                  00087d2b    00000003                              : xdc_noinit.o28FP (.text:___xdc__init)
                  00087d2e    00000003     PMCU_BIOS_cpu1_p28FP.o28FP (.text:_ti_sysbios_family_c28_Hwi_Module__startupDone__S)
                  00087d31    00000003     PMCU_BIOS_cpu1_p28FP.o28FP (.text:_ti_sysbios_family_c28_Timer_Module__startupDone__S)
                  00087d34    00000003     sysbios.a28FP : BIOS.obj (.text:_ti_sysbios_gates_GateHwi_leave__E)
                  00087d37    00000003     PMCU_BIOS_cpu1_p28FP.o28FP (.text:_ti_sysbios_hal_Hwi_HwiProxy_Module__startupDone__S)
                  00087d3a    00000003     PMCU_BIOS_cpu1_p28FP.o28FP (.text:_ti_sysbios_hal_Hwi_HwiProxy_startup__E)
                  00087d3d    00000003     PMCU_BIOS_cpu1_p28FP.o28FP (.text:_ti_sysbios_hal_Hwi_HwiProxy_switchFromBootStack__E)
                  00087d40    00000003     sysbios.a28FP : BIOS.obj (.text:_ti_sysbios_hal_Hwi_startup__E)
                  00087d43    00000003     PMCU_BIOS_cpu1_p28FP.o28FP (.text:_ti_sysbios_hal_Timer_TimerProxy_Module__startupDone__S)
                  00087d46    00000003     PMCU_BIOS_cpu1_p28FP.o28FP (.text:_ti_sysbios_knl_Clock_TimerProxy_Module__startupDone__S)
                  00087d49    00000003     sysbios.a28FP : BIOS.obj (.text:_ti_sysbios_knl_Idle_loop__E)
                  00087d4c    00000003                   : BIOS.obj (.text:_ti_sysbios_knl_Queue_Instance_init__E)
                  00087d4f    00000003     PMCU_BIOS_cpu1_p28FP.o28FP (.text:_ti_sysbios_knl_Task_SupportProxy_Module__startupDone__S)
                  00087d52    00000003     sysbios.a28FP : BIOS.obj (.text:_ti_sysbios_knl_Task_startup__E)
                  00087d55    00000003     PMCU_BIOS_cpu1_p28FP.o28FP (.text:_xdc_runtime_Startup_reset__I)
                  00087d58    00000003     ti.targets.rts2800.a28FP : System.o28FP (.text:_xdc_runtime_System_Module_startup__E)
                  00087d5b    00000003     PMCU_BIOS_cpu1_p28FP.o28FP (.text:_xdc_runtime_System_SupportProxy_ready__E)
                  00087d5e    00000003     ti.targets.rts2800.a28FP : System.o28FP (.text:_xdc_runtime_System_abortStd__E)
                  00087d61    00000003                              : System.o28FP (.text:_xdc_runtime_System_exitStd__E)
                  00087d64    00000002     PMCU_BIOS_cpu1_p28FP.o28FP (.text:_ti_sysbios_family_c28_TaskSupport_Module__startupDone__S)
                  00087d66    00000002     sysbios.a28FP : BIOS.obj (.text:_ti_sysbios_family_c28_Timer_getMaxTicks__E)
                  00087d68    00000002                   : BIOS.obj (.text:_ti_sysbios_gates_GateHwi_query__E)
                  00087d6a    00000002                   : BIOS.obj (.text:_ti_sysbios_gates_GateMutex_query__E)
                  00087d6c    00000002     ti.targets.rts2800.a28FP : Error.o28FP (.text:_xdc_runtime_Error_getSite__E)
                  00087d6e    00000001     sysbios.a28FP : c28_Hwi_asm.obj (.text:_ti_sysbios_family_c28_Hwi_interruptReturn__I)
                  00087d6f    00000001                   : BIOS.obj (.text:_ti_sysbios_gates_GateHwi_Instance_init__E)

.switch    0    00087d70    0000001c     
                  00087d70    0000001c     sysbios.a28FP : BIOS.obj (.switch:_ti_sysbios_family_c28_Hwi_clearInterrupt__E)

.econst    0    00088000    00003671     
                  00088000    00001942     PMCU_BIOS_cpu1_p28FP.o28FP (.econst:xdc_runtime_Text_charTab__A)
                  00089942    00000c83     Cmd_Task.obj (.econst:.string)
                  0008a5c5    00000001     PMCU_BIOS_cpu1_p28FP.o28FP (.econst:ti_sysbios_family_c28_Hwi_Module__id__C)
                  0008a5c6    00000248     Can_Task.obj (.econst:.string)
                  0008a80e    000001c0     PMCU_BIOS_cpu1_p28FP.o28FP (.econst:_ti_sysbios_family_c28_Hwi_vectors)
                  0008a9ce    00000189     PMCU_Main.obj (.econst:.string)
                  0008ab57    00000101     rts2800_fpu32.lib : ctype.obj (.econst:.string:__ctypes_)
                  0008ac58    000000b3     PMCU_GpioXint.obj (.econst:.string)
                  0008ad0b    00000001     PMCU_BIOS_cpu1_p28FP.o28FP (.econst:ti_sysbios_family_c28_Hwi_Module__loggerDefined__C)
                  0008ad0c    0000009f     SpiB_ExtADC_Task.obj (.econst:.string)
                  0008adab    00000001     PMCU_BIOS_cpu1_p28FP.o28FP (.econst:ti_sysbios_family_c28_Hwi_NUM_INTERRUPTS_ALL__C)
                  0008adac    00000090     Ipc_Handler.obj (.econst:.string)
                  0008ae3c    00000081     PMCU_BIOS_cpu1_p28FP.o28FP (.econst:.string)
                  0008aebd    00000001     PMCU_BIOS_cpu1_p28FP.o28FP (.econst:ti_sysbios_family_c28_Hwi_Object__count__C)
                  0008aebe    0000006b     SpiA_ExtTemp_Task.obj (.econst:.string)
                  0008af29    00000001     PMCU_BIOS_cpu1_p28FP.o28FP (.econst:ti_sysbios_family_c28_TaskSupport_Module__id__C)
                  0008af2a    00000067     SpiC_ExtDAC_Task.obj (.econst:.string)
                  0008af91    00000001     PMCU_BIOS_cpu1_p28FP.o28FP (.econst:ti_sysbios_family_c28_Timer_Module__id__C)
                  0008af92    0000005a     PMCU_Emif.obj (.econst:.string)
                  0008afec    0000005a     PMCU_BIOS_cpu1_p28FP.o28FP (.econst:xdc_runtime_Text_nodeTab__A)
                  0008b046    00000058     ti.targets.rts2800.a28FP : Error.o28FP (.econst:.string)
                  0008b09e    00000056     PMCU_BIOS_cpu1_p28FP.o28FP (.econst)
                  0008b0f4    0000004a     SpiA_LowDriver.obj (.econst:.string)
                  0008b13e    0000004a     SpiB_LowDriver.obj (.econst:.string)
                  0008b188    0000004a     SpiC_LowDriver.obj (.econst:.string)
                  0008b1d2    00000049     PMCU_PI_Task.obj (.econst:.string)
                  0008b21b    00000001     PMCU_BIOS_cpu1_p28FP.o28FP (.econst:ti_sysbios_family_c28_Timer_startupNeeded__C)
                  0008b21c    00000047     ti.targets.rts2800.a28FP : Log.o28FP (.econst:.string)
                  0008b263    00000001     PMCU_BIOS_cpu1_p28FP.o28FP (.econst:ti_sysbios_gates_GateMutex_Module__id__C)
                  0008b264    00000043     ti.targets.rts2800.a28FP : Text.o28FP (.econst:.string)
                  0008b2a7    00000001     PMCU_BIOS_cpu1_p28FP.o28FP (.econst:ti_sysbios_hal_Hwi_Module__id__C)
                  0008b2a8    0000002a     ti.targets.rts2800.a28FP : Startup.o28FP (.econst:.string)
                  0008b2d2    00000026     rts2800_fpu32.lib : _printfi.obj (.econst:.string)
                  0008b2f8    00000022     uartstdio.obj (.econst:.string)
                  0008b31a    0000001e     PMCU_BIOS_cpu1_p28FP.o28FP (.econst:xdc_runtime_LoggerBuf_Module__FXNS__C)
                  0008b338    0000001c     rts2800_fpu32.lib : _printfi.obj (.econst)
                  0008b354    0000001c                       : s_scalbn.obj (.econst)
                  0008b370    00000018     ustdlib.obj (.econst:.string)
                  0008b388    00000018     ustdlib.obj (.econst:_g_psDaysToMonth)
                  0008b3a0    00000016     PMCU_BIOS_cpu1_p28FP.o28FP (.econst:xdc_runtime_Startup_sfxnTab__A)
                  0008b3b6    00000014     PMCU_Mgmt_Task.obj (.econst:.string)
                  0008b3ca    00000014     PMCU_BIOS_cpu1_p28FP.o28FP (.econst:ti_sysbios_heaps_HeapMem_Module__FXNS__C)
                  0008b3de    00000012     PMCU_BIOS_cpu1_p28FP.o28FP (.econst:ti_sysbios_gates_GateHwi_Module__FXNS__C)
                  0008b3f0    00000012     PMCU_BIOS_cpu1_p28FP.o28FP (.econst:ti_sysbios_gates_GateMutex_Module__FXNS__C)
                  0008b402    00000012     PMCU_BIOS_cpu1_p28FP.o28FP (.econst:ti_sysbios_heaps_HeapMem_Object__PARAMS__C)
                  0008b414    00000012     PMCU_BIOS_cpu1_p28FP.o28FP (.econst:xdc_runtime_LoggerBuf_Object__PARAMS__C)
                  0008b426    00000011     ti.targets.rts2800.a28FP : System.o28FP (.econst:_digtohex)
                  0008b437    00000001     PMCU_BIOS_cpu1_p28FP.o28FP (.econst:ti_sysbios_heaps_HeapMem_Module__id__C)
                  0008b438    00000010     PMCU_BIOS_cpu1_p28FP.o28FP (.econst:ti_sysbios_gates_GateHwi_Object__DESC__C)
                  0008b448    00000010     PMCU_BIOS_cpu1_p28FP.o28FP (.econst:ti_sysbios_gates_GateMutex_Object__DESC__C)
                  0008b458    00000010     PMCU_BIOS_cpu1_p28FP.o28FP (.econst:ti_sysbios_heaps_HeapMem_Object__DESC__C)
                  0008b468    00000010     PMCU_BIOS_cpu1_p28FP.o28FP (.econst:ti_sysbios_knl_Queue_Object__DESC__C)
                  0008b478    00000010     PMCU_BIOS_cpu1_p28FP.o28FP (.econst:ti_sysbios_knl_Semaphore_Object__DESC__C)
                  0008b488    00000010     PMCU_BIOS_cpu1_p28FP.o28FP (.econst:ti_sysbios_knl_Semaphore_Object__PARAMS__C)
                  0008b498    00000010     PMCU_BIOS_cpu1_p28FP.o28FP (.econst:xdc_runtime_LoggerBuf_Object__DESC__C)
                  0008b4a8    0000000c     ustdlib.obj (.econst:_g_pfExponents)
                  0008b4b4    0000000c     PMCU_BIOS_cpu1_p28FP.o28FP (.econst:ti_sysbios_gates_GateHwi_Object__PARAMS__C)
                  0008b4c0    0000000c     PMCU_BIOS_cpu1_p28FP.o28FP (.econst:ti_sysbios_gates_GateMutex_Object__PARAMS__C)
                  0008b4cc    0000000c     PMCU_BIOS_cpu1_p28FP.o28FP (.econst:ti_sysbios_knl_Queue_Object__PARAMS__C)
                  0008b4d8    0000000b     PMCU_BIOS_cpu1_p28FP.o28FP (.econst:xdc_runtime_Startup_sfxnRts__A)
                  0008b4e3    00000009     can.obj (.econst:_g_ui16CANBitValues)
                  0008b4ec    00000008     uartstdio.obj (.econst:_g_ui32UARTBase)
                  0008b4f4    00000008     rts2800_fpu32.lib : s_frexp.obj (.econst)
                  0008b4fc    00000007     ti.targets.rts2800.a28FP : System.o28FP (.econst:.string)
                  0008b503    00000001     PMCU_BIOS_cpu1_p28FP.o28FP (.econst:ti_sysbios_heaps_HeapMem_Object__count__C)
                  0008b504    00000006     uartstdio.obj (.econst:_g_ui32UARTPeriph)
                  0008b50a    00000006     PMCU_BIOS_cpu1_p28FP.o28FP (.econst:xdc_runtime_Startup_firstFxns__A)
                  0008b510    00000005     ti.targets.rts2800.a28FP : Assert.o28FP (.econst:.string)
                  0008b515    00000001     PMCU_BIOS_cpu1_p28FP.o28FP (.econst:ti_sysbios_knl_Clock_Module__id__C)
                  0008b516    00000004     PMCU_BIOS_cpu1_p28FP.o28FP (.econst:ti_sysbios_knl_Idle_funcList__C)
                  0008b51a    00000004     PMCU_BIOS_cpu1_p28FP.o28FP (.econst:xdc_runtime_Startup_firstFxns__C)
                  0008b51e    00000004     PMCU_BIOS_cpu1_p28FP.o28FP (.econst:xdc_runtime_Startup_lastFxns__C)
                  0008b522    00000002     PMCU_BIOS_cpu1_p28FP.o28FP (.econst:ti_sysbios_BIOS_installedErrorHook__C)
                  0008b524    00000002     PMCU_BIOS_cpu1_p28FP.o28FP (.econst:ti_sysbios_family_c28_Hwi_A_badIntNum__C)
                  0008b526    00000002     PMCU_BIOS_cpu1_p28FP.o28FP (.econst:ti_sysbios_family_c28_Hwi_A_invalidArg__C)
                  0008b528    00000002     PMCU_BIOS_cpu1_p28FP.o28FP (.econst:ti_sysbios_family_c28_Hwi_E_unpluggedInterrupt__C)
                  0008b52a    00000002     PMCU_BIOS_cpu1_p28FP.o28FP (.econst:ti_sysbios_family_c28_Hwi_LD_end__C)
                  0008b52c    00000002     PMCU_BIOS_cpu1_p28FP.o28FP (.econst:ti_sysbios_family_c28_Hwi_LM_begin__C)
                  0008b52e    00000002     PMCU_BIOS_cpu1_p28FP.o28FP (.econst:ti_sysbios_family_c28_Hwi_Module__diagsEnabled__C)
                  0008b530    00000002     PMCU_BIOS_cpu1_p28FP.o28FP (.econst:ti_sysbios_family_c28_Hwi_Module__diagsIncluded__C)
                  0008b532    00000002     PMCU_BIOS_cpu1_p28FP.o28FP (.econst:ti_sysbios_family_c28_Hwi_Module__diagsMask__C)
                  0008b534    00000002     PMCU_BIOS_cpu1_p28FP.o28FP (.econst:ti_sysbios_family_c28_Hwi_Module__loggerFxn1__C)
                  0008b536    00000002     PMCU_BIOS_cpu1_p28FP.o28FP (.econst:ti_sysbios_family_c28_Hwi_Module__loggerFxn8__C)
                  0008b538    00000002     PMCU_BIOS_cpu1_p28FP.o28FP (.econst:ti_sysbios_family_c28_Hwi_Module__loggerObj__C)
                  0008b53a    00000002     PMCU_BIOS_cpu1_p28FP.o28FP (.econst:ti_sysbios_family_c28_Hwi_Object__table__C)
                  0008b53c    00000002     PMCU_BIOS_cpu1_p28FP.o28FP (.econst:ti_sysbios_family_c28_TaskSupport_E_invalidStack__C)
                  0008b53e    00000002     PMCU_BIOS_cpu1_p28FP.o28FP (.econst:ti_sysbios_family_c28_Timer_Module__diagsEnabled__C)
                  0008b540    00000002     PMCU_BIOS_cpu1_p28FP.o28FP (.econst:ti_sysbios_family_c28_Timer_Module__diagsIncluded__C)
                  0008b542    00000002     PMCU_BIOS_cpu1_p28FP.o28FP (.econst:ti_sysbios_family_c28_Timer_Module__diagsMask__C)
                  0008b544    00000002     PMCU_BIOS_cpu1_p28FP.o28FP (.econst:ti_sysbios_gates_GateMutex_A_badContext__C)
                  0008b546    00000002     PMCU_BIOS_cpu1_p28FP.o28FP (.econst:ti_sysbios_gates_GateMutex_Instance_State_sem__O)
                  0008b548    00000002     PMCU_BIOS_cpu1_p28FP.o28FP (.econst:ti_sysbios_gates_GateMutex_Module__diagsEnabled__C)
                  0008b54a    00000002     PMCU_BIOS_cpu1_p28FP.o28FP (.econst:ti_sysbios_gates_GateMutex_Module__diagsIncluded__C)
                  0008b54c    00000002     PMCU_BIOS_cpu1_p28FP.o28FP (.econst:ti_sysbios_gates_GateMutex_Module__diagsMask__C)
                  0008b54e    00000002     PMCU_BIOS_cpu1_p28FP.o28FP (.econst:ti_sysbios_hal_Hwi_E_stackOverflow__C)
                  0008b550    00000002     PMCU_BIOS_cpu1_p28FP.o28FP (.econst:ti_sysbios_heaps_HeapMem_A_align__C)
                  0008b552    00000002     PMCU_BIOS_cpu1_p28FP.o28FP (.econst:ti_sysbios_heaps_HeapMem_A_heapSize__C)
                  0008b554    00000002     PMCU_BIOS_cpu1_p28FP.o28FP (.econst:ti_sysbios_heaps_HeapMem_A_invalidFree__C)
                  0008b556    00000002     PMCU_BIOS_cpu1_p28FP.o28FP (.econst:ti_sysbios_heaps_HeapMem_A_zeroBlock__C)
                  0008b558    00000002     PMCU_BIOS_cpu1_p28FP.o28FP (.econst:ti_sysbios_heaps_HeapMem_E_memory__C)
                  0008b55a    00000002     PMCU_BIOS_cpu1_p28FP.o28FP (.econst:ti_sysbios_heaps_HeapMem_Module__diagsEnabled__C)
                  0008b55c    00000002     PMCU_BIOS_cpu1_p28FP.o28FP (.econst:ti_sysbios_heaps_HeapMem_Module__diagsIncluded__C)
                  0008b55e    00000002     PMCU_BIOS_cpu1_p28FP.o28FP (.econst:ti_sysbios_heaps_HeapMem_Module__diagsMask__C)
                  0008b560    00000002     PMCU_BIOS_cpu1_p28FP.o28FP (.econst:ti_sysbios_heaps_HeapMem_Module__gateObj__C)
                  0008b562    00000002     PMCU_BIOS_cpu1_p28FP.o28FP (.econst:ti_sysbios_heaps_HeapMem_Object__table__C)
                  0008b564    00000002     PMCU_BIOS_cpu1_p28FP.o28FP (.econst:ti_sysbios_heaps_HeapMem_reqAlign__C)
                  0008b566    00000002     PMCU_BIOS_cpu1_p28FP.o28FP (.econst:ti_sysbios_knl_Clock_LM_begin__C)
                  0008b568    00000002     PMCU_BIOS_cpu1_p28FP.o28FP (.econst:ti_sysbios_knl_Clock_LM_tick__C)
                  0008b56a    00000002     PMCU_BIOS_cpu1_p28FP.o28FP (.econst:ti_sysbios_knl_Clock_LW_delayed__C)
                  0008b56c    00000002     PMCU_BIOS_cpu1_p28FP.o28FP (.econst:ti_sysbios_knl_Clock_Module_State_clockQ__O)
                  0008b56e    00000002     PMCU_BIOS_cpu1_p28FP.o28FP (.econst:ti_sysbios_knl_Clock_Module__diagsEnabled__C)
                  0008b570    00000002     PMCU_BIOS_cpu1_p28FP.o28FP (.econst:ti_sysbios_knl_Clock_Module__diagsIncluded__C)
                  0008b572    00000002     PMCU_BIOS_cpu1_p28FP.o28FP (.econst:ti_sysbios_knl_Clock_Module__diagsMask__C)
                  0008b574    00000002     PMCU_BIOS_cpu1_p28FP.o28FP (.econst:ti_sysbios_knl_Clock_Module__loggerFxn1__C)
                  0008b576    00000002     PMCU_BIOS_cpu1_p28FP.o28FP (.econst:ti_sysbios_knl_Clock_Module__loggerFxn2__C)
                  0008b578    00000002     PMCU_BIOS_cpu1_p28FP.o28FP (.econst:ti_sysbios_knl_Clock_Module__loggerObj__C)
                  0008b57a    00000002     PMCU_BIOS_cpu1_p28FP.o28FP (.econst:ti_sysbios_knl_Event_A_badContext__C)
                  0008b57c    00000002     PMCU_BIOS_cpu1_p28FP.o28FP (.econst:ti_sysbios_knl_Event_A_eventInUse__C)
                  0008b57e    00000002     PMCU_BIOS_cpu1_p28FP.o28FP (.econst:ti_sysbios_knl_Event_A_nullEventId__C)
                  0008b580    00000002     PMCU_BIOS_cpu1_p28FP.o28FP (.econst:ti_sysbios_knl_Event_A_nullEventMasks__C)
                  0008b582    00000002     PMCU_BIOS_cpu1_p28FP.o28FP (.econst:ti_sysbios_knl_Event_A_pendTaskDisabled__C)
                  0008b584    00000002     PMCU_BIOS_cpu1_p28FP.o28FP (.econst:ti_sysbios_knl_Event_Instance_State_pendQ__O)
                  0008b586    00000002     PMCU_BIOS_cpu1_p28FP.o28FP (.econst:ti_sysbios_knl_Event_LM_pend__C)
                  0008b588    00000002     PMCU_BIOS_cpu1_p28FP.o28FP (.econst:ti_sysbios_knl_Event_LM_post__C)
                  0008b58a    00000002     PMCU_BIOS_cpu1_p28FP.o28FP (.econst:ti_sysbios_knl_Event_Module__diagsEnabled__C)
                  0008b58c    00000002     PMCU_BIOS_cpu1_p28FP.o28FP (.econst:ti_sysbios_knl_Event_Module__diagsIncluded__C)
                  0008b58e    00000002     PMCU_BIOS_cpu1_p28FP.o28FP (.econst:ti_sysbios_knl_Event_Module__diagsMask__C)
                  0008b590    00000002     PMCU_BIOS_cpu1_p28FP.o28FP (.econst:ti_sysbios_knl_Event_Module__loggerFxn4__C)
                  0008b592    00000002     PMCU_BIOS_cpu1_p28FP.o28FP (.econst:ti_sysbios_knl_Event_Module__loggerFxn8__C)
                  0008b594    00000002     PMCU_BIOS_cpu1_p28FP.o28FP (.econst:ti_sysbios_knl_Event_Module__loggerObj__C)
                  0008b596    00000002     PMCU_BIOS_cpu1_p28FP.o28FP (.econst:ti_sysbios_knl_Idle_funcList__A)
                  0008b598    00000002     PMCU_BIOS_cpu1_p28FP.o28FP (.econst:ti_sysbios_knl_Mailbox_Instance_State_dataQue__O)
                  0008b59a    00000002     PMCU_BIOS_cpu1_p28FP.o28FP (.econst:ti_sysbios_knl_Mailbox_Instance_State_dataSem__O)
                  0008b59c    00000002     PMCU_BIOS_cpu1_p28FP.o28FP (.econst:ti_sysbios_knl_Mailbox_Instance_State_freeQue__O)
                  0008b59e    00000002     PMCU_BIOS_cpu1_p28FP.o28FP (.econst:ti_sysbios_knl_Mailbox_Instance_State_freeSem__O)
                  0008b5a0    00000002     PMCU_BIOS_cpu1_p28FP.o28FP (.econst:ti_sysbios_knl_Mailbox_Object__table__C)
                  0008b5a2    00000002     PMCU_BIOS_cpu1_p28FP.o28FP (.econst:ti_sysbios_knl_Queue_Object__table__C)
                  0008b5a4    00000002     PMCU_BIOS_cpu1_p28FP.o28FP (.econst:ti_sysbios_knl_Semaphore_A_badContext__C)
                  0008b5a6    00000002     PMCU_BIOS_cpu1_p28FP.o28FP (.econst:ti_sysbios_knl_Semaphore_A_overflow__C)
                  0008b5a8    00000002     PMCU_BIOS_cpu1_p28FP.o28FP (.econst:ti_sysbios_knl_Semaphore_A_pendTaskDisabled__C)
                  0008b5aa    00000002     PMCU_BIOS_cpu1_p28FP.o28FP (.econst:ti_sysbios_knl_Semaphore_Instance_State_pendQ__O)
                  0008b5ac    00000002     PMCU_BIOS_cpu1_p28FP.o28FP (.econst:ti_sysbios_knl_Semaphore_LM_pend__C)
                  0008b5ae    00000002     PMCU_BIOS_cpu1_p28FP.o28FP (.econst:ti_sysbios_knl_Semaphore_LM_post__C)
                  0008b5b0    00000002     PMCU_BIOS_cpu1_p28FP.o28FP (.econst:ti_sysbios_knl_Semaphore_Module__diagsEnabled__C)
                  0008b5b2    00000002     PMCU_BIOS_cpu1_p28FP.o28FP (.econst:ti_sysbios_knl_Semaphore_Module__diagsIncluded__C)
                  0008b5b4    00000002     PMCU_BIOS_cpu1_p28FP.o28FP (.econst:ti_sysbios_knl_Semaphore_Module__diagsMask__C)
                  0008b5b6    00000002     PMCU_BIOS_cpu1_p28FP.o28FP (.econst:ti_sysbios_knl_Semaphore_Module__loggerFxn2__C)
                  0008b5b8    00000002     PMCU_BIOS_cpu1_p28FP.o28FP (.econst:ti_sysbios_knl_Semaphore_Module__loggerFxn4__C)
                  0008b5ba    00000002     PMCU_BIOS_cpu1_p28FP.o28FP (.econst:ti_sysbios_knl_Semaphore_Module__loggerObj__C)
                  0008b5bc    00000002     PMCU_BIOS_cpu1_p28FP.o28FP (.econst:ti_sysbios_knl_Semaphore_eventPost__C)
                  0008b5be    00000002     PMCU_BIOS_cpu1_p28FP.o28FP (.econst:ti_sysbios_knl_Semaphore_eventSync__C)
                  0008b5c0    00000002     PMCU_BIOS_cpu1_p28FP.o28FP (.econst:ti_sysbios_knl_Swi_LD_end__C)
                  0008b5c2    00000002     PMCU_BIOS_cpu1_p28FP.o28FP (.econst:ti_sysbios_knl_Swi_LM_begin__C)
                  0008b5c4    00000002     PMCU_BIOS_cpu1_p28FP.o28FP (.econst:ti_sysbios_knl_Swi_LM_post__C)
                  0008b5c6    00000002     PMCU_BIOS_cpu1_p28FP.o28FP (.econst:ti_sysbios_knl_Swi_Module__diagsEnabled__C)
                  0008b5c8    00000002     PMCU_BIOS_cpu1_p28FP.o28FP (.econst:ti_sysbios_knl_Swi_Module__diagsIncluded__C)
                  0008b5ca    00000002     PMCU_BIOS_cpu1_p28FP.o28FP (.econst:ti_sysbios_knl_Swi_Module__diagsMask__C)
                  0008b5cc    00000002     PMCU_BIOS_cpu1_p28FP.o28FP (.econst:ti_sysbios_knl_Swi_Module__loggerFxn1__C)
                  0008b5ce    00000002     PMCU_BIOS_cpu1_p28FP.o28FP (.econst:ti_sysbios_knl_Swi_Module__loggerFxn4__C)
                  0008b5d0    00000002     PMCU_BIOS_cpu1_p28FP.o28FP (.econst:ti_sysbios_knl_Swi_Module__loggerObj__C)
                  0008b5d2    00000002     PMCU_BIOS_cpu1_p28FP.o28FP (.econst:ti_sysbios_knl_Swi_Object__table__C)
                  0008b5d4    00000002     PMCU_BIOS_cpu1_p28FP.o28FP (.econst:ti_sysbios_knl_Task_A_badTimeout__C)
                  0008b5d6    00000002     PMCU_BIOS_cpu1_p28FP.o28FP (.econst:ti_sysbios_knl_Task_A_sleepTaskDisabled__C)
                  0008b5d8    00000002     PMCU_BIOS_cpu1_p28FP.o28FP (.econst:ti_sysbios_knl_Task_E_spOutOfBounds__C)
                  0008b5da    00000002     PMCU_BIOS_cpu1_p28FP.o28FP (.econst:ti_sysbios_knl_Task_E_stackOverflow__C)
                  0008b5dc    00000002     PMCU_BIOS_cpu1_p28FP.o28FP (.econst:ti_sysbios_knl_Task_LD_block__C)
                  0008b5de    00000002     PMCU_BIOS_cpu1_p28FP.o28FP (.econst:ti_sysbios_knl_Task_LD_exit__C)
                  0008b5e0    00000002     PMCU_BIOS_cpu1_p28FP.o28FP (.econst:ti_sysbios_knl_Task_LD_ready__C)
                  0008b5e2    00000002     PMCU_BIOS_cpu1_p28FP.o28FP (.econst:ti_sysbios_knl_Task_LM_sleep__C)
                  0008b5e4    00000002     PMCU_BIOS_cpu1_p28FP.o28FP (.econst:ti_sysbios_knl_Task_LM_switch__C)
                  0008b5e6    00000002     PMCU_BIOS_cpu1_p28FP.o28FP (.econst:ti_sysbios_knl_Task_Module_State_inactiveQ__O)
                  0008b5e8    00000002     PMCU_BIOS_cpu1_p28FP.o28FP (.econst:ti_sysbios_knl_Task_Module__diagsEnabled__C)
                  0008b5ea    00000002     PMCU_BIOS_cpu1_p28FP.o28FP (.econst:ti_sysbios_knl_Task_Module__diagsIncluded__C)
                  0008b5ec    00000002     PMCU_BIOS_cpu1_p28FP.o28FP (.econst:ti_sysbios_knl_Task_Module__diagsMask__C)
                  0008b5ee    00000002     PMCU_BIOS_cpu1_p28FP.o28FP (.econst:ti_sysbios_knl_Task_Module__loggerFxn2__C)
                  0008b5f0    00000002     PMCU_BIOS_cpu1_p28FP.o28FP (.econst:ti_sysbios_knl_Task_Module__loggerFxn4__C)
                  0008b5f2    00000002     PMCU_BIOS_cpu1_p28FP.o28FP (.econst:ti_sysbios_knl_Task_Module__loggerObj__C)
                  0008b5f4    00000002     PMCU_BIOS_cpu1_p28FP.o28FP (.econst:ti_sysbios_knl_Task_Object__table__C)
                  0008b5f6    00000002     PMCU_BIOS_cpu1_p28FP.o28FP (.econst:ti_sysbios_knl_Task_allBlockedFunc__C)
                  0008b5f8    00000002     uartstdio.obj (.econst)
                  0008b5fa    00000002     ustdlib.obj (.econst)
                  0008b5fc    00000002     PMCU_BIOS_cpu1_p28FP.o28FP (.econst:xdc_runtime_Assert_E_assertFailed__C)
                  0008b5fe    00000002     PMCU_BIOS_cpu1_p28FP.o28FP (.econst:xdc_runtime_Core_A_initializedParams__C)
                  0008b600    00000002     PMCU_BIOS_cpu1_p28FP.o28FP (.econst:xdc_runtime_Core_Module__diagsEnabled__C)
                  0008b602    00000002     PMCU_BIOS_cpu1_p28FP.o28FP (.econst:xdc_runtime_Core_Module__diagsIncluded__C)
                  0008b604    00000002     PMCU_BIOS_cpu1_p28FP.o28FP (.econst:xdc_runtime_Core_Module__diagsMask__C)
                  0008b606    00000002     PMCU_BIOS_cpu1_p28FP.o28FP (.econst:xdc_runtime_Error_E_memory__C)
                  0008b608    00000002     PMCU_BIOS_cpu1_p28FP.o28FP (.econst:xdc_runtime_Error_Module__diagsEnabled__C)
                  0008b60a    00000002     PMCU_BIOS_cpu1_p28FP.o28FP (.econst:xdc_runtime_Error_Module__diagsIncluded__C)
                  0008b60c    00000002     PMCU_BIOS_cpu1_p28FP.o28FP (.econst:xdc_runtime_Error_Module__diagsMask__C)
                  0008b60e    00000002     PMCU_BIOS_cpu1_p28FP.o28FP (.econst:xdc_runtime_Error_Module__loggerFxn8__C)
                  0008b610    00000002     PMCU_BIOS_cpu1_p28FP.o28FP (.econst:xdc_runtime_Error_Module__loggerObj__C)
                  0008b612    00000002     PMCU_BIOS_cpu1_p28FP.o28FP (.econst:xdc_runtime_Error_policyFxn__C)
                  0008b614    00000002     PMCU_BIOS_cpu1_p28FP.o28FP (.econst:xdc_runtime_Error_raiseHook__C)
                  0008b616    00000002     PMCU_BIOS_cpu1_p28FP.o28FP (.econst:xdc_runtime_IFilterLogger_Interface__BASE__C)
                  0008b618    00000002     PMCU_BIOS_cpu1_p28FP.o28FP (.econst:xdc_runtime_IGateProvider_Interface__BASE__C)
                  0008b61a    00000002     PMCU_BIOS_cpu1_p28FP.o28FP (.econst:xdc_runtime_IHeap_Interface__BASE__C)
                  0008b61c    00000002     PMCU_BIOS_cpu1_p28FP.o28FP (.econst:xdc_runtime_ILogger_Interface__BASE__C)
                  0008b61e    00000002     PMCU_BIOS_cpu1_p28FP.o28FP (.econst:xdc_runtime_IModule_Interface__BASE__C)
                  0008b620    00000002     PMCU_BIOS_cpu1_p28FP.o28FP (.econst:xdc_runtime_Log_L_error__C)
                  0008b622    00000002     PMCU_BIOS_cpu1_p28FP.o28FP (.econst:xdc_runtime_LoggerBuf_E_badLevel__C)
                  0008b624    00000002     PMCU_BIOS_cpu1_p28FP.o28FP (.econst:xdc_runtime_LoggerBuf_Module__gateObj__C)
                  0008b626    00000002     PMCU_BIOS_cpu1_p28FP.o28FP (.econst:xdc_runtime_LoggerBuf_Object__table__C)
                  0008b628    00000002     PMCU_BIOS_cpu1_p28FP.o28FP (.econst:xdc_runtime_LoggerBuf_statusLogger__C)
                  0008b62a    00000002     PMCU_BIOS_cpu1_p28FP.o28FP (.econst:xdc_runtime_Main_Module__diagsEnabled__C)
                  0008b62c    00000002     PMCU_BIOS_cpu1_p28FP.o28FP (.econst:xdc_runtime_Main_Module__diagsIncluded__C)
                  0008b62e    00000002     PMCU_BIOS_cpu1_p28FP.o28FP (.econst:xdc_runtime_Main_Module__diagsMask__C)
                  0008b630    00000002     PMCU_BIOS_cpu1_p28FP.o28FP (.econst:xdc_runtime_Memory_defaultHeapInstance__C)
                  0008b632    00000002     PMCU_BIOS_cpu1_p28FP.o28FP (.econst:xdc_runtime_Startup_execImpl__C)
                  0008b634    00000002     PMCU_BIOS_cpu1_p28FP.o28FP (.econst:xdc_runtime_Startup_sfxnRts__C)
                  0008b636    00000002     PMCU_BIOS_cpu1_p28FP.o28FP (.econst:xdc_runtime_Startup_sfxnTab__C)
                  0008b638    00000002     PMCU_BIOS_cpu1_p28FP.o28FP (.econst:xdc_runtime_Startup_startModsFxn__C)
                  0008b63a    00000002     PMCU_BIOS_cpu1_p28FP.o28FP (.econst:xdc_runtime_SysMin_bufSize__C)
                  0008b63c    00000002     PMCU_BIOS_cpu1_p28FP.o28FP (.econst:xdc_runtime_SysMin_outputFunc__C)
                  0008b63e    00000002     PMCU_BIOS_cpu1_p28FP.o28FP (.econst:xdc_runtime_System_Module__gateObj__C)
                  0008b640    00000002     PMCU_BIOS_cpu1_p28FP.o28FP (.econst:xdc_runtime_System_abortFxn__C)
                  0008b642    00000002     PMCU_BIOS_cpu1_p28FP.o28FP (.econst:xdc_runtime_System_exitFxn__C)
                  0008b644    00000002     PMCU_BIOS_cpu1_p28FP.o28FP (.econst:xdc_runtime_System_extendFxn__C)
                  0008b646    00000002     PMCU_BIOS_cpu1_p28FP.o28FP (.econst:xdc_runtime_Text_charTab__C)
                  0008b648    00000002     PMCU_BIOS_cpu1_p28FP.o28FP (.econst:xdc_runtime_Text_nameEmpty__C)
                  0008b64a    00000002     PMCU_BIOS_cpu1_p28FP.o28FP (.econst:xdc_runtime_Text_nameStatic__C)
                  0008b64c    00000002     PMCU_BIOS_cpu1_p28FP.o28FP (.econst:xdc_runtime_Text_nameUnknown__C)
                  0008b64e    00000002     PMCU_BIOS_cpu1_p28FP.o28FP (.econst:xdc_runtime_Text_nodeTab__C)
                  0008b650    00000002     PMCU_BIOS_cpu1_p28FP.o28FP (.econst:xdc_runtime_Text_visitRopeFxn__C)
                  0008b652    00000001     PMCU_BIOS_cpu1_p28FP.o28FP (.econst:ti_sysbios_knl_Clock_Module__loggerDefined__C)
                  0008b653    00000001     PMCU_BIOS_cpu1_p28FP.o28FP (.econst:ti_sysbios_knl_Event_Module__id__C)
                  0008b654    00000001     PMCU_BIOS_cpu1_p28FP.o28FP (.econst:ti_sysbios_knl_Event_Module__loggerDefined__C)
                  0008b655    00000001     PMCU_BIOS_cpu1_p28FP.o28FP (.econst:ti_sysbios_knl_Mailbox_Object__count__C)
                  0008b656    00000001     PMCU_BIOS_cpu1_p28FP.o28FP (.econst:ti_sysbios_knl_Mailbox_maxTypeAlign__C)
                  0008b657    00000001     PMCU_BIOS_cpu1_p28FP.o28FP (.econst:ti_sysbios_knl_Queue_Object__count__C)
                  0008b658    00000001     PMCU_BIOS_cpu1_p28FP.o28FP (.econst:ti_sysbios_knl_Semaphore_Module__id__C)
                  0008b659    00000001     PMCU_BIOS_cpu1_p28FP.o28FP (.econst:ti_sysbios_knl_Semaphore_Module__loggerDefined__C)
                  0008b65a    00000001     PMCU_BIOS_cpu1_p28FP.o28FP (.econst:ti_sysbios_knl_Swi_Module__id__C)
                  0008b65b    00000001     PMCU_BIOS_cpu1_p28FP.o28FP (.econst:ti_sysbios_knl_Swi_Module__loggerDefined__C)
                  0008b65c    00000001     PMCU_BIOS_cpu1_p28FP.o28FP (.econst:ti_sysbios_knl_Swi_Object__count__C)
                  0008b65d    00000001     PMCU_BIOS_cpu1_p28FP.o28FP (.econst:ti_sysbios_knl_Task_Module__id__C)
                  0008b65e    00000001     PMCU_BIOS_cpu1_p28FP.o28FP (.econst:ti_sysbios_knl_Task_Module__loggerDefined__C)
                  0008b65f    00000001     PMCU_BIOS_cpu1_p28FP.o28FP (.econst:ti_sysbios_knl_Task_Object__count__C)
                  0008b660    00000001     PMCU_BIOS_cpu1_p28FP.o28FP (.econst:ti_sysbios_knl_Task_numConstructedTasks__C)
                  0008b661    00000001     PMCU_BIOS_cpu1_p28FP.o28FP (.econst:xdc_runtime_Core_Module__id__C)
                  0008b662    00000001     PMCU_BIOS_cpu1_p28FP.o28FP (.econst:xdc_runtime_Error_Module__loggerDefined__C)
                  0008b663    00000001     PMCU_BIOS_cpu1_p28FP.o28FP (.econst:xdc_runtime_Error_maxDepth__C)
                  0008b664    00000001     PMCU_BIOS_cpu1_p28FP.o28FP (.econst:xdc_runtime_Error_policy__C)
                  0008b665    00000001     PMCU_BIOS_cpu1_p28FP.o28FP (.econst:xdc_runtime_LoggerBuf_Module__id__C)
                  0008b666    00000001     PMCU_BIOS_cpu1_p28FP.o28FP (.econst:xdc_runtime_LoggerBuf_Object__count__C)
                  0008b667    00000001     PMCU_BIOS_cpu1_p28FP.o28FP (.econst:xdc_runtime_LoggerBuf_filterByLevel__C)
                  0008b668    00000001     PMCU_BIOS_cpu1_p28FP.o28FP (.econst:xdc_runtime_Main_Module__id__C)
                  0008b669    00000001     PMCU_BIOS_cpu1_p28FP.o28FP (.econst:xdc_runtime_Memory_Module__id__C)
                  0008b66a    00000001     PMCU_BIOS_cpu1_p28FP.o28FP (.econst:xdc_runtime_Startup_maxPasses__C)
                  0008b66b    00000001     PMCU_BIOS_cpu1_p28FP.o28FP (.econst:xdc_runtime_SysMin_flushAtExit__C)
                  0008b66c    00000001     PMCU_BIOS_cpu1_p28FP.o28FP (.econst:xdc_runtime_System_maxAtexitHandlers__C)
                  0008b66d    00000001     PMCU_BIOS_cpu1_p28FP.o28FP (.econst:xdc_runtime_Text_charCnt__C)
                  0008b66e    00000001     PMCU_BIOS_cpu1_p28FP.o28FP (.econst:xdc_runtime_Text_isLoaded__C)
                  0008b66f    00000001     PMCU_BIOS_cpu1_p28FP.o28FP (.econst:xdc_runtime_Text_registryModsLastId__C)
                  0008b670    00000001     PMCU_BIOS_cpu1_p28FP.o28FP (.econst:xdc_runtime_Text_unnamedModsLastId__C)

.stack     1    00000122    00000200     UNINITIALIZED
                  00000122    00000200     --HOLE--

AdcaResultFile 
*          1    00000b00    00000018     UNINITIALIZED
                  00000b00    00000018     F2837xD_GlobalVariableDefs.obj (AdcaResultFile)

AdcbResultFile 
*          1    00000b20    00000018     UNINITIALIZED
                  00000b20    00000018     F2837xD_GlobalVariableDefs.obj (AdcbResultFile)

AdccResultFile 
*          1    00000b40    00000018     UNINITIALIZED
                  00000b40    00000018     F2837xD_GlobalVariableDefs.obj (AdccResultFile)

AdcdResultFile 
*          1    00000b60    00000018     UNINITIALIZED
                  00000b60    00000018     F2837xD_GlobalVariableDefs.obj (AdcdResultFile)

CpuTimer0RegsFile 
*          1    00000c00    00000008     UNINITIALIZED
                  00000c00    00000008     F2837xD_GlobalVariableDefs.obj (CpuTimer0RegsFile)

CpuTimer1RegsFile 
*          1    00000c08    00000008     UNINITIALIZED
                  00000c08    00000008     F2837xD_GlobalVariableDefs.obj (CpuTimer1RegsFile)

CpuTimer2RegsFile 
*          1    00000c10    00000008     UNINITIALIZED
                  00000c10    00000008     F2837xD_GlobalVariableDefs.obj (CpuTimer2RegsFile)

PieCtrlRegsFile 
*          1    00000ce0    0000001a     UNINITIALIZED
                  00000ce0    0000001a     F2837xD_GlobalVariableDefs.obj (PieCtrlRegsFile)

DmaRegsFile 
*          1    00001000    000000e0     UNINITIALIZED
                  00001000    000000e0     F2837xD_GlobalVariableDefs.obj (DmaRegsFile)

Cla1RegsFile 
*          1    00001400    0000003e     UNINITIALIZED
                  00001400    0000003e     F2837xD_GlobalVariableDefs.obj (Cla1RegsFile)

EPwm1RegsFile 
*          1    00004000    00000100     UNINITIALIZED
                  00004000    00000100     F2837xD_GlobalVariableDefs.obj (EPwm1RegsFile)

EPwm2RegsFile 
*          1    00004100    00000100     UNINITIALIZED
                  00004100    00000100     F2837xD_GlobalVariableDefs.obj (EPwm2RegsFile)

EPwm3RegsFile 
*          1    00004200    00000100     UNINITIALIZED
                  00004200    00000100     F2837xD_GlobalVariableDefs.obj (EPwm3RegsFile)

EPwm4RegsFile 
*          1    00004300    00000100     UNINITIALIZED
                  00004300    00000100     F2837xD_GlobalVariableDefs.obj (EPwm4RegsFile)

EPwm5RegsFile 
*          1    00004400    00000100     UNINITIALIZED
                  00004400    00000100     F2837xD_GlobalVariableDefs.obj (EPwm5RegsFile)

EPwm6RegsFile 
*          1    00004500    00000100     UNINITIALIZED
                  00004500    00000100     F2837xD_GlobalVariableDefs.obj (EPwm6RegsFile)

EPwm7RegsFile 
*          1    00004600    00000100     UNINITIALIZED
                  00004600    00000100     F2837xD_GlobalVariableDefs.obj (EPwm7RegsFile)

EPwm8RegsFile 
*          1    00004700    00000100     UNINITIALIZED
                  00004700    00000100     F2837xD_GlobalVariableDefs.obj (EPwm8RegsFile)

EPwm9RegsFile 
*          1    00004800    00000100     UNINITIALIZED
                  00004800    00000100     F2837xD_GlobalVariableDefs.obj (EPwm9RegsFile)

EPwm10RegsFile 
*          1    00004900    00000100     UNINITIALIZED
                  00004900    00000100     F2837xD_GlobalVariableDefs.obj (EPwm10RegsFile)

EPwm11RegsFile 
*          1    00004a00    00000100     UNINITIALIZED
                  00004a00    00000100     F2837xD_GlobalVariableDefs.obj (EPwm11RegsFile)

EPwm12RegsFile 
*          1    00004b00    00000100     UNINITIALIZED
                  00004b00    00000100     F2837xD_GlobalVariableDefs.obj (EPwm12RegsFile)

ECap1RegsFile 
*          1    00005000    00000020     UNINITIALIZED
                  00005000    00000020     F2837xD_GlobalVariableDefs.obj (ECap1RegsFile)

ECap2RegsFile 
*          1    00005020    00000020     UNINITIALIZED
                  00005020    00000020     F2837xD_GlobalVariableDefs.obj (ECap2RegsFile)

ECap3RegsFile 
*          1    00005040    00000020     UNINITIALIZED
                  00005040    00000020     F2837xD_GlobalVariableDefs.obj (ECap3RegsFile)

ECap4RegsFile 
*          1    00005060    00000020     UNINITIALIZED
                  00005060    00000020     F2837xD_GlobalVariableDefs.obj (ECap4RegsFile)

ECap5RegsFile 
*          1    00005080    00000020     UNINITIALIZED
                  00005080    00000020     F2837xD_GlobalVariableDefs.obj (ECap5RegsFile)

ECap6RegsFile 
*          1    000050a0    00000020     UNINITIALIZED
                  000050a0    00000020     F2837xD_GlobalVariableDefs.obj (ECap6RegsFile)

EQep1RegsFile 
*          1    00005100    00000022     UNINITIALIZED
                  00005100    00000022     F2837xD_GlobalVariableDefs.obj (EQep1RegsFile)

EQep2RegsFile 
*          1    00005140    00000022     UNINITIALIZED
                  00005140    00000022     F2837xD_GlobalVariableDefs.obj (EQep2RegsFile)

EQep3RegsFile 
*          1    00005180    00000022     UNINITIALIZED
                  00005180    00000022     F2837xD_GlobalVariableDefs.obj (EQep3RegsFile)

DacaRegsFile 
*          1    00005c00    00000008     UNINITIALIZED
                  00005c00    00000008     F2837xD_GlobalVariableDefs.obj (DacaRegsFile)

DacbRegsFile 
*          1    00005c10    00000008     UNINITIALIZED
                  00005c10    00000008     F2837xD_GlobalVariableDefs.obj (DacbRegsFile)

DaccRegsFile 
*          1    00005c20    00000008     UNINITIALIZED
                  00005c20    00000008     F2837xD_GlobalVariableDefs.obj (DaccRegsFile)

Cmpss1RegsFile 
*          1    00005c80    00000020     UNINITIALIZED
                  00005c80    00000020     F2837xD_GlobalVariableDefs.obj (Cmpss1RegsFile)

Cmpss2RegsFile 
*          1    00005ca0    00000020     UNINITIALIZED
                  00005ca0    00000020     F2837xD_GlobalVariableDefs.obj (Cmpss2RegsFile)

Cmpss3RegsFile 
*          1    00005cc0    00000020     UNINITIALIZED
                  00005cc0    00000020     F2837xD_GlobalVariableDefs.obj (Cmpss3RegsFile)

Cmpss4RegsFile 
*          1    00005ce0    00000020     UNINITIALIZED
                  00005ce0    00000020     F2837xD_GlobalVariableDefs.obj (Cmpss4RegsFile)

Cmpss5RegsFile 
*          1    00005d00    00000020     UNINITIALIZED
                  00005d00    00000020     F2837xD_GlobalVariableDefs.obj (Cmpss5RegsFile)

Cmpss6RegsFile 
*          1    00005d20    00000020     UNINITIALIZED
                  00005d20    00000020     F2837xD_GlobalVariableDefs.obj (Cmpss6RegsFile)

Cmpss7RegsFile 
*          1    00005d40    00000020     UNINITIALIZED
                  00005d40    00000020     F2837xD_GlobalVariableDefs.obj (Cmpss7RegsFile)

Cmpss8RegsFile 
*          1    00005d60    00000020     UNINITIALIZED
                  00005d60    00000020     F2837xD_GlobalVariableDefs.obj (Cmpss8RegsFile)

Sdfm1RegsFile 
*          1    00005e00    00000080     UNINITIALIZED
                  00005e00    00000080     F2837xD_GlobalVariableDefs.obj (Sdfm1RegsFile)

Sdfm2RegsFile 
*          1    00005e80    00000080     UNINITIALIZED
                  00005e80    00000080     F2837xD_GlobalVariableDefs.obj (Sdfm2RegsFile)

McbspaRegsFile 
*          1    00006000    00000024     UNINITIALIZED
                  00006000    00000024     F2837xD_GlobalVariableDefs.obj (McbspaRegsFile)

McbspbRegsFile 
*          1    00006040    00000024     UNINITIALIZED
                  00006040    00000024     F2837xD_GlobalVariableDefs.obj (McbspbRegsFile)

SpiaRegsFile 
*          1    00006100    00000010     UNINITIALIZED
                  00006100    00000010     F2837xD_GlobalVariableDefs.obj (SpiaRegsFile)

SpibRegsFile 
*          1    00006110    00000010     UNINITIALIZED
                  00006110    00000010     F2837xD_GlobalVariableDefs.obj (SpibRegsFile)

SpicRegsFile 
*          1    00006120    00000010     UNINITIALIZED
                  00006120    00000010     F2837xD_GlobalVariableDefs.obj (SpicRegsFile)

UppRegsFile 
*          1    00006200    00000048     UNINITIALIZED
                  00006200    00000048     F2837xD_GlobalVariableDefs.obj (UppRegsFile)

WdRegsFile 
*          1    00007000    0000002b     UNINITIALIZED
                  00007000    0000002b     F2837xD_GlobalVariableDefs.obj (WdRegsFile)

NmiIntruptRegsFile 
*          1    00007060    00000007     UNINITIALIZED
                  00007060    00000007     F2837xD_GlobalVariableDefs.obj (NmiIntruptRegsFile)

XintRegsFile 
*          1    00007070    0000000b     UNINITIALIZED
                  00007070    0000000b     F2837xD_GlobalVariableDefs.obj (XintRegsFile)

SciaRegsFile 
*          1    00007200    00000010     UNINITIALIZED
                  00007200    00000010     F2837xD_GlobalVariableDefs.obj (SciaRegsFile)

ScibRegsFile 
*          1    00007210    00000010     UNINITIALIZED
                  00007210    00000010     F2837xD_GlobalVariableDefs.obj (ScibRegsFile)

ScicRegsFile 
*          1    00007220    00000010     UNINITIALIZED
                  00007220    00000010     F2837xD_GlobalVariableDefs.obj (ScicRegsFile)

ScidRegsFile 
*          1    00007230    00000010     UNINITIALIZED
                  00007230    00000010     F2837xD_GlobalVariableDefs.obj (ScidRegsFile)

I2caRegsFile 
*          1    00007300    00000022     UNINITIALIZED
                  00007300    00000022     F2837xD_GlobalVariableDefs.obj (I2caRegsFile)

I2cbRegsFile 
*          1    00007340    00000022     UNINITIALIZED
                  00007340    00000022     F2837xD_GlobalVariableDefs.obj (I2cbRegsFile)

AdcaRegsFile 
*          1    00007400    00000080     UNINITIALIZED
                  00007400    00000080     F2837xD_GlobalVariableDefs.obj (AdcaRegsFile)

AdcbRegsFile 
*          1    00007480    00000080     UNINITIALIZED
                  00007480    00000080     F2837xD_GlobalVariableDefs.obj (AdcbRegsFile)

AdccRegsFile 
*          1    00007500    00000080     UNINITIALIZED
                  00007500    00000080     F2837xD_GlobalVariableDefs.obj (AdccRegsFile)

AdcdRegsFile 
*          1    00007580    00000080     UNINITIALIZED
                  00007580    00000080     F2837xD_GlobalVariableDefs.obj (AdcdRegsFile)

InputXbarRegsFile 
*          1    00007900    00000020     UNINITIALIZED
                  00007900    00000020     F2837xD_GlobalVariableDefs.obj (InputXbarRegsFile)

XbarRegsFile 
*          1    00007920    00000020     UNINITIALIZED
                  00007920    00000020     F2837xD_GlobalVariableDefs.obj (XbarRegsFile)

SyncSocRegsFile 
*          1    00007940    00000006     UNINITIALIZED
                  00007940    00000006     F2837xD_GlobalVariableDefs.obj (SyncSocRegsFile)

DmaClaSrcSelRegsFile 
*          1    00007980    0000001a     UNINITIALIZED
                  00007980    0000001a     F2837xD_GlobalVariableDefs.obj (DmaClaSrcSelRegsFile)

EPwmXbarRegsFile 
*          1    00007a00    00000040     UNINITIALIZED
                  00007a00    00000040     F2837xD_GlobalVariableDefs.obj (EPwmXbarRegsFile)

OutputXbarRegsFile 
*          1    00007a80    00000040     UNINITIALIZED
                  00007a80    00000040     F2837xD_GlobalVariableDefs.obj (OutputXbarRegsFile)

GpioCtrlRegsFile 
*          1    00007c00    00000180     UNINITIALIZED
                  00007c00    00000180     F2837xD_GlobalVariableDefs.obj (GpioCtrlRegsFile)

GpioDataRegsFile 
*          1    00007f00    00000030     UNINITIALIZED
                  00007f00    00000030     F2837xD_GlobalVariableDefs.obj (GpioDataRegsFile)

.cio       1    00008040    00000120     UNINITIALIZED
                  00008040    00000120     rts2800_fpu32.lib : trgmsg.obj (.cio)

.ebss      1    0000c000    0000587e     UNINITIALIZED
                  0000c000    00002e03     PMCU_BIOS_cpu1_p28FP.o28FP (.ebss:taskStackSection)
                  0000ee03    00000001     SpiC_ExtDAC_Task.obj (.ebss)
                  0000ee04    00000022     EQEP_PMSM_Control.obj (.ebss)
                  0000ee26    00000017     SpiB_ExtADC_Task.obj (.ebss)
                  0000ee3d    00000002     AdcC_Handler.obj (.ebss)
                  0000ee3f    00000001     rts2800_fpu32.lib : errno.obj (.ebss)
                  0000ee40    00001420     PMCU_Main.obj (.ebss)
                  00010260    00000012     cmdline.obj (.ebss)
                  00010272    0000000a     PMCU_Emif.obj (.ebss)
                  0001027c    00000004     uartstdio.obj (.ebss)
                  00010280    00001040     PMCU_BIOS_cpu1_p28FP.o28FP (.ebss)
                  000112c0    000002c6     Can_Task.obj (.ebss)
                  00011586    00000008     rts2800_fpu32.lib : trgdrv.obj (.ebss)
                  0001158e    00000006                       : exit.obj (.ebss)
                  00011594    00000002     AdcD_Handler.obj (.ebss)
                  00011596    00000002     SpiA_ExtTemp_Task.obj (.ebss)
                  00011598    00000002     rts2800_fpu32.lib : _lock.obj (.ebss:__lock)
                  0001159a    00000002                       : _lock.obj (.ebss:__unlock)
                  0001159c    00000001     ustdlib.obj (.ebss)
                  0001159d    00000023     --HOLE--
                  000115c0    000001a2     Cmd_Task.obj (.ebss)
                  00011762    0000001e     --HOLE--
                  00011780    000000b3     PMCU_GpioXint.obj (.ebss)
                  00011833    0000000d     --HOLE--
                  00011840    0000003e     PMCU_PI_Task.obj (.ebss)

GETBUFFER 
*          0    0003f800    00000000     DSECT

GETWRITEIDX 
*          0    0003f800    00000000     DSECT

PUTREADIDX 
*          0    0003f800    00000000     DSECT

xdc.meta   0    00000000    0000010c     COPY SECTION
                  00000000    0000010c     PMCU_BIOS_cpu1_p28FP.o28FP (xdc.meta)

PieVectTableFile 
*          0    00000d00    000001c0     DSECT
                  00000d00    000001c0     F2837xD_GlobalVariableDefs.obj (PieVectTableFile)

EmuKeyVar 
*          0    00000d00    00000001     DSECT
                  00000d00    00000001     F2837xD_GlobalVariableDefs.obj (EmuKeyVar)

EmuBModeVar 
*          0    00000d01    00000001     DSECT
                  00000d01    00000001     F2837xD_GlobalVariableDefs.obj (EmuBModeVar)

FlashCallbackVar 
*          0    00000d02    00000000     DSECT

FlashScalingVar 
*          0    00000d02    00000000     DSECT

Emif1RegsFile 
*          1    00047000    00000070     UNINITIALIZED
                  00047000    00000070     F2837xD_GlobalVariableDefs.obj (Emif1RegsFile)

Emif2RegsFile 
*          1    00047800    00000070     UNINITIALIZED
                  00047800    00000070     F2837xD_GlobalVariableDefs.obj (Emif2RegsFile)

IpcRegsFile 
*          1    00050000    00000024     UNINITIALIZED
                  00050000    00000024     F2837xD_GlobalVariableDefs.obj (IpcRegsFile)

FlashPumpSemaphoreRegsFile 
*          1    00050024    00000002     UNINITIALIZED
                  00050024    00000002     F2837xD_GlobalVariableDefs.obj (FlashPumpSemaphoreRegsFile)

DevCfgRegsFile 
*          1    0005d000    0000012e     UNINITIALIZED
                  0005d000    0000012e     F2837xD_GlobalVariableDefs.obj (DevCfgRegsFile)

AnalogSubsysRegsFile 
*          1    0005d180    00000048     UNINITIALIZED
                  0005d180    00000048     F2837xD_GlobalVariableDefs.obj (AnalogSubsysRegsFile)

Cla1SoftIntRegsFile 
*          1    00000ce0    00000004     DSECT
                  00000ce0    00000004     F2837xD_GlobalVariableDefs.obj (Cla1SoftIntRegsFile)

ClkCfgRegsFile 
*          1    0005d200    00000032     UNINITIALIZED
                  0005d200    00000032     F2837xD_GlobalVariableDefs.obj (ClkCfgRegsFile)

CpuSysRegsFile 
*          1    0005d300    00000082     UNINITIALIZED
                  0005d300    00000082     F2837xD_GlobalVariableDefs.obj (CpuSysRegsFile)

RomPrefetchRegsFile 
*          1    0005e608    00000002     UNINITIALIZED
                  0005e608    00000002     F2837xD_GlobalVariableDefs.obj (RomPrefetchRegsFile)

DcsmZ1RegsFile 
*          1    0005f000    00000024     UNINITIALIZED
                  0005f000    00000024     F2837xD_GlobalVariableDefs.obj (DcsmZ1RegsFile)

DcsmZ2RegsFile 
*          1    0005f040    00000024     UNINITIALIZED
                  0005f040    00000024     F2837xD_GlobalVariableDefs.obj (DcsmZ2RegsFile)

DcsmCommonRegsFile 
*          1    0005f070    00000008     UNINITIALIZED
                  0005f070    00000008     F2837xD_GlobalVariableDefs.obj (DcsmCommonRegsFile)

MemCfgRegsFile 
*          1    0005f400    00000080     UNINITIALIZED
                  0005f400    00000080     F2837xD_GlobalVariableDefs.obj (MemCfgRegsFile)

Emif1ConfigRegsFile 
*          1    0005f480    00000020     UNINITIALIZED
                  0005f480    00000020     F2837xD_GlobalVariableDefs.obj (Emif1ConfigRegsFile)

Emif2ConfigRegsFile 
*          1    0005f4a0    00000020     UNINITIALIZED
                  0005f4a0    00000020     F2837xD_GlobalVariableDefs.obj (Emif2ConfigRegsFile)

AccessProtectionRegsFile 
*          1    0005f4c0    00000040     UNINITIALIZED
                  0005f4c0    00000040     F2837xD_GlobalVariableDefs.obj (AccessProtectionRegsFile)

MemoryErrorRegsFile 
*          1    0005f500    00000040     UNINITIALIZED
                  0005f500    00000040     F2837xD_GlobalVariableDefs.obj (MemoryErrorRegsFile)

RomWaitStateRegsFile 
*          1    0005f540    00000002     UNINITIALIZED
                  0005f540    00000002     F2837xD_GlobalVariableDefs.obj (RomWaitStateRegsFile)

Flash0CtrlRegsFile 
*          1    0005f800    00000182     UNINITIALIZED
                  0005f800    00000182     F2837xD_GlobalVariableDefs.obj (Flash0CtrlRegsFile)

Flash0EccRegsFile 
*          1    0005fb00    00000028     UNINITIALIZED
                  0005fb00    00000028     F2837xD_GlobalVariableDefs.obj (Flash0EccRegsFile)

DcsmZ1OtpFile 
*          1    00078000    00000020     NOLOAD SECTION
                  00078000    00000020     F2837xD_GlobalVariableDefs.obj (DcsmZ1OtpFile)

DcsmZ2OtpFile 
*          1    00078200    00000020     NOLOAD SECTION
                  00078200    00000020     F2837xD_GlobalVariableDefs.obj (DcsmZ2OtpFile)

MODULE SUMMARY

       Module                           code    ro data   rw data
       ------                           ----    -------   -------
    .\
       PMCU_Main.obj                    118     0         5545   
       PMCU_PI_Task.obj                 325     0         151    
       PMCU_Mgmt_Task.obj               54      0         20     
    +--+--------------------------------+-------+---------+---------+
       Total:                           497     0         5716   
                                                                 
    .\AdcInternal\
       AdcC_Handler.obj                 216     0         2      
       AdcD_Handler.obj                 206     0         2      
       AdcA_Handler.obj                 181     0         0      
       AdcB_Handler.obj                 181     0         0      
    +--+--------------------------------+-------+---------+---------+
       Total:                           784     0         4      
                                                                 
    .\Can\
       Can_Task.obj                     2005    0         1336   
       can.obj                          1326    0         9      
    +--+--------------------------------+-------+---------+---------+
       Total:                           3331    0         1345   
                                                                 
    .\Cmd\
       Cmd_Task.obj                     1722    0         3849   
       cmdline.obj                      73      0         18     
    +--+--------------------------------+-------+---------+---------+
       Total:                           1795    0         3867   
                                                                 
    .\EPwm\
       EPwm_Handler.obj                 115     0         0      
    +--+--------------------------------+-------+---------+---------+
       Total:                           115     0         0      
                                                                 
    .\Emif\
       PMCU_Emif.obj                    184     0         104    
    +--+--------------------------------+-------+---------+---------+
       Total:                           184     0         104    
                                                                 
    .\F28377D_Low_Driver\
       F2837xD_GlobalVariableDefs.obj   0       0         7597   
       F2837xD_SysCtrl.obj              949     0         0      
       F2837xD_Gpio.obj                 580     0         0      
       F2837xD_EPwm.obj                 253     0         0      
       F2837xD_Adc.obj                  221     0         0      
       F2837xD_Spi.obj                  157     0         0      
       F2837xD_usDelay.obj              8       0         0      
    +--+--------------------------------+-------+---------+---------+
       Total:                           2168    0         7597   
                                                                 
    .\GpioXint\
       PMCU_GpioXint.obj                264     0         475    
    +--+--------------------------------+-------+---------+---------+
       Total:                           264     0         475    
                                                                 
    .\Ipc\
       Ipc_Handler.obj                  176     0         144    
    +--+--------------------------------+-------+---------+---------+
       Total:                           176     0         144    
                                                                 
    .\PMSM_Control\source\
       EQEP_PMSM_Control.obj            0       0         119    
    +--+--------------------------------+-------+---------+---------+
       Total:                           0       0         119    
                                                                 
    .\SpiA\
       SpiA_LowDriver.obj               131     0         74     
       SpiA_ExtTemp_Task.obj            94      0         109    
    +--+--------------------------------+-------+---------+---------+
       Total:                           225     0         183    
                                                                 
    .\SpiB\
       SpiB_ExtADC_Task.obj             132     0         182    
       SpiB_LowDriver.obj               202     0         74     
    +--+--------------------------------+-------+---------+---------+
       Total:                           334     0         256    
                                                                 
    .\SpiB\AD7689\
       AD7689_ExtADC.obj                225     0         0      
    +--+--------------------------------+-------+---------+---------+
       Total:                           225     0         0      
                                                                 
    .\SpiC\
       SpiC_LowDriver.obj               190     0         74     
       SpiC_ExtDAC_Task.obj             70      0         104    
    +--+--------------------------------+-------+---------+---------+
       Total:                           260     0         178    
                                                                 
    .\SpiC\AD5764\
       AD5764_ExtDAC.obj                109     0         0      
    +--+--------------------------------+-------+---------+---------+
       Total:                           109     0         0      
                                                                 
    .\Utils\
       ustdlib.obj                      1498    0         67     
       uart.obj                         745     0         0      
       uartstdio.obj                    615     0         63     
       sysctl.obj                       587     0         0      
       interrupt.obj                    473     0         0      
    +--+--------------------------------+-------+---------+---------+
       Total:                           3918    0         130    
                                                                 
    C:\Users\kohjy\workspace_v6_2\Test2_PMSM_Porting_F28377D_CPU1\CPU1_FLASH_DEBUG\configPkg\package\cfg\
       PMCU_BIOS_cpu1_p28FP.o28FP       1380    0         25928  
    +--+--------------------------------+-------+---------+---------+
       Total:                           1380    0         25928  
                                                                 
    C:\Users\kohjy\workspace_v6_2\Test2_PMSM_Porting_F28377D_CPU1\src\sysbios\sysbios.a28FP
       BIOS.obj                         6965    0         28     
       c28_Hwi_disp_asm.obj             155     0         0      
       c28_TaskSupport_asm.obj          75      0         0      
       c28_Hwi_asm.obj                  52      0         0      
       c28_IntrinsicsSupport_asm.obj    6       0         0      
    +--+--------------------------------+-------+---------+---------+
       Total:                           7253    0         28     
                                                                 
    C:\ti\bios_6_46_02_47\packages\ti\catalog\c2800\initF2837x\lib\Boot.a28FP
       Boot.o28FP                       86      0         0      
       Boot_asm.o28FP                   2       0         0      
    +--+--------------------------------+-------+---------+---------+
       Total:                           88      0         0      
                                                                 
    C:\ti\bios_6_46_02_47\packages\ti\targets\rts2800\lib\boot.a28FP
       boot_cg.o28FP                    99      0         0      
    +--+--------------------------------+-------+---------+---------+
       Total:                           99      0         0      
                                                                 
    C:\ti\bios_6_46_02_47\packages\ti\targets\rts2800\lib\ti.targets.rts2800.a28FP
       System.o28FP                     855     0         24     
       LoggerBuf.o28FP                  683     0         0      
       Text.o28FP                       413     0         67     
       Error.o28FP                      325     0         88     
       Core-mem.o28FP                   296     0         0      
       Startup.o28FP                    182     0         42     
       Core-smem.o28FP                  162     0         0      
       Memory.o28FP                     127     0         0      
       SysMin.o28FP                     126     0         0      
       Log.o28FP                        0       0         71     
       Core-params.o28FP                66      0         0      
       Assert.o28FP                     50      0         5      
       Core-label.o28FP                 26      0         0      
       Registry.o28FP                   14      0         0      
       Gate.o28FP                       12      0         0      
       xdc_noinit.o28FP                 3       0         0      
    +--+--------------------------------+-------+---------+---------+
       Total:                           3340    0         297    
                                                                 
    C:\ti\ccsv6\tools\compiler\ti-cgt-c2000_15.12.5.LTS\lib\rts2800_fpu32.lib
       _printfi.obj                     3033    0         66     
       trgdrv.obj                       636     0         8      
       trgmsg.obj                       148     0         288    
       ll_div.obj                       263     0         0      
       ctype.obj                        0       0         257    
       s_scalbn.obj                     188     0         28     
       fd_add.obj                       156     0         0      
       fd_div.obj                       139     0         0      
       fd_mpy.obj                       131     0         0      
       s_frexp.obj                      90      0         8      
       cpy_tbl.obj                      70      0         0      
       exit.obj                         41      0         20     
       sprintf.obj                      50      0         0      
       atoi.obj                         49      0         0      
       ltoa.obj                         46      0         0      
       fd_cmp.obj                       42      0         0      
       l_div.obj                        42      0         0      
       s_copysign.obj                   36      0         0      
       i_div.obj                        34      0         0      
       fd_toi.obj                       33      0         0      
       fd_tol.obj                       31      0         0      
       ll_cmp.obj                       30      0         0      
       memcpy.obj                       30      0         0      
       i_tofd.obj                       29      0         0      
       fs_tofd.obj                      28      0         0      
       l_tofd.obj                       28      0         0      
       cpy_utils.obj                    26      0         0      
       args_main.obj                    25      0         0      
       ll_aox.obj                       24      0         0      
       _lock.obj                        9       0         14     
       fd_sub.obj                       14      0         0      
       memccpy.obj                      13      0         0      
       memset.obj                       12      0         0      
       strchr.obj                       12      0         0      
       u_div.obj                        11      0         0      
       strcmp.obj                       10      0         0      
       fd_neg.obj                       9       0         0      
       strlen.obj                       8       0         0      
       errno.obj                        0       0         5      
       strcpy.obj                       5       0         0      
    +--+--------------------------------+-------+---------+---------+
       Total:                           5581    0         694    
                                                                 
       Stack:                           0       0         512    
       Linker Generated:                0       10        0      
    +--+--------------------------------+-------+---------+---------+
       Grand Total:                     32126   10        47577  


LINKER GENERATED COPY TABLES

binit @ 00087d8c records: 1, size/record: 8, table size: 10
	.text:ti_catalog_c2800_initF2837x_flashfuncs: copy 39 bytes from load addr=00080004 at page=0 to run addr=0000b000 at page=0


GLOBAL DATA SYMBOLS: SORTED BY DATA PAGE

address     data page           name
--------    ----------------    ----
00000000       0 (00000000)     ___ISA__
00000013       0 (00000000)     ___TARG__
00000037       0 (00000000)     ___PLAT__

0000005d       1 (00000040)     ___TRDR__

00000084       2 (00000080)     ___ASM__

00000122       4 (00000100)     __stack

00000b00      2c (00000b00)     _AdcaResultRegs
00000b20      2c (00000b00)     _AdcbResultRegs

00000b40      2d (00000b40)     _AdccResultRegs
00000b60      2d (00000b40)     _AdcdResultRegs

00000c00      30 (00000c00)     _CpuTimer0Regs
00000c08      30 (00000c00)     _CpuTimer1Regs
00000c10      30 (00000c00)     _CpuTimer2Regs

00000ce0      33 (00000cc0)     _Cla1SoftIntRegs
00000ce0      33 (00000cc0)     _PieCtrlRegs

00000d00      34 (00000d00)     _EmuKey
00000d00      34 (00000d00)     _PieVectTable
00000d01      34 (00000d00)     _EmuBMode

00001000      40 (00001000)     _DmaRegs

00001400      50 (00001400)     _Cla1Regs

00004000     100 (00004000)     _EPwm1Regs

00004100     104 (00004100)     _EPwm2Regs

00004200     108 (00004200)     _EPwm3Regs

00004300     10c (00004300)     _EPwm4Regs

00004400     110 (00004400)     _EPwm5Regs

00004500     114 (00004500)     _EPwm6Regs

00004600     118 (00004600)     _EPwm7Regs

00004700     11c (00004700)     _EPwm8Regs

00004800     120 (00004800)     _EPwm9Regs

00004900     124 (00004900)     _EPwm10Regs

00004a00     128 (00004a00)     _EPwm11Regs

00004b00     12c (00004b00)     _EPwm12Regs

00005000     140 (00005000)     _ECap1Regs
00005020     140 (00005000)     _ECap2Regs

00005040     141 (00005040)     _ECap3Regs
00005060     141 (00005040)     _ECap4Regs

00005080     142 (00005080)     _ECap5Regs
000050a0     142 (00005080)     _ECap6Regs

00005100     144 (00005100)     _EQep1Regs

00005140     145 (00005140)     _EQep2Regs

00005180     146 (00005180)     _EQep3Regs

00005c00     170 (00005c00)     _DacaRegs
00005c10     170 (00005c00)     _DacbRegs
00005c20     170 (00005c00)     _DaccRegs

00005c80     172 (00005c80)     _Cmpss1Regs
00005ca0     172 (00005c80)     _Cmpss2Regs

00005cc0     173 (00005cc0)     _Cmpss3Regs
00005ce0     173 (00005cc0)     _Cmpss4Regs

00005d00     174 (00005d00)     _Cmpss5Regs
00005d20     174 (00005d00)     _Cmpss6Regs

00005d40     175 (00005d40)     _Cmpss7Regs
00005d60     175 (00005d40)     _Cmpss8Regs

00005e00     178 (00005e00)     _Sdfm1Regs

00005e80     17a (00005e80)     _Sdfm2Regs

00006000     180 (00006000)     _McbspaRegs

00006040     181 (00006040)     _McbspbRegs

00006100     184 (00006100)     _SpiaRegs
00006110     184 (00006100)     _SpibRegs
00006120     184 (00006100)     _SpicRegs

00006200     188 (00006200)     _UppRegs

00007000     1c0 (00007000)     _WdRegs

00007060     1c1 (00007040)     _NmiIntruptRegs
00007070     1c1 (00007040)     _XintRegs

00007200     1c8 (00007200)     _SciaRegs
00007210     1c8 (00007200)     _ScibRegs
00007220     1c8 (00007200)     _ScicRegs
00007230     1c8 (00007200)     _ScidRegs

00007300     1cc (00007300)     _I2caRegs

00007340     1cd (00007340)     _I2cbRegs

00007400     1d0 (00007400)     _AdcaRegs

00007480     1d2 (00007480)     _AdcbRegs

00007500     1d4 (00007500)     _AdccRegs

00007580     1d6 (00007580)     _AdcdRegs

00007900     1e4 (00007900)     _InputXbarRegs
00007920     1e4 (00007900)     _XbarRegs

00007940     1e5 (00007940)     _SyncSocRegs

00007980     1e6 (00007980)     _DmaClaSrcSelRegs

00007a00     1e8 (00007a00)     _EPwmXbarRegs

00007a80     1ea (00007a80)     _OutputXbarRegs

00007c00     1f0 (00007c00)     _GpioCtrlRegs

00007f00     1fc (00007f00)     _GpioDataRegs

00008040     201 (00008040)     __CIOBUF_

0000c000     300 (0000c000)     _ti_sysbios_knl_Task_Instance_State_6_stack__A

0000c100     304 (0000c100)     _ti_sysbios_knl_Task_Instance_State_5_stack__A

0000c200     308 (0000c200)     _ti_sysbios_knl_Task_Instance_State_10_stack__A

0000c300     30c (0000c300)     _ti_sysbios_knl_Task_Instance_State_8_stack__A

0000c400     310 (0000c400)     _ti_sysbios_knl_Task_Instance_State_1_stack__A

0000c600     318 (0000c600)     _ti_sysbios_knl_Task_Instance_State_3_stack__A

0000c800     320 (0000c800)     _ti_sysbios_knl_Task_Instance_State_2_stack__A

0000ca00     328 (0000ca00)     _ti_sysbios_knl_Task_Instance_State_4_stack__A

0000cc00     330 (0000cc00)     _ti_sysbios_knl_Task_Instance_State_9_stack__A

0000d000     340 (0000d000)     _ti_sysbios_knl_Task_Instance_State_0_stack__A

0000d600     358 (0000d600)     _ti_sysbios_knl_Task_Instance_State_7_stack__A

0000de00     378 (0000de00)     _ti_sysbios_heaps_HeapMem_Instance_State_0_buf__A

0000ee03     3b8 (0000ee00)     _ExtDAC_DebugOn
0000ee04     3b8 (0000ee00)     _threshold_t_value
0000ee06     3b8 (0000ee00)     _threshold_m_value
0000ee08     3b8 (0000ee00)     _m_rpm
0000ee0a     3b8 (0000ee00)     _T1_delta
0000ee0c     3b8 (0000ee00)     _t1_rpm
0000ee0e     3b8 (0000ee00)     _motor4_rpm
0000ee10     3b8 (0000ee00)     _t1_sec
0000ee12     3b8 (0000ee00)     _t1_hz
0000ee14     3b8 (0000ee00)     _motor_dir
0000ee16     3b8 (0000ee00)     _M_old
0000ee18     3b8 (0000ee00)     _qep_tcnt
0000ee1a     3b8 (0000ee00)     _T_ov
0000ee1c     3b8 (0000ee00)     _m_sec
0000ee1e     3b8 (0000ee00)     _m_hz
0000ee20     3b8 (0000ee00)     _M_new
0000ee22     3b8 (0000ee00)     _M_delta
0000ee24     3b8 (0000ee00)     _UT_PRD
0000ee26     3b8 (0000ee00)     _Extcnt
0000ee27     3b8 (0000ee00)     _ExtADC_DebugOn
0000ee28     3b8 (0000ee00)     _ExtADC_Display_Interval
0000ee29     3b8 (0000ee00)     _recv_data
0000ee3f     3b8 (0000ee00)     _errno

0000ee40     3b9 (0000ee40)     _TorqueIndex
0000ee41     3b9 (0000ee40)     _SpeedIndex
0000ee42     3b9 (0000ee40)     _MFluxIndex
0000ee44     3b9 (0000ee40)     _deltaMFlux
0000ee46     3b9 (0000ee40)     _deltaTorque
0000ee48     3b9 (0000ee40)     _iddd
0000ee4a     3b9 (0000ee40)     _iqqq
0000ee4c     3b9 (0000ee40)     _MagFlux
0000ee4e     3b9 (0000ee40)     _iRefC
0000ee50     3b9 (0000ee40)     _torqCmd
0000ee52     3b9 (0000ee40)     _iRefTMax
0000ee54     3b9 (0000ee40)     _deltaRpm
0000ee56     3b9 (0000ee40)     _tableY2
0000ee58     3b9 (0000ee40)     _tableX1
0000ee5a     3b9 (0000ee40)     _tableMin
0000ee5c     3b9 (0000ee40)     _tableMax
0000ee5e     3b9 (0000ee40)     _tableY1
0000ee60     3b9 (0000ee40)     _tableX2

0000ee80     3ba (0000ee80)     _MFluxTable

0000eec0     3bb (0000eec0)     _rpmTable

0000ef00     3bc (0000ef00)     _torqueTable

0000ef80     3be (0000ef80)     _IqTable_Mot

0000f900     3e4 (0000f900)     _IdTable_Mot

00010272     409 (00010240)     _Ecnt
00010273     409 (00010240)     _i
00010274     409 (00010240)     _Emif_DebugOn
00010275     409 (00010240)     _ErrCount
00010276     409 (00010240)     _EMIF_Display_Interval
00010278     409 (00010240)     _EMIF_Read_OffAddr
0001027a     409 (00010240)     _TEST_STATUS
0001027e     409 (00010240)     _g_ui32Base

00010280     40a (00010280)     _xdc_runtime_Error_Module__state__V
00010282     40a (00010280)     _ti_sysbios_knl_Task_Module_State_0_idleTask__A
00010284     40a (00010280)     ___xdc__init__addr
00010286     40a (00010280)     _xdc_runtime_Memory_Module__state__V
00010288     40a (00010280)     _ti_sysbios_gates_GateHwi_Object__table__V
0001028a     40a (00010280)     _xdc_runtime_LoggerBuf_Module__state__V
0001028e     40a (00010280)     _ti_sysbios_knl_Queue_Module__root__V
00010292     40a (00010280)     _ti_sysbios_knl_Event_Module__root__V
00010296     40a (00010280)     _ti_sysbios_hal_Hwi_Module__root__V
0001029a     40a (00010280)     _xdc_runtime_Registry_Module__state__V
0001029e     40a (00010280)     _ti_sysbios_knl_Swi_Module__root__V
000102a2     40a (00010280)     _ti_sysbios_knl_Clock_Module__root__V
000102a6     40a (00010280)     _xdc_runtime_Text_Module__state__V
000102aa     40a (00010280)     _ti_sysbios_knl_Semaphore_Module__root__V
000102ae     40a (00010280)     _ti_sysbios_knl_Mailbox_Module__root__V
000102b2     40a (00010280)     _ti_sysbios_gates_GateHwi_Module__root__V
000102b6     40a (00010280)     _xdc_runtime_LoggerBuf_Module__root__V
000102ba     40a (00010280)     _ti_sysbios_knl_Task_Module__root__V

000102c0     40b (000102c0)     _ti_sysbios_gates_GateMutex_Module__root__V
000102c4     40b (000102c0)     _ti_sysbios_family_c28_Hwi_Module__root__V
000102c8     40b (000102c0)     _ti_sysbios_family_c28_Timer_Module__root__V
000102cc     40b (000102c0)     _xdc_runtime_SysMin_Module__state__V
000102d0     40b (000102c0)     _xdc_runtime_System_Module__state__V
000102d4     40b (000102c0)     _xdc_runtime_Startup_Module__state__V
000102d8     40b (000102c0)     _ti_sysbios_hal_Timer_Module__root__V
000102dc     40b (000102c0)     _ti_sysbios_heaps_HeapMem_Module__root__V
000102e0     40b (000102c0)     _ti_sysbios_family_c28_Timer_Module__state__V
000102e8     40b (000102c0)     _xdc_runtime_System_Module_State_0_atexitHandlers__A
000102f0     40b (000102c0)     _ti_sysbios_knl_Semaphore_Object__table__V

00010300     40c (00010300)     _ti_sysbios_knl_Swi_Module__state__V
0001030c     40c (00010300)     _ti_sysbios_heaps_HeapMem_Object__table__V
00010318     40c (00010300)     _ti_sysbios_family_c28_Hwi_Module__state__V
00010328     40c (00010300)     _ti_sysbios_knl_Mailbox_Instance_State_4_allocBuf__A

00010340     40d (00010340)     _ti_sysbios_knl_Mailbox_Instance_State_9_allocBuf__A
00010352     40d (00010340)     _xdc_runtime_LoggerBuf_Object__table__V
00010364     40d (00010340)     _ti_sysbios_knl_Mailbox_Instance_State_3_allocBuf__A

00010380     40e (00010380)     _ti_sysbios_BIOS_Module__state__V
00010392     40e (00010380)     _ti_sysbios_knl_Swi_Object__table__V
000103a6     40e (00010380)     _ti_sysbios_knl_Clock_Module__state__V

000103c0     40f (000103c0)     _ti_sysbios_gates_GateMutex_Object__table__V
000103dc     40f (000103c0)     _ti_sysbios_knl_Task_Module__state__V

00010400     410 (00010400)     _ti_sysbios_knl_Mailbox_Instance_State_2_allocBuf__A

00010440     411 (00010440)     _ti_sysbios_knl_Mailbox_Instance_State_6_allocBuf__A

00010480     412 (00010480)     _ti_sysbios_family_c28_Timer_Object__table__V

000104c0     413 (000104c0)     _ti_sysbios_knl_Mailbox_Instance_State_5_allocBuf__A

00010500     414 (00010500)     _ti_sysbios_knl_Event_Object__table__V

00010540     415 (00010540)     _ti_sysbios_knl_Mailbox_Instance_State_1_allocBuf__A

00010580     416 (00010580)     _ti_sysbios_knl_Mailbox_Instance_State_0_allocBuf__A

000105c0     417 (000105c0)     _ti_sysbios_knl_Swi_Module_State_0_readyQ__A

00010600     418 (00010600)     _ti_sysbios_knl_Task_Module_State_0_readyQ__A

00010640     419 (00010640)     _ti_sysbios_family_c28_Hwi_Object__table__V

00010740     41d (00010740)     _ti_sysbios_knl_Mailbox_Instance_State_8_allocBuf__A

00010880     422 (00010880)     _ti_sysbios_knl_Mailbox_Instance_State_7_allocBuf__A

000109c0     427 (000109c0)     _ti_sysbios_knl_Task_Object__table__V

00010b40     42d (00010b40)     _ti_sysbios_knl_Mailbox_Object__table__V

00010d00     434 (00010d00)     _ti_sysbios_family_c28_Hwi_Module_State_0_dispatchTable__A

00010ec0     43b (00010ec0)     _xdc_runtime_LoggerBuf_Instance_State_0_entryArr__A

000110c0     443 (000110c0)     _xdc_runtime_SysMin_Module_State_0_outbuf__A

000112c0     44b (000112c0)     _CANA_Err_Int_Enable
000112c1     44b (000112c0)     _Aerror_message
000112c2     44b (000112c0)     _Berror_message
000112c3     44b (000112c0)     _CAN_DebugOn
000112c4     44b (000112c0)     _CANB_Err_Int_Enable
000112c6     44b (000112c0)     _g_ulRxMsgCount
000112c8     44b (000112c0)     _u32CanAErrorStatus
000112ca     44b (000112c0)     _g_bErrFlag
000112cc     44b (000112c0)     _u32CntTXMsgData
000112ce     44b (000112c0)     _g_ulTxMsgCount
000112d0     44b (000112c0)     _ucTXMsgDataB
000112d8     44b (000112c0)     _g_ulRxMsgCountPMSM
000112e0     44b (000112c0)     _ucRXMsgDataB
000112e8     44b (000112c0)     _g_ulTxMsgCountPMSMB
000112f0     44b (000112c0)     _ucRXMsgDataA
000112f8     44b (000112c0)     _ucTXMsgDataA

00011300     44c (00011300)     _sTXCANMessageA
0001130a     44c (00011300)     _sRXCANMessageA
00011314     44c (00011300)     _sTXCANMessageB
0001131e     44c (00011300)     _sRXCANMessageB
00011328     44c (00011300)     _g_ulTxMsgCountPMSM

00011340     44d (00011340)     _g_ulRxMsgCountPMSMB
0001134e     44d (00011340)     _ucRXMsgDataPMSM

00011380     44e (00011380)     _ucTXMsgDataPMSMB

000113c0     44f (000113c0)     _sRXCANMessagePMSM

00011400     450 (00011400)     _sTXCANMessagePMSMB

00011440     451 (00011440)     _ucRXMsgDataPMSMB

00011480     452 (00011480)     _ucTXMsgDataPMSM

000114c0     453 (000114c0)     _sTXCANMessagePMSM

00011540     455 (00011540)     _sRXCANMessagePMSMB

0001158e     456 (00011580)     ___TI_enable_exit_profile_output
00011590     456 (00011580)     ___TI_cleanup_ptr
00011592     456 (00011580)     ___TI_dtors_ptr
00011596     456 (00011580)     _TempReadInterval
00011597     456 (00011580)     _Temp_DebugOn
00011598     456 (00011580)     __lock
0001159a     456 (00011580)     __unlock

000115c2     457 (000115c0)     _g_sFresultStrings

00011640     459 (00011640)     _string_display

000116c0     45b (000116c0)     _g_psCmdTable

00011780     45e (00011780)     _ExtInt_DebugOn

000117c0     45f (000117c0)     _GPIO_Conf_InitVal

00011840     461 (00011840)     _Ccnt
00011841     461 (00011840)     _Bcnt
00011842     461 (00011840)     _BackTicker
00011843     461 (00011840)     _Acnt
00011844     461 (00011840)     _ADC_Display_Interval
00011845     461 (00011840)     _Dcnt
00011846     461 (00011840)     _IsrTicker4
00011847     461 (00011840)     _TickCNT500ms
00011848     461 (00011840)     _TickCNT100ms
00011849     461 (00011840)     _TickCNT1000ms
0001184a     461 (00011840)     _ADC_DebugOn
0001184b     461 (00011840)     _TickCNT10ms
0001184c     461 (00011840)     _IsrTicker1
0001184e     461 (00011840)     _PwmCarrier
00011850     461 (00011840)     _CurrentRisingEdgeDelay
00011852     461 (00011840)     _CurrentCarrier2
00011854     461 (00011840)     _PwmDuty
00011856     461 (00011840)     _PwmCarrier2
00011858     461 (00011840)     _PwmDuty2
0001185a     461 (00011840)     _CurrentFallingEdgeDelay2
0001185c     461 (00011840)     _CurrentRisingEdgeDelay2
0001185e     461 (00011840)     _CurrentCarrier
00011860     461 (00011840)     _CurrentFallingEdgeDelay
00011862     461 (00011840)     _CurrentDuty2
00011864     461 (00011840)     _CurrentDuty
00011866     461 (00011840)     _AdcA_Cur
0001186c     461 (00011840)     _AdcD_Cur
00011872     461 (00011840)     _AdcB_Cur
00011878     461 (00011840)     _AdcC_Cur

00047000    11c0 (00047000)     _Emif1Regs

00047800    11e0 (00047800)     _Emif2Regs

00050000    1400 (00050000)     _IpcRegs
00050024    1400 (00050000)     _FlashPumpSemaphoreRegs

0005d000    1740 (0005d000)     _DevCfgRegs

0005d180    1746 (0005d180)     _AnalogSubsysRegs

0005d200    1748 (0005d200)     _ClkCfgRegs

0005d300    174c (0005d300)     _CpuSysRegs

0005e608    1798 (0005e600)     _RomPrefetchRegs

0005f000    17c0 (0005f000)     _DcsmZ1Regs

0005f040    17c1 (0005f040)     _DcsmZ2Regs
0005f070    17c1 (0005f040)     _DcsmCommonRegs

0005f400    17d0 (0005f400)     _MemCfgRegs

0005f480    17d2 (0005f480)     _Emif1ConfigRegs
0005f4a0    17d2 (0005f480)     _Emif2ConfigRegs

0005f4c0    17d3 (0005f4c0)     _AccessProtectionRegs

0005f500    17d4 (0005f500)     _MemoryErrorRegs

0005f540    17d5 (0005f540)     _RomWaitStateRegs

0005f800    17e0 (0005f800)     _Flash0CtrlRegs

0005fb00    17ec (0005fb00)     _Flash0EccRegs

00078000    1e00 (00078000)     _DcsmZ1Otp

00078200    1e08 (00078200)     _DcsmZ2Otp

00088000    2200 (00088000)     _xdc_runtime_Text_charTab__A

0008a5c5    2297 (0008a5c0)     _ti_sysbios_family_c28_Hwi_Module__id__C

0008a80e    22a0 (0008a800)     _ti_sysbios_family_c28_Hwi_vectors

0008ab57    22ad (0008ab40)     __ctypes_

0008ad0b    22b4 (0008ad00)     _ti_sysbios_family_c28_Hwi_Module__loggerDefined__C

0008adab    22b6 (0008ad80)     _ti_sysbios_family_c28_Hwi_NUM_INTERRUPTS_ALL__C

0008aebd    22ba (0008ae80)     _ti_sysbios_family_c28_Hwi_Object__count__C

0008af29    22bc (0008af00)     _ti_sysbios_family_c28_TaskSupport_Module__id__C

0008af91    22be (0008af80)     _ti_sysbios_family_c28_Timer_Module__id__C

0008afec    22bf (0008afc0)     _xdc_runtime_Text_nodeTab__A

0008b09e    22c2 (0008b080)     _Ext1Hwi
0008b0a0    22c2 (0008b080)     _Ext2Hwi
0008b0a2    22c2 (0008b080)     _Ipc0Hwi
0008b0a4    22c2 (0008b080)     _Ipc0Mbx
0008b0a6    22c2 (0008b080)     _GPIOXint_Debug
0008b0a8    22c2 (0008b080)     _EmifEvent
0008b0aa    22c2 (0008b080)     _Ext3Hwi
0008b0ac    22c2 (0008b080)     _ExtIntEvent
0008b0ae    22c2 (0008b080)     _IntAppEvent
0008b0b0    22c2 (0008b080)     _IntAppMbx
0008b0b2    22c2 (0008b080)     _AdcCHwi
0008b0b4    22c2 (0008b080)     _AdcDHwi
0008b0b6    22c2 (0008b080)     _ePwmEvent
0008b0b8    22c2 (0008b080)     _EpwmMbx
0008b0ba    22c2 (0008b080)     _ePwm1Hwi
0008b0bc    22c2 (0008b080)     _ePwm4Hwi
0008b0be    22c2 (0008b080)     _CanATxRxTask

0008b0c0    22c3 (0008b0c0)     _CanBTxRxTask
0008b0c2    22c3 (0008b0c0)     _MgmtEvent
0008b0c4    22c3 (0008b0c0)     _MgmtMbx
0008b0c6    22c3 (0008b0c0)     _ControlTaskHd
0008b0c8    22c3 (0008b0c0)     _TickforTmr
0008b0ca    22c3 (0008b0c0)     _CMDtaskHd
0008b0cc    22c3 (0008b0c0)     _MgmtTaskHd
0008b0ce    22c3 (0008b0c0)     _CanAHwi
0008b0d0    22c3 (0008b0c0)     _CanBHwi
0008b0d2    22c3 (0008b0c0)     _EmifMbx
0008b0d4    22c3 (0008b0c0)     _EMIF_Debug
0008b0d6    22c3 (0008b0c0)     _CanBEvent
0008b0d8    22c3 (0008b0c0)     _CanBRxMbx
0008b0da    22c3 (0008b0c0)     _CanAEvent
0008b0dc    22c3 (0008b0c0)     _CanARxMbx
0008b0de    22c3 (0008b0c0)     _SpiBTaskHandle
0008b0e0    22c3 (0008b0c0)     _ExtDacEvent
0008b0e2    22c3 (0008b0c0)     _ExtAdcEvent
0008b0e4    22c3 (0008b0c0)     _SpiBMbx
0008b0e6    22c3 (0008b0c0)     _AdcAHwi
0008b0e8    22c3 (0008b0c0)     _AdcBHwi
0008b0ea    22c3 (0008b0c0)     _SpiCMbx
0008b0ec    22c3 (0008b0c0)     _SpiCTaskHandle
0008b0ee    22c3 (0008b0c0)     _SpiAMbx
0008b0f0    22c3 (0008b0c0)     _SpiATaskHandle
0008b0f2    22c3 (0008b0c0)     _adcResultSem

0008b21b    22c8 (0008b200)     _ti_sysbios_family_c28_Timer_startupNeeded__C

0008b263    22c9 (0008b240)     _ti_sysbios_gates_GateMutex_Module__id__C

0008b2a7    22ca (0008b280)     _ti_sysbios_hal_Hwi_Module__id__C

0008b31a    22cc (0008b300)     _xdc_runtime_LoggerBuf_Module__FXNS__C

0008b3a0    22ce (0008b380)     _xdc_runtime_Startup_sfxnTab__A

0008b3ca    22cf (0008b3c0)     _ti_sysbios_heaps_HeapMem_Module__FXNS__C
0008b3de    22cf (0008b3c0)     _ti_sysbios_gates_GateHwi_Module__FXNS__C
0008b3f0    22cf (0008b3c0)     _ti_sysbios_gates_GateMutex_Module__FXNS__C

0008b402    22d0 (0008b400)     _ti_sysbios_heaps_HeapMem_Object__PARAMS__C
0008b414    22d0 (0008b400)     _xdc_runtime_LoggerBuf_Object__PARAMS__C
0008b437    22d0 (0008b400)     _ti_sysbios_heaps_HeapMem_Module__id__C
0008b438    22d0 (0008b400)     _ti_sysbios_gates_GateHwi_Object__DESC__C

0008b448    22d1 (0008b440)     _ti_sysbios_gates_GateMutex_Object__DESC__C
0008b458    22d1 (0008b440)     _ti_sysbios_heaps_HeapMem_Object__DESC__C
0008b468    22d1 (0008b440)     _ti_sysbios_knl_Queue_Object__DESC__C
0008b478    22d1 (0008b440)     _ti_sysbios_knl_Semaphore_Object__DESC__C

0008b488    22d2 (0008b480)     _ti_sysbios_knl_Semaphore_Object__PARAMS__C
0008b498    22d2 (0008b480)     _xdc_runtime_LoggerBuf_Object__DESC__C
0008b4b4    22d2 (0008b480)     _ti_sysbios_gates_GateHwi_Object__PARAMS__C

0008b4c0    22d3 (0008b4c0)     _ti_sysbios_gates_GateMutex_Object__PARAMS__C
0008b4cc    22d3 (0008b4c0)     _ti_sysbios_knl_Queue_Object__PARAMS__C
0008b4d8    22d3 (0008b4c0)     _xdc_runtime_Startup_sfxnRts__A

0008b503    22d4 (0008b500)     _ti_sysbios_heaps_HeapMem_Object__count__C
0008b50a    22d4 (0008b500)     _xdc_runtime_Startup_firstFxns__A
0008b515    22d4 (0008b500)     _ti_sysbios_knl_Clock_Module__id__C
0008b516    22d4 (0008b500)     _ti_sysbios_knl_Idle_funcList__C
0008b51a    22d4 (0008b500)     _xdc_runtime_Startup_firstFxns__C
0008b51e    22d4 (0008b500)     _xdc_runtime_Startup_lastFxns__C
0008b522    22d4 (0008b500)     _ti_sysbios_BIOS_installedErrorHook__C
0008b524    22d4 (0008b500)     _ti_sysbios_family_c28_Hwi_A_badIntNum__C
0008b526    22d4 (0008b500)     _ti_sysbios_family_c28_Hwi_A_invalidArg__C
0008b528    22d4 (0008b500)     _ti_sysbios_family_c28_Hwi_E_unpluggedInterrupt__C
0008b52a    22d4 (0008b500)     _ti_sysbios_family_c28_Hwi_LD_end__C
0008b52c    22d4 (0008b500)     _ti_sysbios_family_c28_Hwi_LM_begin__C
0008b52e    22d4 (0008b500)     _ti_sysbios_family_c28_Hwi_Module__diagsEnabled__C
0008b530    22d4 (0008b500)     _ti_sysbios_family_c28_Hwi_Module__diagsIncluded__C
0008b532    22d4 (0008b500)     _ti_sysbios_family_c28_Hwi_Module__diagsMask__C
0008b534    22d4 (0008b500)     _ti_sysbios_family_c28_Hwi_Module__loggerFxn1__C
0008b536    22d4 (0008b500)     _ti_sysbios_family_c28_Hwi_Module__loggerFxn8__C
0008b538    22d4 (0008b500)     _ti_sysbios_family_c28_Hwi_Module__loggerObj__C
0008b53a    22d4 (0008b500)     _ti_sysbios_family_c28_Hwi_Object__table__C
0008b53c    22d4 (0008b500)     _ti_sysbios_family_c28_TaskSupport_E_invalidStack__C
0008b53e    22d4 (0008b500)     _ti_sysbios_family_c28_Timer_Module__diagsEnabled__C

0008b540    22d5 (0008b540)     _ti_sysbios_family_c28_Timer_Module__diagsIncluded__C
0008b542    22d5 (0008b540)     _ti_sysbios_family_c28_Timer_Module__diagsMask__C
0008b544    22d5 (0008b540)     _ti_sysbios_gates_GateMutex_A_badContext__C
0008b546    22d5 (0008b540)     _ti_sysbios_gates_GateMutex_Instance_State_sem__O
0008b548    22d5 (0008b540)     _ti_sysbios_gates_GateMutex_Module__diagsEnabled__C
0008b54a    22d5 (0008b540)     _ti_sysbios_gates_GateMutex_Module__diagsIncluded__C
0008b54c    22d5 (0008b540)     _ti_sysbios_gates_GateMutex_Module__diagsMask__C
0008b54e    22d5 (0008b540)     _ti_sysbios_hal_Hwi_E_stackOverflow__C
0008b550    22d5 (0008b540)     _ti_sysbios_heaps_HeapMem_A_align__C
0008b552    22d5 (0008b540)     _ti_sysbios_heaps_HeapMem_A_heapSize__C
0008b554    22d5 (0008b540)     _ti_sysbios_heaps_HeapMem_A_invalidFree__C
0008b556    22d5 (0008b540)     _ti_sysbios_heaps_HeapMem_A_zeroBlock__C
0008b558    22d5 (0008b540)     _ti_sysbios_heaps_HeapMem_E_memory__C
0008b55a    22d5 (0008b540)     _ti_sysbios_heaps_HeapMem_Module__diagsEnabled__C
0008b55c    22d5 (0008b540)     _ti_sysbios_heaps_HeapMem_Module__diagsIncluded__C
0008b55e    22d5 (0008b540)     _ti_sysbios_heaps_HeapMem_Module__diagsMask__C
0008b560    22d5 (0008b540)     _ti_sysbios_heaps_HeapMem_Module__gateObj__C
0008b562    22d5 (0008b540)     _ti_sysbios_heaps_HeapMem_Object__table__C
0008b564    22d5 (0008b540)     _ti_sysbios_heaps_HeapMem_reqAlign__C
0008b566    22d5 (0008b540)     _ti_sysbios_knl_Clock_LM_begin__C
0008b568    22d5 (0008b540)     _ti_sysbios_knl_Clock_LM_tick__C
0008b56a    22d5 (0008b540)     _ti_sysbios_knl_Clock_LW_delayed__C
0008b56c    22d5 (0008b540)     _ti_sysbios_knl_Clock_Module_State_clockQ__O
0008b56e    22d5 (0008b540)     _ti_sysbios_knl_Clock_Module__diagsEnabled__C
0008b570    22d5 (0008b540)     _ti_sysbios_knl_Clock_Module__diagsIncluded__C
0008b572    22d5 (0008b540)     _ti_sysbios_knl_Clock_Module__diagsMask__C
0008b574    22d5 (0008b540)     _ti_sysbios_knl_Clock_Module__loggerFxn1__C
0008b576    22d5 (0008b540)     _ti_sysbios_knl_Clock_Module__loggerFxn2__C
0008b578    22d5 (0008b540)     _ti_sysbios_knl_Clock_Module__loggerObj__C
0008b57a    22d5 (0008b540)     _ti_sysbios_knl_Event_A_badContext__C
0008b57c    22d5 (0008b540)     _ti_sysbios_knl_Event_A_eventInUse__C
0008b57e    22d5 (0008b540)     _ti_sysbios_knl_Event_A_nullEventId__C

0008b580    22d6 (0008b580)     _ti_sysbios_knl_Event_A_nullEventMasks__C
0008b582    22d6 (0008b580)     _ti_sysbios_knl_Event_A_pendTaskDisabled__C
0008b584    22d6 (0008b580)     _ti_sysbios_knl_Event_Instance_State_pendQ__O
0008b586    22d6 (0008b580)     _ti_sysbios_knl_Event_LM_pend__C
0008b588    22d6 (0008b580)     _ti_sysbios_knl_Event_LM_post__C
0008b58a    22d6 (0008b580)     _ti_sysbios_knl_Event_Module__diagsEnabled__C
0008b58c    22d6 (0008b580)     _ti_sysbios_knl_Event_Module__diagsIncluded__C
0008b58e    22d6 (0008b580)     _ti_sysbios_knl_Event_Module__diagsMask__C
0008b590    22d6 (0008b580)     _ti_sysbios_knl_Event_Module__loggerFxn4__C
0008b592    22d6 (0008b580)     _ti_sysbios_knl_Event_Module__loggerFxn8__C
0008b594    22d6 (0008b580)     _ti_sysbios_knl_Event_Module__loggerObj__C
0008b596    22d6 (0008b580)     _ti_sysbios_knl_Idle_funcList__A
0008b598    22d6 (0008b580)     _ti_sysbios_knl_Mailbox_Instance_State_dataQue__O
0008b59a    22d6 (0008b580)     _ti_sysbios_knl_Mailbox_Instance_State_dataSem__O
0008b59c    22d6 (0008b580)     _ti_sysbios_knl_Mailbox_Instance_State_freeQue__O
0008b59e    22d6 (0008b580)     _ti_sysbios_knl_Mailbox_Instance_State_freeSem__O
0008b5a0    22d6 (0008b580)     _ti_sysbios_knl_Mailbox_Object__table__C
0008b5a2    22d6 (0008b580)     _ti_sysbios_knl_Queue_Object__table__C
0008b5a4    22d6 (0008b580)     _ti_sysbios_knl_Semaphore_A_badContext__C
0008b5a6    22d6 (0008b580)     _ti_sysbios_knl_Semaphore_A_overflow__C
0008b5a8    22d6 (0008b580)     _ti_sysbios_knl_Semaphore_A_pendTaskDisabled__C
0008b5aa    22d6 (0008b580)     _ti_sysbios_knl_Semaphore_Instance_State_pendQ__O
0008b5ac    22d6 (0008b580)     _ti_sysbios_knl_Semaphore_LM_pend__C
0008b5ae    22d6 (0008b580)     _ti_sysbios_knl_Semaphore_LM_post__C
0008b5b0    22d6 (0008b580)     _ti_sysbios_knl_Semaphore_Module__diagsEnabled__C
0008b5b2    22d6 (0008b580)     _ti_sysbios_knl_Semaphore_Module__diagsIncluded__C
0008b5b4    22d6 (0008b580)     _ti_sysbios_knl_Semaphore_Module__diagsMask__C
0008b5b6    22d6 (0008b580)     _ti_sysbios_knl_Semaphore_Module__loggerFxn2__C
0008b5b8    22d6 (0008b580)     _ti_sysbios_knl_Semaphore_Module__loggerFxn4__C
0008b5ba    22d6 (0008b580)     _ti_sysbios_knl_Semaphore_Module__loggerObj__C
0008b5bc    22d6 (0008b580)     _ti_sysbios_knl_Semaphore_eventPost__C
0008b5be    22d6 (0008b580)     _ti_sysbios_knl_Semaphore_eventSync__C

0008b5c0    22d7 (0008b5c0)     _ti_sysbios_knl_Swi_LD_end__C
0008b5c2    22d7 (0008b5c0)     _ti_sysbios_knl_Swi_LM_begin__C
0008b5c4    22d7 (0008b5c0)     _ti_sysbios_knl_Swi_LM_post__C
0008b5c6    22d7 (0008b5c0)     _ti_sysbios_knl_Swi_Module__diagsEnabled__C
0008b5c8    22d7 (0008b5c0)     _ti_sysbios_knl_Swi_Module__diagsIncluded__C
0008b5ca    22d7 (0008b5c0)     _ti_sysbios_knl_Swi_Module__diagsMask__C
0008b5cc    22d7 (0008b5c0)     _ti_sysbios_knl_Swi_Module__loggerFxn1__C
0008b5ce    22d7 (0008b5c0)     _ti_sysbios_knl_Swi_Module__loggerFxn4__C
0008b5d0    22d7 (0008b5c0)     _ti_sysbios_knl_Swi_Module__loggerObj__C
0008b5d2    22d7 (0008b5c0)     _ti_sysbios_knl_Swi_Object__table__C
0008b5d4    22d7 (0008b5c0)     _ti_sysbios_knl_Task_A_badTimeout__C
0008b5d6    22d7 (0008b5c0)     _ti_sysbios_knl_Task_A_sleepTaskDisabled__C
0008b5d8    22d7 (0008b5c0)     _ti_sysbios_knl_Task_E_spOutOfBounds__C
0008b5da    22d7 (0008b5c0)     _ti_sysbios_knl_Task_E_stackOverflow__C
0008b5dc    22d7 (0008b5c0)     _ti_sysbios_knl_Task_LD_block__C
0008b5de    22d7 (0008b5c0)     _ti_sysbios_knl_Task_LD_exit__C
0008b5e0    22d7 (0008b5c0)     _ti_sysbios_knl_Task_LD_ready__C
0008b5e2    22d7 (0008b5c0)     _ti_sysbios_knl_Task_LM_sleep__C
0008b5e4    22d7 (0008b5c0)     _ti_sysbios_knl_Task_LM_switch__C
0008b5e6    22d7 (0008b5c0)     _ti_sysbios_knl_Task_Module_State_inactiveQ__O
0008b5e8    22d7 (0008b5c0)     _ti_sysbios_knl_Task_Module__diagsEnabled__C
0008b5ea    22d7 (0008b5c0)     _ti_sysbios_knl_Task_Module__diagsIncluded__C
0008b5ec    22d7 (0008b5c0)     _ti_sysbios_knl_Task_Module__diagsMask__C
0008b5ee    22d7 (0008b5c0)     _ti_sysbios_knl_Task_Module__loggerFxn2__C
0008b5f0    22d7 (0008b5c0)     _ti_sysbios_knl_Task_Module__loggerFxn4__C
0008b5f2    22d7 (0008b5c0)     _ti_sysbios_knl_Task_Module__loggerObj__C
0008b5f4    22d7 (0008b5c0)     _ti_sysbios_knl_Task_Object__table__C
0008b5f6    22d7 (0008b5c0)     _ti_sysbios_knl_Task_allBlockedFunc__C
0008b5fc    22d7 (0008b5c0)     _xdc_runtime_Assert_E_assertFailed__C
0008b5fe    22d7 (0008b5c0)     _xdc_runtime_Core_A_initializedParams__C

0008b600    22d8 (0008b600)     _xdc_runtime_Core_Module__diagsEnabled__C
0008b602    22d8 (0008b600)     _xdc_runtime_Core_Module__diagsIncluded__C
0008b604    22d8 (0008b600)     _xdc_runtime_Core_Module__diagsMask__C
0008b606    22d8 (0008b600)     _xdc_runtime_Error_E_memory__C
0008b608    22d8 (0008b600)     _xdc_runtime_Error_Module__diagsEnabled__C
0008b60a    22d8 (0008b600)     _xdc_runtime_Error_Module__diagsIncluded__C
0008b60c    22d8 (0008b600)     _xdc_runtime_Error_Module__diagsMask__C
0008b60e    22d8 (0008b600)     _xdc_runtime_Error_Module__loggerFxn8__C
0008b610    22d8 (0008b600)     _xdc_runtime_Error_Module__loggerObj__C
0008b612    22d8 (0008b600)     _xdc_runtime_Error_policyFxn__C
0008b614    22d8 (0008b600)     _xdc_runtime_Error_raiseHook__C
0008b616    22d8 (0008b600)     _xdc_runtime_IFilterLogger_Interface__BASE__C
0008b618    22d8 (0008b600)     _xdc_runtime_IGateProvider_Interface__BASE__C
0008b61a    22d8 (0008b600)     _xdc_runtime_IHeap_Interface__BASE__C
0008b61c    22d8 (0008b600)     _xdc_runtime_ILogger_Interface__BASE__C
0008b61e    22d8 (0008b600)     _xdc_runtime_IModule_Interface__BASE__C
0008b620    22d8 (0008b600)     _xdc_runtime_Log_L_error__C
0008b622    22d8 (0008b600)     _xdc_runtime_LoggerBuf_E_badLevel__C
0008b624    22d8 (0008b600)     _xdc_runtime_LoggerBuf_Module__gateObj__C
0008b626    22d8 (0008b600)     _xdc_runtime_LoggerBuf_Object__table__C
0008b628    22d8 (0008b600)     _xdc_runtime_LoggerBuf_statusLogger__C
0008b62a    22d8 (0008b600)     _xdc_runtime_Main_Module__diagsEnabled__C
0008b62c    22d8 (0008b600)     _xdc_runtime_Main_Module__diagsIncluded__C
0008b62e    22d8 (0008b600)     _xdc_runtime_Main_Module__diagsMask__C
0008b630    22d8 (0008b600)     _xdc_runtime_Memory_defaultHeapInstance__C
0008b632    22d8 (0008b600)     _xdc_runtime_Startup_execImpl__C
0008b634    22d8 (0008b600)     _xdc_runtime_Startup_sfxnRts__C
0008b636    22d8 (0008b600)     _xdc_runtime_Startup_sfxnTab__C
0008b638    22d8 (0008b600)     _xdc_runtime_Startup_startModsFxn__C
0008b63a    22d8 (0008b600)     _xdc_runtime_SysMin_bufSize__C
0008b63c    22d8 (0008b600)     _xdc_runtime_SysMin_outputFunc__C
0008b63e    22d8 (0008b600)     _xdc_runtime_System_Module__gateObj__C

0008b640    22d9 (0008b640)     _xdc_runtime_System_abortFxn__C
0008b642    22d9 (0008b640)     _xdc_runtime_System_exitFxn__C
0008b644    22d9 (0008b640)     _xdc_runtime_System_extendFxn__C
0008b646    22d9 (0008b640)     _xdc_runtime_Text_charTab__C
0008b648    22d9 (0008b640)     _xdc_runtime_Text_nameEmpty__C
0008b64a    22d9 (0008b640)     _xdc_runtime_Text_nameStatic__C
0008b64c    22d9 (0008b640)     _xdc_runtime_Text_nameUnknown__C
0008b64e    22d9 (0008b640)     _xdc_runtime_Text_nodeTab__C
0008b650    22d9 (0008b640)     _xdc_runtime_Text_visitRopeFxn__C
0008b652    22d9 (0008b640)     _ti_sysbios_knl_Clock_Module__loggerDefined__C
0008b653    22d9 (0008b640)     _ti_sysbios_knl_Event_Module__id__C
0008b654    22d9 (0008b640)     _ti_sysbios_knl_Event_Module__loggerDefined__C
0008b655    22d9 (0008b640)     _ti_sysbios_knl_Mailbox_Object__count__C
0008b656    22d9 (0008b640)     _ti_sysbios_knl_Mailbox_maxTypeAlign__C
0008b657    22d9 (0008b640)     _ti_sysbios_knl_Queue_Object__count__C
0008b658    22d9 (0008b640)     _ti_sysbios_knl_Semaphore_Module__id__C
0008b659    22d9 (0008b640)     _ti_sysbios_knl_Semaphore_Module__loggerDefined__C
0008b65a    22d9 (0008b640)     _ti_sysbios_knl_Swi_Module__id__C
0008b65b    22d9 (0008b640)     _ti_sysbios_knl_Swi_Module__loggerDefined__C
0008b65c    22d9 (0008b640)     _ti_sysbios_knl_Swi_Object__count__C
0008b65d    22d9 (0008b640)     _ti_sysbios_knl_Task_Module__id__C
0008b65e    22d9 (0008b640)     _ti_sysbios_knl_Task_Module__loggerDefined__C
0008b65f    22d9 (0008b640)     _ti_sysbios_knl_Task_Object__count__C
0008b660    22d9 (0008b640)     _ti_sysbios_knl_Task_numConstructedTasks__C
0008b661    22d9 (0008b640)     _xdc_runtime_Core_Module__id__C
0008b662    22d9 (0008b640)     _xdc_runtime_Error_Module__loggerDefined__C
0008b663    22d9 (0008b640)     _xdc_runtime_Error_maxDepth__C
0008b664    22d9 (0008b640)     _xdc_runtime_Error_policy__C
0008b665    22d9 (0008b640)     _xdc_runtime_LoggerBuf_Module__id__C
0008b666    22d9 (0008b640)     _xdc_runtime_LoggerBuf_Object__count__C
0008b667    22d9 (0008b640)     _xdc_runtime_LoggerBuf_filterByLevel__C
0008b668    22d9 (0008b640)     _xdc_runtime_Main_Module__id__C
0008b669    22d9 (0008b640)     _xdc_runtime_Memory_Module__id__C
0008b66a    22d9 (0008b640)     _xdc_runtime_Startup_maxPasses__C
0008b66b    22d9 (0008b640)     _xdc_runtime_SysMin_flushAtExit__C
0008b66c    22d9 (0008b640)     _xdc_runtime_System_maxAtexitHandlers__C
0008b66d    22d9 (0008b640)     _xdc_runtime_Text_charCnt__C
0008b66e    22d9 (0008b640)     _xdc_runtime_Text_isLoaded__C
0008b66f    22d9 (0008b640)     _xdc_runtime_Text_registryModsLastId__C
0008b670    22d9 (0008b640)     _xdc_runtime_Text_unnamedModsLastId__C


GLOBAL SYMBOLS: SORTED ALPHABETICALLY BY Name 

page  address   name                                                      
----  -------   ----                                                      
abs   ffffffff  .text                                                     
0     00087138  C$$EXIT                                                   
0     00085bb3  C$$IO$$                                                   
0     000858ff  FD$$ADD                                                   
0     000870e4  FD$$CMP                                                   
0     00085c82  FD$$DIV                                                   
0     00085e14  FD$$MPY                                                   
0     00087bf8  FD$$NEG                                                   
0     00087a1d  FD$$SUB                                                   
0     000872a7  FD$$TOI                                                   
0     00087345  FD$$TOL                                                   
0     0008744d  FS$$TOFD                                                  
0     00087243  I$$DIV                                                    
0     00087254  I$$MOD                                                    
0     000873f8  I$$TOFD                                                   
0     0008710e  L$$DIV                                                    
0     0008711d  L$$MOD                                                    
0     00087469  L$$TOFD                                                   
0     000876e7  LL$$AND                                                   
0     00087382  LL$$CMP                                                   
0     0008462d  LL$$DIV                                                   
0     00084669  LL$$MOD                                                   
0     000876ef  LL$$OR                                                    
0     000876f7  LL$$XOR                                                   
0     00087ba3  U$$DIV                                                    
0     00087ba8  U$$MOD                                                    
0     0008712b  UL$$DIV                                                   
0     00087132  UL$$MOD                                                   
0     00087394  ULL$$CMP                                                  
0     000846a3  ULL$$DIV                                                  
0     000846d2  ULL$$MOD                                                  
0     0008643d  _AD5764_SPIB_CS_HIGH                                      
0     00086438  _AD5764_SPIB_CS_LOW                                       
0     00086442  _AD5764_SPIC_Init                                         
0     000851bd  _AD5764_SPIC_ReadByte                                     
0     000851ca  _AD5764_SPIC_ReadWord                                     
0     0008646e  _AD5764_SPIC_Read_DAC                                     
0     000851b6  _AD5764_SPIC_SendByte                                     
0     000851c3  _AD5764_SPIC_SendWord                                     
0     0008644d  _AD5764_SPIC_Write_DAC                                    
0     00084f84  _AD7689_SPIB_CS_HIGH                                      
0     00084f7c  _AD7689_SPIB_CS_LOW                                       
0     00084927  _AD7689_SPIB_Init                                         
0     00084f69  _AD7689_SPIB_ReadByte                                     
0     00084f76  _AD7689_SPIB_ReadWord                                     
0     0008492d  _AD7689_SPIB_Read_All_Raw                                 
0     00084f6f  _AD7689_SPIB_SendWord                                     
0     00084f62  _AD7689_SPI_SendByte                                      
1     0001184a  _ADC_DebugOn                                              
1     00011844  _ADC_Display_Interval                                     
1     0005f4c0  _AccessProtectionRegs                                     
1     00011843  _Acnt                                                     
0     00085500  _AdcA1_Isr                                                
0     0008b0e6  _AdcAHwi                                                  
1     00011866  _AdcA_Cur                                                 
0     000855b5  _AdcB1_Isr                                                
0     0008b0e8  _AdcBHwi                                                  
1     00011872  _AdcB_Cur                                                 
0     00084d5b  _AdcC1_Isr                                                
0     0008b0b2  _AdcCHwi                                                  
1     00011878  _AdcC_Cur                                                 
0     00084f00  _AdcD1_Isr                                                
0     0008b0b4  _AdcDHwi                                                  
1     0001186c  _AdcD_Cur                                                 
0     00084bbe  _AdcSetMode                                               
1     00007400  _AdcaRegs                                                 
1     00000b00  _AdcaResultRegs                                           
1     00007480  _AdcbRegs                                                 
1     00000b20  _AdcbResultRegs                                           
1     00007500  _AdccRegs                                                 
1     00000b40  _AdccResultRegs                                           
1     00007580  _AdcdRegs                                                 
1     00000b60  _AdcdResultRegs                                           
1     000112c1  _Aerror_message                                           
1     0005d180  _AnalogSubsysRegs                                         
0     00081e1b  _AuxAuxClkSel                                             
0     00081e05  _AuxIntOsc2Sel                                            
0     00081e0f  _AuxXtalOscSel                                            
1     00011842  _BackTicker                                               
1     00011841  _Bcnt                                                     
1     000112c2  _Berror_message                                           
0     00080d9d  _CANAIntHandler                                           
1     000112c0  _CANA_Err_Int_Enable                                      
0     00080fc5  _CANBIntHandler                                           
1     000112c4  _CANB_Err_Int_Enable                                      
0     0008275b  _CANBitRateSet                                            
0     00082730  _CANBitTimingGet                                          
0     000827ca  _CANBitTimingSet                                          
0     00082709  _CANClkSourceSelect                                       
0     00082701  _CANDisable                                               
0     000826f8  _CANEnable                                                
0     000828d6  _CANErrCntrGet                                            
0     00082af2  _CANGlobalIntClear                                        
0     00082ae8  _CANGlobalIntDisable                                      
0     00082adf  _CANGlobalIntEnable                                       
0     00082afb  _CANGlobalIntstatusGet                                    
0     0008264b  _CANInit                                                  
0     0008286a  _CANIntClear                                              
0     00082840  _CANIntDisable                                            
0     00082832  _CANIntEnable                                             
0     00082815  _CANIntRegister                                           
0     00082850  _CANIntStatus                                             
0     00082825  _CANIntUnregister                                         
0     00082ab9  _CANMessageClear                                          
0     000829e3  _CANMessageGet                                            
0     000828f1  _CANMessageSet                                            
0     000828a4  _CANRetryGet                                              
0     00082893  _CANRetrySet                                              
0     000828ae  _CANStatusGet                                             
1     000112c3  _CAN_DebugOn                                              
0     0008b0ca  _CMDtaskHd                                                
0     00084c61  _CalAdcINL                                                
0     0008b0da  _CanAEvent                                                
0     0008b0ce  _CanAHwi                                                  
0     0008b0dc  _CanARxMbx                                                
0     0008b0be  _CanATxRxTask                                             
0     0008127f  _CanA_EableTxRx                                           
0     00080da7  _CanA_TxRx_Task                                           
0     0008b0d6  _CanBEvent                                                
0     0008b0d0  _CanBHwi                                                  
0     0008b0d8  _CanBRxMbx                                                
0     0008b0c0  _CanBTxRxTask                                             
0     0008136e  _CanB_EableTxRx                                           
0     00080fcf  _CanB_TxRx_Task                                           
0     00080d70  _CanMsg_prnt                                              
1     00011840  _Ccnt                                                     
1     00001400  _Cla1Regs                                                 
0     00000ce0  _Cla1SoftIntRegs                                          
1     0005d200  _ClkCfgRegs                                               
0     000868d0  _CmdLineProcess                                           
0     000814b5  _Cmd_Can                                                  
0     00081582  _Cmd_CanDebug                                             
0     00081561  _Cmd_CanRpt                                               
0     000818b7  _Cmd_Dac                                                  
0     00081816  _Cmd_EMIF1_ContiRD                                        
0     000815fb  _Cmd_EMIF1_RD                                             
0     000815c0  _Cmd_EMIF1_WR                                             
0     000816b2  _Cmd_ExtAdcDebug                                          
0     000816d9  _Cmd_ExtAdcDisplay                                        
0     00081836  _Cmd_ExtIntDebug                                          
0     0008185d  _Cmd_ExtIntEnable                                         
0     00081637  _Cmd_IntAdcDebug                                          
0     0008168b  _Cmd_IntAdcDisplay                                        
0     0008148f  _Cmd_IntTmr                                               
0     00081a9b  _Cmd_Task                                                 
0     00081869  _Cmd_TempDebug                                            
0     00081890  _Cmd_TempDisplay                                          
0     00081974  _Cmd_epwm_Carrier                                         
0     00081a21  _Cmd_epwm_Debug                                           
0     000818f1  _Cmd_epwm_Duty                                            
0     000819e1  _Cmd_epwm_Info                                            
0     00081a69  _Cmd_help                                                 
0     00081700  _Cmd_readGPIO                                             
0     00081750  _Cmd_readGPIOAll                                          
0     000817a7  _Cmd_writeGPIO                                            
1     00005c80  _Cmpss1Regs                                               
1     00005ca0  _Cmpss2Regs                                               
1     00005cc0  _Cmpss3Regs                                               
1     00005ce0  _Cmpss4Regs                                               
1     00005d00  _Cmpss5Regs                                               
1     00005d20  _Cmpss6Regs                                               
1     00005d40  _Cmpss7Regs                                               
1     00005d60  _Cmpss8Regs                                               
0     00085460  _ConfigureAdcA                                            
0     00085515  _ConfigureAdcB                                            
0     00084cab  _ConfigureAdcC                                            
0     00084e5a  _ConfigureAdcD                                            
0     00086180  _ConfigureUART                                            
0     0008b0c6  _ControlTaskHd                                            
1     0005d300  _CpuSysRegs                                               
1     00000c00  _CpuTimer0Regs                                            
1     00000c08  _CpuTimer1Regs                                            
1     00000c10  _CpuTimer2Regs                                            
0     00081dc4  _CsmUnlock                                                
1     0001185e  _CurrentCarrier                                           
1     00011852  _CurrentCarrier2                                          
1     00011864  _CurrentDuty                                              
1     00011862  _CurrentDuty2                                             
1     00011860  _CurrentFallingEdgeDelay                                  
1     0001185a  _CurrentFallingEdgeDelay2                                 
1     00011850  _CurrentRisingEdgeDelay                                   
1     0001185c  _CurrentRisingEdgeDelay2                                  
1     00005c00  _DacaRegs                                                 
1     00005c10  _DacbRegs                                                 
1     00005c20  _DaccRegs                                                 
1     00011845  _Dcnt                                                     
1     0005f070  _DcsmCommonRegs                                           
1     00078000  _DcsmZ1Otp                                                
1     0005f000  _DcsmZ1Regs                                               
1     00078200  _DcsmZ2Otp                                                
1     0005f040  _DcsmZ2Regs                                               
1     0005d000  _DevCfgRegs                                               
0     00081c28  _DisableDog                                               
0     00081be9  _DisablePeripheralClocks                                  
1     00007980  _DmaClaSrcSelRegs                                         
1     00001000  _DmaRegs                                                  
1     00005000  _ECap1Regs                                                
1     00005020  _ECap2Regs                                                
1     00005040  _ECap3Regs                                                
1     00005060  _ECap4Regs                                                
1     00005080  _ECap5Regs                                                
1     000050a0  _ECap6Regs                                                
0     0008b0d4  _EMIF_Debug                                               
0     0008534b  _EMIF_Debug_Task                                          
0     00085397  _EMIF_Debug_Tick                                          
1     00010276  _EMIF_Display_Interval                                    
1     00010278  _EMIF_Read_OffAddr                                        
1     00004900  _EPwm10Regs                                               
1     00004a00  _EPwm11Regs                                               
1     00004b00  _EPwm12Regs                                               
0     000861eb  _EPwm1Isr                                                 
1     00004000  _EPwm1Regs                                                
0     000861fa  _EPwm2Isr                                                 
1     00004100  _EPwm2Regs                                                
1     00004200  _EPwm3Regs                                                
0     00086206  _EPwm4Isr                                                 
1     00004300  _EPwm4Regs                                                
0     00086215  _EPwm5Isr                                                 
1     00004400  _EPwm5Regs                                                
1     00004500  _EPwm6Regs                                                
1     00004600  _EPwm7Regs                                                
1     00004700  _EPwm8Regs                                                
1     00004800  _EPwm9Regs                                                
1     00007a00  _EPwmXbarRegs                                             
1     00005100  _EQep1Regs                                                
1     00005140  _EQep2Regs                                                
1     00005180  _EQep3Regs                                                
1     00010272  _Ecnt                                                     
1     0005f480  _Emif1ConfigRegs                                          
1     00047000  _Emif1Regs                                                
1     0005f4a0  _Emif2ConfigRegs                                          
1     00047800  _Emif2Regs                                                
0     0008b0a8  _EmifEvent                                                
0     0008b0d2  _EmifMbx                                                  
1     00010274  _Emif_DebugOn                                             
0     00000d01  _EmuBMode                                                 
0     00000d00  _EmuKey                                                   
0     00085de7  _Enable_SpiA_for_TMP123                                   
0     00084fb5  _Enable_SpiB_for_AD7689                                   
0     000851fb  _Enable_SpiC_for_AD5764                                   
0     0008b0b8  _EpwmMbx                                                  
1     00010275  _ErrCount                                                 
0     0008b09e  _Ext1Hwi                                                  
0     0008b0a0  _Ext2Hwi                                                  
0     0008b0aa  _Ext3Hwi                                                  
1     0000ee27  _ExtADC_DebugOn                                           
1     0000ee28  _ExtADC_Display_Interval                                  
0     0008b0e2  _ExtAdcEvent                                              
1     0000ee03  _ExtDAC_DebugOn                                           
0     0008b0e0  _ExtDacEvent                                              
0     0008b0ac  _ExtIntEvent                                              
1     00011780  _ExtInt_DebugOn                                           
1     0000ee26  _Extcnt                                                   
0     00008037  _F28x_usDelay                                             
1     0005f800  _Flash0CtrlRegs                                           
1     0005fb00  _Flash0EccRegs                                            
0     00008029  _FlashOff                                                 
1     00050024  _FlashPumpSemaphoreRegs                                   
0     0008b0a6  _GPIOXint_Debug                                           
0     000845f6  _GPIOXint_Debug_Task                                      
1     000117c0  _GPIO_Conf_InitVal                                        
0     0008372c  _GPIO_EnableUnbondedIOPullups                             
0     00083707  _GPIO_EnableUnbondedIOPullupsFor100Pin                    
0     000836ee  _GPIO_EnableUnbondedIOPullupsFor176Pin                    
0     00083742  _GPIO_ReadPin                                             
0     00083693  _GPIO_SetupLock                                           
0     00083573  _GPIO_SetupPinMux                                         
0     000835ff  _GPIO_SetupPinOptions                                     
0     000836bc  _GPIO_SetupXINT1Gpio                                      
0     000836c6  _GPIO_SetupXINT2Gpio                                      
0     000836d0  _GPIO_SetupXINT3Gpio                                      
0     000836da  _GPIO_SetupXINT4Gpio                                      
0     000836e4  _GPIO_SetupXINT5Gpio                                      
0     00083759  _GPIO_WritePin                                            
1     00007c00  _GpioCtrlRegs                                             
1     00007f00  _GpioDataRegs                                             
0     00081e39  _HALT                                                     
0     00081e52  _HIB                                                      
0     00083037  _HOSTclock                                                
0     0008300e  _HOSTclose                                                
0     00082fe6  _HOSTgetenv                                               
0     00082f85  _HOSTlseek                                                
0     00082f45  _HOSTopen                                                 
0     00082f06  _HOSTread                                                 
0     00082ec8  _HOSTrename                                               
0     00082e92  _HOSTtime                                                 
0     00082e4d  _HOSTtime64                                               
0     00082e29  _HOSTunlink                                               
0     00082df1  _HOSTwrite                                                
1     00007300  _I2caRegs                                                 
1     00007340  _I2cbRegs                                                 
0     00081e25  _IDLE                                                     
0     00087431  _IPC2_ISR                                                 
0     0008743f  _IPC3_ISR                                                 
1     0000f900  _IdTable_Mot                                              
0     00085454  _InitAdcA                                                 
0     00085509  _InitAdcB                                                 
0     00084c9b  _InitAdcC                                                 
0     00084e4a  _InitAdcD                                                 
0     00081cfc  _InitAuxPll                                               
0     000811ed  _InitCanA                                                 
0     00081236  _InitCanB                                                 
0     00086221  _InitEPwm                                                 
0     000847f7  _InitEPwm10Gpio                                           
0     0008480a  _InitEPwm11Gpio                                           
0     0008481e  _InitEPwm12Gpio                                           
0     0008474d  _InitEPwm1Gpio                                            
0     0008475f  _InitEPwm2Gpio                                            
0     00084771  _InitEPwm3Gpio                                            
0     00084785  _InitEPwm4Gpio                                            
0     00084799  _InitEPwm5Gpio                                            
0     000847ab  _InitEPwm6Gpio                                            
0     000847bd  _InitEPwm7Gpio                                            
0     000847d1  _InitEPwm8Gpio                                            
0     000847e5  _InitEPwm9Gpio                                            
0     00084734  _InitEPwmGpio                                             
0     00008000  _InitFlash                                                
0     00083533  _InitGpio                                                 
0     00084525  _InitGpio_PMCU                                            
0     00085acb  _InitIPCwithCPU2                                          
0     00081b65  _InitPeripheralClocks                                     
0     00085862  _InitSpiGpio                                              
0     00085869  _InitSpiaGpio                                             
0     0008588f  _InitSpibGpio                                             
0     000858c5  _InitSpicGpio                                             
0     00081b28  _InitSysCtrl                                              
0     00081c36  _InitSysPll                                               
0     00086d4b  _Init_IntTmr                                              
1     00007900  _InputXbarRegs                                            
0     000841a1  _IntAdc_prnt                                              
0     0008b0ae  _IntAppEvent                                              
0     0008b0b0  _IntAppMbx                                                
0     000879c8  _IntDefaultHandler                                        
0     00083ea2  _IntDisable                                               
0     00083e0f  _IntEnable                                                
0     00083f22  _IntIFRClear                                              
0     00083ddf  _IntMasterDisable                                         
0     00083dd7  _IntMasterEnable                                          
0     00083de7  _IntRegister                                              
0     00083dfa  _IntUnregister                                            
0     0008b0a2  _Ipc0Hwi                                                  
0     0008b0a4  _Ipc0Mbx                                                  
0     00085b38  _Ipc0_Isr                                                 
0     00085b4a  _Ipc1_Isr                                                 
1     00050000  _IpcRegs                                                  
0     00085b52  _IpcRx_Task                                               
1     0000ef80  _IqTable_Mot                                              
1     0001184c  _IsrTicker1                                               
1     00011846  _IsrTicker4                                               
0     0008769f  _LoggerBuf_instanceStartup                                
1     0000ee42  _MFluxIndex                                               
1     0000ee80  _MFluxTable                                               
1     0000ee22  _M_delta                                                  
1     0000ee20  _M_new                                                    
1     0000ee16  _M_old                                                    
1     0000ee4c  _MagFlux                                                  
1     00006000  _McbspaRegs                                               
1     00006040  _McbspbRegs                                               
1     0005f400  _MemCfgRegs                                               
1     0005f500  _MemoryErrorRegs                                          
0     0008b0c2  _MgmtEvent                                                
0     0008b0c4  _MgmtMbx                                                  
0     0008b0cc  _MgmtTaskHd                                               
0     00086d61  _Mgmt_Task                                                
1     00007060  _NmiIntruptRegs                                           
1     00007a80  _OutputXbarRegs                                           
1     00000ce0  _PieCtrlRegs                                              
0     00000d00  _PieVectTable                                             
1     0001184e  _PwmCarrier                                               
1     00011856  _PwmCarrier2                                              
1     00011854  _PwmDuty                                                  
1     00011858  _PwmDuty2                                                 
0     000800bf  _RamfuncsLoadEnd                                          
abs   0000003f  _RamfuncsLoadSize                                         
0     00080080  _RamfuncsLoadStart                                        
0     0000803f  _RamfuncsRunEnd                                           
abs   0000003f  _RamfuncsRunSize                                          
0     00008000  _RamfuncsRunStart                                         
0     00081c10  _ReleaseFlashPump                                         
1     0005e608  _RomPrefetchRegs                                          
1     0005f540  _RomWaitStateRegs                                         
0     00081e2e  _STANDBY                                                  
1     00007200  _SciaRegs                                                 
1     00007210  _ScibRegs                                                 
1     00007220  _ScicRegs                                                 
1     00007230  _ScidRegs                                                 
1     00005e00  _Sdfm1Regs                                                
1     00005e80  _Sdfm2Regs                                                
0     00081c01  _SeizeFlashPump                                           
0     00085b0b  _Send_Ipc2CPU2                                            
0     00081c1a  _ServiceDog                                               
0     00085dbf  _Set_max_speed_for_SpiA                                   
0     00084f8c  _Set_max_speed_for_SpiB                                   
0     000851d0  _Set_max_speed_for_SpiC                                   
0     00085480  _SetupAdcA                                                
0     00085535  _SetupAdcB                                                
0     00084ccb  _SetupAdcC                                                
0     00084e7a  _SetupAdcDsoftware                                        
0     00084583  _Setup_GPIO_for_ExtInterrupt                              
1     0000ee41  _SpeedIndex                                               
0     0008b0ee  _SpiAMbx                                                  
0     0008b0f0  _SpiATaskHandle                                           
0     00083fa1  _SpiA_Task                                                
0     0008b0e4  _SpiBMbx                                                  
0     0008b0de  _SpiBTaskHandle                                           
0     00085d31  _SpiB_Task                                                
0     0008b0ea  _SpiCMbx                                                  
0     0008b0ec  _SpiCTaskHandle                                           
0     00086960  _SpiC_Task                                                
1     00006100  _SpiaRegs                                                 
1     00006110  _SpibRegs                                                 
1     00006120  _SpicRegs                                                 
0     0008547b  _StartAdcAsoftware                                        
0     00085530  _StartAdcBsoftware                                        
0     00084cc6  _StartAdcCsoftware                                        
0     00084e75  _StartAdcDsoftware                                        
1     00007940  _SyncSocRegs                                              
0     0008393a  _SysCtlAuxClockSet                                        
0     0008383b  _SysCtlClockGet                                           
0     0008389e  _SysCtlClockSet                                           
0     0000803b  _SysCtlDelay                                              
0     00083887  _SysCtlLowSpeedClockGet                                   
0     00083816  _SysCtlPeripheralDisable                                  
0     000837fc  _SysCtlPeripheralEnable                                   
0     00083777  _SysCtlPeripheralPresent                                  
0     00083796  _SysCtlPeripheralReady                                    
0     000837d0  _SysCtlPeripheralReset                                    
0     00083831  _SysCtlReset                                              
0     000839b9  _SysCtlUSBPLLDisable                                      
0     000839b8  _SysCtlUSBPLLEnable                                       
0     00081de5  _SysIntOsc1Sel                                            
0     00081def  _SysIntOsc2Sel                                            
0     00081df9  _SysXtalOscSel                                            
1     0000ee0a  _T1_delta                                                 
1     0001027a  _TEST_STATUS                                              
0     00085db3  _TMP123_SPIA_ReadByte                                     
0     00085db9  _TMP123_SPIA_ReadWord                                     
1     0000ee1a  _T_ov                                                     
0     000841c0  _Task_Control                                             
1     00011596  _TempReadInterval                                         
1     00011597  _Temp_DebugOn                                             
0     00085ae4  _Test_memcpy                                              
1     00011849  _TickCNT1000ms                                            
1     00011848  _TickCNT100ms                                             
1     0001184b  _TickCNT10ms                                              
1     00011847  _TickCNT500ms                                             
0     00085d8a  _TickExtAdc_Isr                                           
0     000842dd  _TickTmr_Isr                                              
0     0008b0c8  _TickforTmr                                               
1     0000ee40  _TorqueIndex                                              
0     00082ca4  _UARTBusy                                                 
0     00082c6c  _UARTCharGet                                              
0     00082c47  _UARTCharGetNonBlocking                                   
0     00082c97  _UARTCharPut                                              
0     00082c84  _UARTCharPutNonBlocking                                   
0     00082c10  _UARTCharsAvail                                           
0     00082b92  _UARTConfigGetExpClk                                      
0     00082b63  _UARTConfigSetExpClk                                      
0     00082bc0  _UARTDisable                                              
0     00082bb6  _UARTEnable                                               
0     00082bed  _UARTFIFODisable                                          
0     00082be4  _UARTFIFOEnable                                           
0     00082b35  _UARTFIFOIntLevelGet                                      
0     00082b1b  _UARTFIFOIntLevelSet                                      
0     00082b4b  _UARTFIFOLevelGet                                         
0     00082da8  _UARTIntClear                                             
0     00082d42  _UARTIntDisable                                           
0     00082d11  _UARTIntEnable                                            
0     00082d78  _UARTIntStatus                                            
0     00082b12  _UARTParityModeGet                                        
0     00082b08  _UARTParityModeSet                                        
0     00082cb5  _UARTRXIntRegister                                        
0     00082ce5  _UARTRXIntUnregister                                      
0     00082ddb  _UARTRxErrorClear                                         
0     00082dd5  _UARTRxErrorGet                                           
0     00082c36  _UARTSpaceAvail                                           
0     0008306d  _UARTStdioConfig                                          
0     00082ccd  _UARTTXIntRegister                                        
0     00082cfb  _UARTTXIntUnregister                                      
0     00082c06  _UARTTxIntModeGet                                         
0     00082bf6  _UARTTxIntModeSet                                         
0     0008310f  _UARTgetc                                                 
0     000830c0  _UARTgets                                                 
0     00081ad1  _UARTgetsNonblocking                                      
0     000832c9  _UARTprintf                                               
0     00082bd3  _UARTsetLoopBack                                          
0     00083115  _UARTvprintf                                              
0     0008309f  _UARTwrite                                                
1     0000ee24  _UT_PRD                                                   
1     00006200  _UppRegs                                                  
1     00007000  _WdRegs                                                   
0     000845c6  _XINT1_Isr                                                
0     000845d6  _XINT2_Isr                                                
0     000845e6  _XINT3_Isr                                                
1     00007920  _XbarRegs                                                 
1     00007070  _XintRegs                                                 
1     00008040  __CIOBUF_                                                 
1     00000322  __STACK_END                                               
abs   00000200  __STACK_SIZE                                              
0     00087d8c  __TI_table_binit                                          
0     00000084  ___ASM__                                                  
0     00000000  ___ISA__                                                  
0     00000037  ___PLAT__                                                 
0     00000013  ___TARG__                                                 
1     00011590  ___TI_cleanup_ptr                                         
1     00011592  ___TI_dtors_ptr                                           
1     0001158e  ___TI_enable_exit_profile_output                          
abs   ffffffff  ___TI_pprof_out_hndl                                      
0     00080b74  ___TI_printfi                                             
abs   ffffffff  ___TI_prof_data_size                                      
abs   ffffffff  ___TI_prof_data_start                                     
0     00085bb8  ___TI_readmsg                                             
0     00085b60  ___TI_writemsg                                            
0     0000005d  ___TRDR__                                                 
0     00087d8c  ___binit__                                                
abs   ffffffff  ___c_args__                                               
0     0008b674  ___cinit__                                                
abs   ffffffff  ___etext__                                                
abs   ffffffff  ___pinit__                                                
abs   ffffffff  ___text__                                                 
0     00087d2b  ___xdc__init                                              
1     00010284  ___xdc__init__addr                                        
0     0008766e  __args_main                                               
0     0008ab57  __ctypes_                                                 
1     00011598  __lock                                                    
0     00087bf7  __nop                                                     
0     00087bf3  __register_lock                                           
0     00087bef  __register_unlock                                         
1     00000122  __stack                                                   
1     0001159a  __unlock                                                  
0     00087138  _abort                                                    
0     0008b0f2  _adcResultSem                                             
0     00086f4f  _atoi                                                     
0     00080c99  _buildCanMsg                                              
0     00080cca  _buildVarMsg                                              
0     0008648d  _c_int00                                                  
0     000869a6  _copy_in                                                  
0     000871fc  _copysignl                                                
0     0008755a  _ddcopy                                                   
0     00086175  _delay_loop                                               
1     0000ee44  _deltaMFlux                                               
1     0000ee54  _deltaRpm                                                 
1     0000ee46  _deltaTorque                                              
0     0008755a  _dpcopy                                                   
0     0008b0ba  _ePwm1Hwi                                                 
0     0008b0bc  _ePwm4Hwi                                                 
0     0008b0b6  _ePwmEvent                                                
0     0008533f  _emif1_read_ushort                                        
0     00085332  _emif1_write_ushort                                       
1     0000ee3f  _errno                                                    
0     0008713a  _exit                                                     
0     000865b0  _frexpl                                                   
1     000112ca  _g_bErrFlag                                               
1     000116c0  _g_psCmdTable                                             
1     000115c2  _g_sFresultStrings                                        
1     0001027e  _g_ui32Base                                               
1     000112c6  _g_ulRxMsgCount                                           
1     000112d8  _g_ulRxMsgCountPMSM                                       
1     00011340  _g_ulRxMsgCountPMSMB                                      
1     000112ce  _g_ulTxMsgCount                                           
1     00011328  _g_ulTxMsgCountPMSM                                       
1     000112e8  _g_ulTxMsgCountPMSMB                                      
0     00080d01  _get_idxTxA                                               
0     00080d46  _get_idxTxB                                               
1     00010273  _i                                                        
1     0000ee4e  _iRefC                                                    
1     0000ee52  _iRefTMax                                                 
1     0000ee48  _iddd                                                     
1     0000ee4a  _iqqq                                                     
0     0008522a  _ldexpl                                                   
0     00086fdc  _ltoa                                                     
1     0000ee1e  _m_hz                                                     
1     0000ee08  _m_rpm                                                    
1     0000ee1c  _m_sec                                                    
0     000861b3  _main                                                     
0     00087aba  _memccpy                                                  
0     000873a0  _memcpy                                                   
0     00087b33  _memset                                                   
1     0000ee0e  _motor4_rpm                                               
1     0000ee14  _motor_dir                                                
0     000861ab  _myOutputFunc                                             
0     00085328  _off_InvMagnCon                                           
0     0008531e  _on_InvMagnCon                                            
0     00080cf5  _parsingCanMsg                                            
0     0008755a  _pdcopy                                                   
0     0008755a  _ppcopy                                                   
1     0000ee18  _qep_tcnt                                                 
0     00085300  _read_FaultGroup1                                         
0     0008530a  _read_FaultGroup2                                         
0     00085314  _read_FaultGroup3                                         
0     000852e6  _read_Resolver1                                           
0     000852ee  _read_Resolver2                                           
1     0000ee29  _recv_data                                                
0     000852f6  _reset_Resolver1                                          
0     000852fb  _reset_Resolver2                                          
1     0000eec0  _rpmTable                                                 
1     0001130a  _sRXCANMessageA                                           
1     0001131e  _sRXCANMessageB                                           
1     000113c0  _sRXCANMessagePMSM                                        
1     00011540  _sRXCANMessagePMSMB                                       
1     00011300  _sTXCANMessageA                                           
1     00011314  _sTXCANMessageB                                           
1     000114c0  _sTXCANMessagePMSM                                        
1     00011400  _sTXCANMessagePMSMB                                       
0     0008522a  _scalbnl                                                  
0     00085dd9  _spiA_fifo_init                                           
0     00084fa6  _spiB_fifo_init                                           
0     000851ec  _spiC_fifo_init                                           
0     00086eec  _sprintf                                                  
0     00087b3f  _strchr                                                   
0     00087bb8  _strcmp                                                   
0     00087d0e  _strcpy                                                   
1     00011640  _string_display                                           
0     00087c39  _strlen                                                   
1     0000ee12  _t1_hz                                                    
1     0000ee0c  _t1_rpm                                                   
1     0000ee10  _t1_sec                                                   
1     0000ee5c  _tableMax                                                 
1     0000ee5a  _tableMin                                                 
1     0000ee58  _tableX1                                                  
1     0000ee60  _tableX2                                                  
1     0000ee5e  _tableY1                                                  
1     0000ee56  _tableY2                                                  
1     0000ee06  _threshold_m_value                                        
1     0000ee04  _threshold_t_value                                        
0     00080000  _ti_catalog_c2800_initF2837x_Boot_entry                   
0     00085ffc  _ti_catalog_c2800_initF2837x_Boot_init                    
0     0000b000  _ti_catalog_c2800_initF2837x_Boot_initFlash               
0     00087c01  _ti_catalog_c2800_initF2837x_Boot_initSharedRAMs          
0     00087c41  _ti_catalog_c2800_initF2837x_Boot_initStartup             
1     00010380  _ti_sysbios_BIOS_Module__state__V                         
0     00087c8e  _ti_sysbios_BIOS_RtsGateProxy_enter__E                    
0     00087c48  _ti_sysbios_BIOS_RtsGateProxy_leave__E                    
0     000876ff  _ti_sysbios_BIOS_atExitFunc__I                            
0     00087861  _ti_sysbios_BIOS_errorRaiseHook__I                        
0     00087ac7  _ti_sysbios_BIOS_exitFunc__I                              
0     0008b522  _ti_sysbios_BIOS_installedErrorHook__C                    
0     00083fff  _ti_sysbios_BIOS_linkedWithIncorrectBootLibrary__E        
0     00085b5f  _ti_sysbios_BIOS_nullFunc__I                              
0     00087a2b  _ti_sysbios_BIOS_registerRTSLock__I                       
0     00087a38  _ti_sysbios_BIOS_removeRTSLock__I                         
0     00081ff0  _ti_sysbios_BIOS_rtsLock__I                               
0     00086e22  _ti_sysbios_BIOS_rtsUnlock__I                             
0     00087c09  _ti_sysbios_BIOS_setThreadType__E                         
0     000877fa  _ti_sysbios_BIOS_startFunc__I                             
0     00087c94  _ti_sysbios_BIOS_start__E                                 
0     0008b524  _ti_sysbios_family_c28_Hwi_A_badIntNum__C                 
0     0008b526  _ti_sysbios_family_c28_Hwi_A_invalidArg__C                
0     0008b528  _ti_sysbios_family_c28_Hwi_E_unpluggedInterrupt__C        
0     0008b52a  _ti_sysbios_family_c28_Hwi_LD_end__C                      
0     0008b52c  _ti_sysbios_family_c28_Hwi_LM_begin__C                    
1     00010d00  _ti_sysbios_family_c28_Hwi_Module_State_0_dispatchTable__A
0     0008b52e  _ti_sysbios_family_c28_Hwi_Module__diagsEnabled__C        
0     0008b530  _ti_sysbios_family_c28_Hwi_Module__diagsIncluded__C       
0     0008b532  _ti_sysbios_family_c28_Hwi_Module__diagsMask__C           
0     0008a5c5  _ti_sysbios_family_c28_Hwi_Module__id__C                  
0     0008ad0b  _ti_sysbios_family_c28_Hwi_Module__loggerDefined__C       
0     0008b534  _ti_sysbios_family_c28_Hwi_Module__loggerFxn1__C          
0     0008b536  _ti_sysbios_family_c28_Hwi_Module__loggerFxn8__C          
0     0008b538  _ti_sysbios_family_c28_Hwi_Module__loggerObj__C           
1     000102c4  _ti_sysbios_family_c28_Hwi_Module__root__V                
0     00087b4b  _ti_sysbios_family_c28_Hwi_Module__startupDone__F         
0     00087d2e  _ti_sysbios_family_c28_Hwi_Module__startupDone__S         
1     00010318  _ti_sysbios_family_c28_Hwi_Module__state__V               
0     00086919  _ti_sysbios_family_c28_Hwi_Module_startup__E              
0     0008adab  _ti_sysbios_family_c28_Hwi_NUM_INTERRUPTS_ALL__C          
0     0008aebd  _ti_sysbios_family_c28_Hwi_Object__count__C               
0     00087574  _ti_sysbios_family_c28_Hwi_Object__get__S                 
0     0008b53a  _ti_sysbios_family_c28_Hwi_Object__table__C               
1     00010640  _ti_sysbios_family_c28_Hwi_Object__table__V               
0     000849ff  _ti_sysbios_family_c28_Hwi_clearInterrupt__E              
0     000878ad  _ti_sysbios_family_c28_Hwi_disableIER__E                  
0     00085e97  _ti_sysbios_family_c28_Hwi_disableInterrupt__E            
0     00085f18  _ti_sysbios_family_c28_Hwi_disablePIEIER__E               
0     00087a45  _ti_sysbios_family_c28_Hwi_dispatchC__I                   
0     0008566d  _ti_sysbios_family_c28_Hwi_dispatchCore__I                
0     000859f8  _ti_sysbios_family_c28_Hwi_dispatchPie                    
0     0008599b  _ti_sysbios_family_c28_Hwi_dispatchTable                  
0     0008795c  _ti_sysbios_family_c28_Hwi_enableIER__E                   
0     00085bf4  _ti_sysbios_family_c28_Hwi_enableInterrupt__E             
0     00086000  _ti_sysbios_family_c28_Hwi_enablePIEIER__E                
0     00087037  _ti_sysbios_family_c28_Hwi_getStackInfo__E                
0     00087d6e  _ti_sysbios_family_c28_Hwi_interruptReturn__I             
0     00087a52  _ti_sysbios_family_c28_Hwi_restoreIER__E                  
0     00087d13  _ti_sysbios_family_c28_Hwi_startup__E                     
0     00087485  _ti_sysbios_family_c28_Hwi_switchAndDispatch__I           
0     00087cfa  _ti_sysbios_family_c28_Hwi_switchFromBootStack__E         
0     00086a72  _ti_sysbios_family_c28_Hwi_unPluggedInterrupt__I          
0     0008a80e  _ti_sysbios_family_c28_Hwi_vectors                        
0     00087c9a  _ti_sysbios_family_c28_IntrinsicsSupport_maxbit__E        
0     0008b53c  _ti_sysbios_family_c28_TaskSupport_E_invalidStack__C      
0     0008af29  _ti_sysbios_family_c28_TaskSupport_Module__id__C          
0     00087d64  _ti_sysbios_family_c28_TaskSupport_Module__startupDone__S 
0     000871d7  _ti_sysbios_family_c28_TaskSupport_buildTaskStack         
0     00087bc2  _ti_sysbios_family_c28_TaskSupport_checkStack__E          
0     00087bcb  _ti_sysbios_family_c28_TaskSupport_glue                   
0     00086c2d  _ti_sysbios_family_c28_TaskSupport_start__E               
0     000873be  _ti_sysbios_family_c28_TaskSupport_swap__E                
0     0008b53e  _ti_sysbios_family_c28_Timer_Module__diagsEnabled__C      
0     0008b540  _ti_sysbios_family_c28_Timer_Module__diagsIncluded__C     
0     0008b542  _ti_sysbios_family_c28_Timer_Module__diagsMask__C         
0     0008af91  _ti_sysbios_family_c28_Timer_Module__id__C                
1     000102c8  _ti_sysbios_family_c28_Timer_Module__root__V              
0     00087b56  _ti_sysbios_family_c28_Timer_Module__startupDone__F       
0     00087d31  _ti_sysbios_family_c28_Timer_Module__startupDone__S       
1     000102e0  _ti_sysbios_family_c28_Timer_Module__state__V             
0     000877ce  _ti_sysbios_family_c28_Timer_Module_startup__E            
1     00010480  _ti_sysbios_family_c28_Timer_Object__table__V             
0     00087874  _ti_sysbios_family_c28_Timer_checkOverflow__I             
0     00086f1e  _ti_sysbios_family_c28_Timer_getFreq__E                   
0     00087d66  _ti_sysbios_family_c28_Timer_getMaxTicks__E               
0     000869ec  _ti_sysbios_family_c28_Timer_postInit__I                  
0     00086661  _ti_sysbios_family_c28_Timer_setPeriodMicroSecs__E        
0     000872c8  _ti_sysbios_family_c28_Timer_setPrescale__E               
0     00087063  _ti_sysbios_family_c28_Timer_start__E                     
0     0008b21b  _ti_sysbios_family_c28_Timer_startupNeeded__C             
0     00087716  _ti_sysbios_family_c28_Timer_startup__E                   
0     00085f96  _ti_sysbios_family_c28_Timer_stopAndClear__I              
0     0008796c  _ti_sysbios_family_c28_Timer_stop__E                      
0     000879d7  _ti_sysbios_family_c28_f2837x_TimestampProvider_get64__E  
0     00087687  _ti_sysbios_family_xxx_Hwi_switchAndRunFunc               
0     00087907  _ti_sysbios_gates_GateHwi_Handle__label__S                
0     00087d6f  _ti_sysbios_gates_GateHwi_Instance_init__E                
0     0008b3de  _ti_sysbios_gates_GateHwi_Module__FXNS__C                 
1     000102b2  _ti_sysbios_gates_GateHwi_Module__root__V                 
0     0008b438  _ti_sysbios_gates_GateHwi_Object__DESC__C                 
0     0008b4b4  _ti_sysbios_gates_GateHwi_Object__PARAMS__C               
0     000872e8  _ti_sysbios_gates_GateHwi_Object__create__S               
0     000878bf  _ti_sysbios_gates_GateHwi_Object__delete__S               
1     00010288  _ti_sysbios_gates_GateHwi_Object__table__V                
0     00087cff  _ti_sysbios_gates_GateHwi_enter__E                        
0     00087d34  _ti_sysbios_gates_GateHwi_leave__E                        
0     00087d68  _ti_sysbios_gates_GateHwi_query__E                        
0     0008b544  _ti_sysbios_gates_GateMutex_A_badContext__C               
0     00087918  _ti_sysbios_gates_GateMutex_Handle__label__S              
0     0008b546  _ti_sysbios_gates_GateMutex_Instance_State_sem__O         
0     00087c11  _ti_sysbios_gates_GateMutex_Instance_finalize__E          
0     0008798c  _ti_sysbios_gates_GateMutex_Instance_init__E              
0     0008b3f0  _ti_sysbios_gates_GateMutex_Module__FXNS__C               
0     0008b548  _ti_sysbios_gates_GateMutex_Module__diagsEnabled__C       
0     0008b54a  _ti_sysbios_gates_GateMutex_Module__diagsIncluded__C      
0     0008b54c  _ti_sysbios_gates_GateMutex_Module__diagsMask__C          
0     0008b263  _ti_sysbios_gates_GateMutex_Module__id__C                 
1     000102c0  _ti_sysbios_gates_GateMutex_Module__root__V               
0     0008b448  _ti_sysbios_gates_GateMutex_Object__DESC__C               
0     0008b4c0  _ti_sysbios_gates_GateMutex_Object__PARAMS__C             
0     00087307  _ti_sysbios_gates_GateMutex_Object__create__S             
0     00087887  _ti_sysbios_gates_GateMutex_Object__delete__S             
1     000103c0  _ti_sysbios_gates_GateMutex_Object__table__V              
0     00086342  _ti_sysbios_gates_GateMutex_enter__E                      
0     00087ad3  _ti_sysbios_gates_GateMutex_leave__E                      
0     00087d6a  _ti_sysbios_gates_GateMutex_query__E                      
0     0008b54e  _ti_sysbios_hal_Hwi_E_stackOverflow__C                    
0     00087d37  _ti_sysbios_hal_Hwi_HwiProxy_Module__startupDone__S       
0     00087c4f  _ti_sysbios_hal_Hwi_HwiProxy_getStackInfo__E              
0     00087d3a  _ti_sysbios_hal_Hwi_HwiProxy_startup__E                   
0     00087d3d  _ti_sysbios_hal_Hwi_HwiProxy_switchFromBootStack__E       
0     0008b2a7  _ti_sysbios_hal_Hwi_Module__id__C                         
1     00010296  _ti_sysbios_hal_Hwi_Module__root__V                       
0     00087bd4  _ti_sysbios_hal_Hwi_Module_startup__E                     
0     00087415  _ti_sysbios_hal_Hwi_checkStack                            
0     000874a0  _ti_sysbios_hal_Hwi_initStack                             
0     00087d40  _ti_sysbios_hal_Hwi_startup__E                            
1     000102d8  _ti_sysbios_hal_Timer_Module__root__V                     
0     00087bdd  _ti_sysbios_hal_Timer_Module_startup__E                   
0     00087d43  _ti_sysbios_hal_Timer_TimerProxy_Module__startupDone__S   
0     0008b550  _ti_sysbios_heaps_HeapMem_A_align__C                      
0     0008b552  _ti_sysbios_heaps_HeapMem_A_heapSize__C                   
0     0008b554  _ti_sysbios_heaps_HeapMem_A_invalidFree__C                
0     0008b556  _ti_sysbios_heaps_HeapMem_A_zeroBlock__C                  
0     0008b558  _ti_sysbios_heaps_HeapMem_E_memory__C                     
0     00087929  _ti_sysbios_heaps_HeapMem_Handle__label__S                
1     0000de00  _ti_sysbios_heaps_HeapMem_Instance_State_0_buf__A         
0     00084831  _ti_sysbios_heaps_HeapMem_Instance_init__E                
0     00087ca0  _ti_sysbios_heaps_HeapMem_Module_GateProxy_enter__E       
0     00087c56  _ti_sysbios_heaps_HeapMem_Module_GateProxy_leave__E       
0     00087ca6  _ti_sysbios_heaps_HeapMem_Module_GateProxy_query__E       
0     0008b3ca  _ti_sysbios_heaps_HeapMem_Module__FXNS__C                 
0     0008b55a  _ti_sysbios_heaps_HeapMem_Module__diagsEnabled__C         
0     0008b55c  _ti_sysbios_heaps_HeapMem_Module__diagsIncluded__C        
0     0008b55e  _ti_sysbios_heaps_HeapMem_Module__diagsMask__C            
0     0008b560  _ti_sysbios_heaps_HeapMem_Module__gateObj__C              
0     0008b437  _ti_sysbios_heaps_HeapMem_Module__id__C                   
1     000102dc  _ti_sysbios_heaps_HeapMem_Module__root__V                 
0     0008b458  _ti_sysbios_heaps_HeapMem_Object__DESC__C                 
0     0008b402  _ti_sysbios_heaps_HeapMem_Object__PARAMS__C               
0     0008b503  _ti_sysbios_heaps_HeapMem_Object__count__C                
0     00087326  _ti_sysbios_heaps_HeapMem_Object__create__S               
0     000878d1  _ti_sysbios_heaps_HeapMem_Object__delete__S               
0     0008772d  _ti_sysbios_heaps_HeapMem_Object__get__S                  
0     0008b562  _ti_sysbios_heaps_HeapMem_Object__table__C                
1     0001030c  _ti_sysbios_heaps_HeapMem_Object__table__V                
0     00081e6f  _ti_sysbios_heaps_HeapMem_allocUnprotected__E             
0     000867f1  _ti_sysbios_heaps_HeapMem_alloc__E                        
0     00084000  _ti_sysbios_heaps_HeapMem_freeUnprotected__E              
0     00087189  _ti_sysbios_heaps_HeapMem_free__E                         
0     0008700a  _ti_sysbios_heaps_HeapMem_getStats__E                     
0     000871b0  _ti_sysbios_heaps_HeapMem_init__I                         
0     00087d17  _ti_sysbios_heaps_HeapMem_isBlocking__E                   
0     0008b564  _ti_sysbios_heaps_HeapMem_reqAlign__C                     
0     0008b566  _ti_sysbios_knl_Clock_LM_begin__C                         
0     0008b568  _ti_sysbios_knl_Clock_LM_tick__C                          
0     0008b56a  _ti_sysbios_knl_Clock_LW_delayed__C                       
0     0008b56c  _ti_sysbios_knl_Clock_Module_State_clockQ__O              
0     0008b56e  _ti_sysbios_knl_Clock_Module__diagsEnabled__C             
0     0008b570  _ti_sysbios_knl_Clock_Module__diagsIncluded__C            
0     0008b572  _ti_sysbios_knl_Clock_Module__diagsMask__C                
0     0008b515  _ti_sysbios_knl_Clock_Module__id__C                       
0     0008b652  _ti_sysbios_knl_Clock_Module__loggerDefined__C            
0     0008b574  _ti_sysbios_knl_Clock_Module__loggerFxn1__C               
0     0008b576  _ti_sysbios_knl_Clock_Module__loggerFxn2__C               
0     0008b578  _ti_sysbios_knl_Clock_Module__loggerObj__C                
1     000102a2  _ti_sysbios_knl_Clock_Module__root__V                     
1     000103a6  _ti_sysbios_knl_Clock_Module__state__V                    
0     000878e3  _ti_sysbios_knl_Clock_Module_startup__E                   
0     00087d46  _ti_sysbios_knl_Clock_TimerProxy_Module__startupDone__S   
0     00087cac  _ti_sysbios_knl_Clock_TimerProxy_getMaxTicks__E           
0     0008750c  _ti_sysbios_knl_Clock_addI__E                             
0     00087744  _ti_sysbios_knl_Clock_doTick__I                           
0     00086d81  _ti_sysbios_knl_Clock_logTick__E                          
0     0008539e  _ti_sysbios_knl_Clock_workFunc__E                         
0     0008b57a  _ti_sysbios_knl_Event_A_badContext__C                     
0     0008b57c  _ti_sysbios_knl_Event_A_eventInUse__C                     
0     0008b57e  _ti_sysbios_knl_Event_A_nullEventId__C                    
0     0008b580  _ti_sysbios_knl_Event_A_nullEventMasks__C                 
0     0008b582  _ti_sysbios_knl_Event_A_pendTaskDisabled__C               
0     0008b584  _ti_sysbios_knl_Event_Instance_State_pendQ__O             
0     0008b586  _ti_sysbios_knl_Event_LM_pend__C                          
0     0008b588  _ti_sysbios_knl_Event_LM_post__C                          
0     0008b58a  _ti_sysbios_knl_Event_Module__diagsEnabled__C             
0     0008b58c  _ti_sysbios_knl_Event_Module__diagsIncluded__C            
0     0008b58e  _ti_sysbios_knl_Event_Module__diagsMask__C                
0     0008b653  _ti_sysbios_knl_Event_Module__id__C                       
0     0008b654  _ti_sysbios_knl_Event_Module__loggerDefined__C            
0     0008b590  _ti_sysbios_knl_Event_Module__loggerFxn4__C               
0     0008b592  _ti_sysbios_knl_Event_Module__loggerFxn8__C               
0     0008b594  _ti_sysbios_knl_Event_Module__loggerObj__C                
1     00010292  _ti_sysbios_knl_Event_Module__root__V                     
1     00010500  _ti_sysbios_knl_Event_Object__table__V                    
0     0008789a  _ti_sysbios_knl_Event_checkEvents__I                      
0     0008758d  _ti_sysbios_knl_Event_pendTimeout__I                      
0     000839ba  _ti_sysbios_knl_Event_pend__E                             
0     00084fe2  _ti_sysbios_knl_Event_post__E                             
0     00087c5d  _ti_sysbios_knl_Event_sync__E                             
0     0008b596  _ti_sysbios_knl_Idle_funcList__A                          
0     0008b516  _ti_sysbios_knl_Idle_funcList__C                          
0     00087d49  _ti_sysbios_knl_Idle_loop__E                              
0     00087839  _ti_sysbios_knl_Idle_run__E                               
1     00010580  _ti_sysbios_knl_Mailbox_Instance_State_0_allocBuf__A      
1     00010540  _ti_sysbios_knl_Mailbox_Instance_State_1_allocBuf__A      
1     00010400  _ti_sysbios_knl_Mailbox_Instance_State_2_allocBuf__A      
1     00010364  _ti_sysbios_knl_Mailbox_Instance_State_3_allocBuf__A      
1     00010328  _ti_sysbios_knl_Mailbox_Instance_State_4_allocBuf__A      
1     000104c0  _ti_sysbios_knl_Mailbox_Instance_State_5_allocBuf__A      
1     00010440  _ti_sysbios_knl_Mailbox_Instance_State_6_allocBuf__A      
1     00010880  _ti_sysbios_knl_Mailbox_Instance_State_7_allocBuf__A      
1     00010740  _ti_sysbios_knl_Mailbox_Instance_State_8_allocBuf__A      
1     00010340  _ti_sysbios_knl_Mailbox_Instance_State_9_allocBuf__A      
0     0008b598  _ti_sysbios_knl_Mailbox_Instance_State_dataQue__O         
0     0008b59a  _ti_sysbios_knl_Mailbox_Instance_State_dataSem__O         
0     0008b59c  _ti_sysbios_knl_Mailbox_Instance_State_freeQue__O         
0     0008b59e  _ti_sysbios_knl_Mailbox_Instance_State_freeSem__O         
1     000102ae  _ti_sysbios_knl_Mailbox_Module__root__V                   
0     0008708f  _ti_sysbios_knl_Mailbox_Module_startup__E                 
0     0008b655  _ti_sysbios_knl_Mailbox_Object__count__C                  
0     0008775b  _ti_sysbios_knl_Mailbox_Object__get__S                    
0     0008b5a0  _ti_sysbios_knl_Mailbox_Object__table__C                  
1     00010b40  _ti_sysbios_knl_Mailbox_Object__table__V                  
0     0008b656  _ti_sysbios_knl_Mailbox_maxTypeAlign__C                   
0     00086b75  _ti_sysbios_knl_Mailbox_pend__E                           
0     000875a6  _ti_sysbios_knl_Mailbox_postInit__I                       
0     00086887  _ti_sysbios_knl_Mailbox_post__E                           
0     00087d4c  _ti_sysbios_knl_Queue_Instance_init__E                    
1     0001028e  _ti_sysbios_knl_Queue_Module__root__V                     
0     0008b468  _ti_sysbios_knl_Queue_Object__DESC__C                     
0     0008b4cc  _ti_sysbios_knl_Queue_Object__PARAMS__C                   
0     0008b657  _ti_sysbios_knl_Queue_Object__count__C                    
0     000879e5  _ti_sysbios_knl_Queue_Object__destruct__S                 
0     000875bf  _ti_sysbios_knl_Queue_Object__get__S                      
0     0008b5a2  _ti_sysbios_knl_Queue_Object__table__C                    
0     000875d8  _ti_sysbios_knl_Queue_construct                           
0     00087cb2  _ti_sysbios_knl_Queue_destruct                            
0     00087c64  _ti_sysbios_knl_Queue_empty__E                            
0     00087adf  _ti_sysbios_knl_Queue_get__E                              
0     00087aeb  _ti_sysbios_knl_Queue_put__E                              
0     0008b5a4  _ti_sysbios_knl_Semaphore_A_badContext__C                 
0     0008b5a6  _ti_sysbios_knl_Semaphore_A_overflow__C                   
0     0008b5a8  _ti_sysbios_knl_Semaphore_A_pendTaskDisabled__C           
0     0008b5aa  _ti_sysbios_knl_Semaphore_Instance_State_pendQ__O         
0     0008784d  _ti_sysbios_knl_Semaphore_Instance_finalize__E            
0     00086ca1  _ti_sysbios_knl_Semaphore_Instance_init__E                
0     0008b5ac  _ti_sysbios_knl_Semaphore_LM_pend__C                      
0     0008b5ae  _ti_sysbios_knl_Semaphore_LM_post__C                      
0     0008b5b0  _ti_sysbios_knl_Semaphore_Module__diagsEnabled__C         
0     0008b5b2  _ti_sysbios_knl_Semaphore_Module__diagsIncluded__C        
0     0008b5b4  _ti_sysbios_knl_Semaphore_Module__diagsMask__C            
0     0008b658  _ti_sysbios_knl_Semaphore_Module__id__C                   
0     0008b659  _ti_sysbios_knl_Semaphore_Module__loggerDefined__C        
0     0008b5b6  _ti_sysbios_knl_Semaphore_Module__loggerFxn2__C           
0     0008b5b8  _ti_sysbios_knl_Semaphore_Module__loggerFxn4__C           
0     0008b5ba  _ti_sysbios_knl_Semaphore_Module__loggerObj__C            
1     000102aa  _ti_sysbios_knl_Semaphore_Module__root__V                 
0     0008b478  _ti_sysbios_knl_Semaphore_Object__DESC__C                 
0     0008b488  _ti_sysbios_knl_Semaphore_Object__PARAMS__C               
0     0008799b  _ti_sysbios_knl_Semaphore_Object__destruct__S             
1     000102f0  _ti_sysbios_knl_Semaphore_Object__table__V                
0     000874bb  _ti_sysbios_knl_Semaphore_construct                       
0     00087cb8  _ti_sysbios_knl_Semaphore_destruct                        
0     0008b5bc  _ti_sysbios_knl_Semaphore_eventPost__C                    
0     0008b5be  _ti_sysbios_knl_Semaphore_eventSync__C                    
0     000875f1  _ti_sysbios_knl_Semaphore_pendTimeout__I                  
0     00083bec  _ti_sysbios_knl_Semaphore_pend__E                         
0     000850ac  _ti_sysbios_knl_Semaphore_post__E                         
0     0008b5c0  _ti_sysbios_knl_Swi_LD_end__C                             
0     0008b5c2  _ti_sysbios_knl_Swi_LM_begin__C                           
0     0008b5c4  _ti_sysbios_knl_Swi_LM_post__C                            
1     000105c0  _ti_sysbios_knl_Swi_Module_State_0_readyQ__A              
0     0008b5c6  _ti_sysbios_knl_Swi_Module__diagsEnabled__C               
0     0008b5c8  _ti_sysbios_knl_Swi_Module__diagsIncluded__C              
0     0008b5ca  _ti_sysbios_knl_Swi_Module__diagsMask__C                  
0     0008b65a  _ti_sysbios_knl_Swi_Module__id__C                         
0     0008b65b  _ti_sysbios_knl_Swi_Module__loggerDefined__C              
0     0008b5cc  _ti_sysbios_knl_Swi_Module__loggerFxn1__C                 
0     0008b5ce  _ti_sysbios_knl_Swi_Module__loggerFxn4__C                 
0     0008b5d0  _ti_sysbios_knl_Swi_Module__loggerObj__C                  
1     0001029e  _ti_sysbios_knl_Swi_Module__root__V                       
1     00010300  _ti_sysbios_knl_Swi_Module__state__V                      
0     0008780f  _ti_sysbios_knl_Swi_Module_startup__E                     
0     0008b65c  _ti_sysbios_knl_Swi_Object__count__C                      
0     00087772  _ti_sysbios_knl_Swi_Object__get__S                        
0     0008b5d2  _ti_sysbios_knl_Swi_Object__table__C                      
1     00010392  _ti_sysbios_knl_Swi_Object__table__V                      
0     00087cbe  _ti_sysbios_knl_Swi_disable__E                            
0     000864f0  _ti_sysbios_knl_Swi_post__E                               
0     00086bb3  _ti_sysbios_knl_Swi_restoreHwi__E                         
0     0008760a  _ti_sysbios_knl_Swi_restore__E                            
0     00086f80  _ti_sysbios_knl_Swi_runLoop__I                            
0     000855be  _ti_sysbios_knl_Swi_run__I                                
0     00086fae  _ti_sysbios_knl_Swi_schedule__I                           
0     00087d1b  _ti_sysbios_knl_Swi_startup__E                            
0     0008b5d4  _ti_sysbios_knl_Task_A_badTimeout__C                      
0     0008b5d6  _ti_sysbios_knl_Task_A_sleepTaskDisabled__C               
0     0008b5d8  _ti_sysbios_knl_Task_E_spOutOfBounds__C                   
0     0008b5da  _ti_sysbios_knl_Task_E_stackOverflow__C                   
1     0000d000  _ti_sysbios_knl_Task_Instance_State_0_stack__A            
1     0000c200  _ti_sysbios_knl_Task_Instance_State_10_stack__A           
1     0000c400  _ti_sysbios_knl_Task_Instance_State_1_stack__A            
1     0000c800  _ti_sysbios_knl_Task_Instance_State_2_stack__A            
1     0000c600  _ti_sysbios_knl_Task_Instance_State_3_stack__A            
1     0000ca00  _ti_sysbios_knl_Task_Instance_State_4_stack__A            
1     0000c100  _ti_sysbios_knl_Task_Instance_State_5_stack__A            
1     0000c000  _ti_sysbios_knl_Task_Instance_State_6_stack__A            
1     0000d600  _ti_sysbios_knl_Task_Instance_State_7_stack__A            
1     0000c300  _ti_sysbios_knl_Task_Instance_State_8_stack__A            
1     0000cc00  _ti_sysbios_knl_Task_Instance_State_9_stack__A            
0     0008b5dc  _ti_sysbios_knl_Task_LD_block__C                          
0     0008b5de  _ti_sysbios_knl_Task_LD_exit__C                           
0     0008b5e0  _ti_sysbios_knl_Task_LD_ready__C                          
0     0008b5e2  _ti_sysbios_knl_Task_LM_sleep__C                          
0     0008b5e4  _ti_sysbios_knl_Task_LM_switch__C                         
1     00010282  _ti_sysbios_knl_Task_Module_State_0_idleTask__A           
1     00010600  _ti_sysbios_knl_Task_Module_State_0_readyQ__A             
0     0008b5e6  _ti_sysbios_knl_Task_Module_State_inactiveQ__O            
0     0008b5e8  _ti_sysbios_knl_Task_Module__diagsEnabled__C              
0     0008b5ea  _ti_sysbios_knl_Task_Module__diagsIncluded__C             
0     0008b5ec  _ti_sysbios_knl_Task_Module__diagsMask__C                 
0     0008b65d  _ti_sysbios_knl_Task_Module__id__C                        
0     0008b65e  _ti_sysbios_knl_Task_Module__loggerDefined__C             
0     0008b5ee  _ti_sysbios_knl_Task_Module__loggerFxn2__C                
0     0008b5f0  _ti_sysbios_knl_Task_Module__loggerFxn4__C                
0     0008b5f2  _ti_sysbios_knl_Task_Module__loggerObj__C                 
1     000102ba  _ti_sysbios_knl_Task_Module__root__V                      
1     000103dc  _ti_sysbios_knl_Task_Module__state__V                     
0     00086e56  _ti_sysbios_knl_Task_Module_startup__E                    
0     0008b65f  _ti_sysbios_knl_Task_Object__count__C                     
0     00087789  _ti_sysbios_knl_Task_Object__get__S                       
0     0008b5f4  _ti_sysbios_knl_Task_Object__table__C                     
1     000109c0  _ti_sysbios_knl_Task_Object__table__V                     
0     00087d4f  _ti_sysbios_knl_Task_SupportProxy_Module__startupDone__S  
0     00087c6b  _ti_sysbios_knl_Task_SupportProxy_checkStack__E           
0     00087a5f  _ti_sysbios_knl_Task_SupportProxy_start__E                
0     00087c72  _ti_sysbios_knl_Task_SupportProxy_swap__E                 
0     0008b5f6  _ti_sysbios_knl_Task_allBlockedFunc__C                    
0     00087265  _ti_sysbios_knl_Task_allBlockedFunction__I                
0     00086550  _ti_sysbios_knl_Task_blockI__E                            
0     0008625e  _ti_sysbios_knl_Task_checkStacks__E                       
0     00087cc4  _ti_sysbios_knl_Task_disable__E                           
0     00087af7  _ti_sysbios_knl_Task_enabled__E                           
0     00087a6c  _ti_sysbios_knl_Task_enter__I                             
0     0008660a  _ti_sysbios_knl_Task_exit__E                              
0     0008b660  _ti_sysbios_knl_Task_numConstructedTasks__C               
0     0008683c  _ti_sysbios_knl_Task_postInit__I                          
0     000874d6  _ti_sysbios_knl_Task_processVitalTaskFlag__I              
0     0008797c  _ti_sysbios_knl_Task_restoreHwi__E                        
0     000877e4  _ti_sysbios_knl_Task_restore__E                           
0     000863b2  _ti_sysbios_knl_Task_schedule__I                          
0     00087a79  _ti_sysbios_knl_Task_sleepTimeout__I                      
0     000842e6  _ti_sysbios_knl_Task_sleep__E                             
0     000862d1  _ti_sysbios_knl_Task_startCore__E                         
0     00087d52  _ti_sysbios_knl_Task_startup__E                           
0     000866b5  _ti_sysbios_knl_Task_unblockI__E                          
0     00087b61  _ti_sysbios_knl_Task_unblock__E                           
1     0000ee50  _torqCmd                                                  
1     0000ef00  _torqueTable                                              
1     000112c8  _u32CanAErrorStatus                                       
1     000112cc  _u32CntTXMsgData                                          
1     000112f0  _ucRXMsgDataA                                             
1     000112e0  _ucRXMsgDataB                                             
1     0001134e  _ucRXMsgDataPMSM                                          
1     00011440  _ucRXMsgDataPMSMB                                         
1     000112f8  _ucTXMsgDataA                                             
1     000112d0  _ucTXMsgDataB                                             
1     00011480  _ucTXMsgDataPMSM                                          
1     00011380  _ucTXMsgDataPMSMB                                         
0     00082260  _ulocaltime                                               
0     00082340  _umktime                                                  
0     000825d0  _urand                                                    
0     00082250  _usnprintf                                                
0     0008223f  _usprintf                                                 
0     000825c9  _usrand                                                   
0     0008258c  _ustrcasecmp                                              
0     000825c0  _ustrcmp                                                  
0     00082523  _ustrlen                                                  
0     0008254d  _ustrncasecmp                                             
0     00082595  _ustrncmp                                                 
0     00082000  _ustrncpy                                                 
0     00082533  _ustrstr                                                  
0     00082409  _ustrtof                                                  
0     0008237d  _ustrtoul                                                 
0     0008202d  _uvsnprintf                                               
0     0008b5fc  _xdc_runtime_Assert_E_assertFailed__C                     
0     00086e88  _xdc_runtime_Assert_raise__I                              
0     0008b5fe  _xdc_runtime_Core_A_initializedParams__C                  
0     0008b600  _xdc_runtime_Core_Module__diagsEnabled__C                 
0     0008b602  _xdc_runtime_Core_Module__diagsIncluded__C                
0     0008b604  _xdc_runtime_Core_Module__diagsMask__C                    
0     0008b661  _xdc_runtime_Core_Module__id__C                           
0     00087526  _xdc_runtime_Core_assignLabel__I                          
0     00086ab4  _xdc_runtime_Core_assignParams__I                         
0     000857c0  _xdc_runtime_Core_constructObject__I                      
0     00084d73  _xdc_runtime_Core_createObject__I                         
0     00086706  _xdc_runtime_Core_deleteObject__I                         
0     0008b606  _xdc_runtime_Error_E_memory__C                            
0     0008b608  _xdc_runtime_Error_Module__diagsEnabled__C                
0     0008b60a  _xdc_runtime_Error_Module__diagsIncluded__C               
0     0008b60c  _xdc_runtime_Error_Module__diagsMask__C                   
0     0008b662  _xdc_runtime_Error_Module__loggerDefined__C               
0     0008b60e  _xdc_runtime_Error_Module__loggerFxn8__C                  
0     0008b610  _xdc_runtime_Error_Module__loggerObj__C                   
1     00010280  _xdc_runtime_Error_Module__state__V                       
0     00087a86  _xdc_runtime_Error_check__E                               
0     00087d6c  _xdc_runtime_Error_getSite__E                             
0     00087c79  _xdc_runtime_Error_init__E                                
0     0008b663  _xdc_runtime_Error_maxDepth__C                            
0     0008571b  _xdc_runtime_Error_policyDefault__E                       
0     0008b612  _xdc_runtime_Error_policyFxn__C                           
0     0008b664  _xdc_runtime_Error_policy__C                              
0     00086db7  _xdc_runtime_Error_print__E                               
0     0008b614  _xdc_runtime_Error_raiseHook__C                           
0     0008793a  _xdc_runtime_Error_raiseX__E                              
0     00086a2f  _xdc_runtime_Error_setX__E                                
0     00087cca  _xdc_runtime_Gate_enterSystem__E                          
0     00087cd0  _xdc_runtime_Gate_leaveSystem__E                          
0     0008b616  _xdc_runtime_IFilterLogger_Interface__BASE__C             
0     0008b618  _xdc_runtime_IGateProvider_Interface__BASE__C             
0     0008b61a  _xdc_runtime_IHeap_Interface__BASE__C                     
0     0008b61c  _xdc_runtime_ILogger_Interface__BASE__C                   
0     0008b61e  _xdc_runtime_IModule_Interface__BASE__C                   
0     0008b620  _xdc_runtime_Log_L_error__C                               
0     0008b622  _xdc_runtime_LoggerBuf_E_badLevel__C                      
0     0008794b  _xdc_runtime_LoggerBuf_Handle__label__S                   
1     00010ec0  _xdc_runtime_LoggerBuf_Instance_State_0_entryArr__A       
0     00087b6c  _xdc_runtime_LoggerBuf_Instance_finalize__E               
0     00086eba  _xdc_runtime_LoggerBuf_Instance_init__E                   
0     00087cd6  _xdc_runtime_LoggerBuf_Module_GateProxy_enter__E          
0     00087c80  _xdc_runtime_LoggerBuf_Module_GateProxy_leave__E          
0     0008b31a  _xdc_runtime_LoggerBuf_Module__FXNS__C                    
0     0008b624  _xdc_runtime_LoggerBuf_Module__gateObj__C                 
0     0008b665  _xdc_runtime_LoggerBuf_Module__id__C                      
1     000102b6  _xdc_runtime_LoggerBuf_Module__root__V                    
1     0001028a  _xdc_runtime_LoggerBuf_Module__state__V                   
0     00087540  _xdc_runtime_LoggerBuf_Module_startup__E                  
0     0008b498  _xdc_runtime_LoggerBuf_Object__DESC__C                    
0     0008b414  _xdc_runtime_LoggerBuf_Object__PARAMS__C                  
0     0008b666  _xdc_runtime_LoggerBuf_Object__count__C                   
0     00086d13  _xdc_runtime_LoggerBuf_Object__create__S                  
0     000878f5  _xdc_runtime_LoggerBuf_Object__delete__S                  
0     000877a0  _xdc_runtime_LoggerBuf_Object__get__S                     
0     0008b626  _xdc_runtime_LoggerBuf_Object__table__C                   
1     00010352  _xdc_runtime_LoggerBuf_Object__table__V                   
0     00087cdc  _xdc_runtime_LoggerBuf_TimestampProxy_get64__E            
0     00087d1f  _xdc_runtime_LoggerBuf_disable__E                         
0     00087d09  _xdc_runtime_LoggerBuf_enable__E                          
0     0008b667  _xdc_runtime_LoggerBuf_filterByLevel__C                   
0     000873db  _xdc_runtime_LoggerBuf_filterOutEvent__I                  
0     00086bf1  _xdc_runtime_LoggerBuf_getFilterLevel__E                  
0     0008769f  _xdc_runtime_LoggerBuf_reset__E                           
0     00086b36  _xdc_runtime_LoggerBuf_setFilterLevel__E                  
0     0008b628  _xdc_runtime_LoggerBuf_statusLogger__C                    
0     00087b77  _xdc_runtime_LoggerBuf_write0__E                          
0     00087a93  _xdc_runtime_LoggerBuf_write1__E                          
0     000879aa  _xdc_runtime_LoggerBuf_write2__E                          
0     00085a36  _xdc_runtime_LoggerBuf_write4__E                          
0     00084adf  _xdc_runtime_LoggerBuf_write8__E                          
0     0008b62a  _xdc_runtime_Main_Module__diagsEnabled__C                 
0     0008b62c  _xdc_runtime_Main_Module__diagsIncluded__C                
0     0008b62e  _xdc_runtime_Main_Module__diagsMask__C                    
0     0008b668  _xdc_runtime_Main_Module__id__C                           
0     00087aa0  _xdc_runtime_Memory_HeapProxy_alloc__E                    
0     00087c21  _xdc_runtime_Memory_HeapProxy_free__E                     
0     0008b669  _xdc_runtime_Memory_Module__id__C                         
1     00010286  _xdc_runtime_Memory_Module__state__V                      
0     00086757  _xdc_runtime_Memory_alloc__E                              
0     00087c29  _xdc_runtime_Memory_calloc__E                             
0     0008b630  _xdc_runtime_Memory_defaultHeapInstance__C                
0     00087b03  _xdc_runtime_Memory_free__E                               
0     00087d23  _xdc_runtime_Memory_getMaxDefaultTypeAlign__E             
0     00087623  _xdc_runtime_Memory_valloc__E                             
1     0001029a  _xdc_runtime_Registry_Module__state__V                    
0     00087a01  _xdc_runtime_Registry_findById__E                         
1     000102d4  _xdc_runtime_Startup_Module__state__V                     
abs   00000001  _xdc_runtime_Startup__EXECFXN__C                          
abs   00000001  _xdc_runtime_Startup__RESETFXN__C                         
0     0008b632  _xdc_runtime_Startup_execImpl__C                          
0     00086ded  _xdc_runtime_Startup_exec__E                              
0     00087b82  _xdc_runtime_Startup_exec__I                              
0     0008b50a  _xdc_runtime_Startup_firstFxns__A                         
0     0008b51a  _xdc_runtime_Startup_firstFxns__C                         
0     0008b51e  _xdc_runtime_Startup_lastFxns__C                          
0     0008b66a  _xdc_runtime_Startup_maxPasses__C                         
0     00087d55  _xdc_runtime_Startup_reset__I                             
0     00087d27  _xdc_runtime_Startup_rtsDone__E                           
0     0008b4d8  _xdc_runtime_Startup_sfxnRts__A                           
0     0008b634  _xdc_runtime_Startup_sfxnRts__C                           
0     0008b3a0  _xdc_runtime_Startup_sfxnTab__A                           
0     0008b636  _xdc_runtime_Startup_sfxnTab__C                           
0     0008b638  _xdc_runtime_Startup_startModsFxn__C                      
0     0008607d  _xdc_runtime_Startup_startMods__I                         
1     000110c0  _xdc_runtime_SysMin_Module_State_0_outbuf__A              
1     000102cc  _xdc_runtime_SysMin_Module__state__V                      
0     00087a0f  _xdc_runtime_SysMin_Module_startup__E                     
0     000877b7  _xdc_runtime_SysMin_abort__E                              
0     0008b63a  _xdc_runtime_SysMin_bufSize__C                            
0     00087b8d  _xdc_runtime_SysMin_exit__E                               
0     0008b66b  _xdc_runtime_SysMin_flushAtExit__C                        
0     00087161  _xdc_runtime_SysMin_flush__E                              
0     0008b63c  _xdc_runtime_SysMin_outputFunc__C                         
0     000874f1  _xdc_runtime_SysMin_output__I                             
0     00087364  _xdc_runtime_SysMin_putch__E                              
0     00087c31  _xdc_runtime_SysMin_ready__E                              
0     00087ce2  _xdc_runtime_System_Module_GateProxy_enter__E             
0     00087c87  _xdc_runtime_System_Module_GateProxy_leave__E             
1     000102e8  _xdc_runtime_System_Module_State_0_atexitHandlers__A      
0     0008b63e  _xdc_runtime_System_Module__gateObj__C                    
1     000102d0  _xdc_runtime_System_Module__state__V                      
0     00087d58  _xdc_runtime_System_Module_startup__E                     
0     00087ce8  _xdc_runtime_System_SupportProxy_abort__E                 
0     00087cee  _xdc_runtime_System_SupportProxy_exit__E                  
0     00087cf4  _xdc_runtime_System_SupportProxy_putch__E                 
0     00087d5b  _xdc_runtime_System_SupportProxy_ready__E                 
0     0008b640  _xdc_runtime_System_abortFxn__C                           
0     00087d5e  _xdc_runtime_System_abortStd__E                           
0     00087aad  _xdc_runtime_System_abort__E                              
0     00087b0f  _xdc_runtime_System_aprintf__E                            
0     0008763c  _xdc_runtime_System_aprintf_va__F                         
0     00087286  _xdc_runtime_System_atexit__E                             
0     0008763c  _xdc_runtime_System_avprintf__E                           
0     000832d4  _xdc_runtime_System_doPrint__I                            
0     0008b642  _xdc_runtime_System_exitFxn__C                            
0     00087d61  _xdc_runtime_System_exitStd__E                            
0     00087b98  _xdc_runtime_System_exit__E                               
0     0008b644  _xdc_runtime_System_extendFxn__C                          
0     00086af6  _xdc_runtime_System_formatNum__I                          
0     0008b66c  _xdc_runtime_System_maxAtexitHandlers__C                  
0     0008441b  _xdc_runtime_System_printfExtend__I                       
0     00087b1b  _xdc_runtime_System_printf__E                             
0     000876b7  _xdc_runtime_System_printf_va__F                          
0     00087220  _xdc_runtime_System_processAtExit__E                      
0     00087655  _xdc_runtime_System_putchar__I                            
0     00087be6  _xdc_runtime_System_snprintf_va__F                        
0     000876b7  _xdc_runtime_System_vprintf__E                            
0     00087be6  _xdc_runtime_System_vsnprintf__E                          
1     000102a6  _xdc_runtime_Text_Module__state__V                        
0     0008b66d  _xdc_runtime_Text_charCnt__C                              
0     00088000  _xdc_runtime_Text_charTab__A                              
0     0008b646  _xdc_runtime_Text_charTab__C                              
0     00087824  _xdc_runtime_Text_cordText__E                             
0     0008b66e  _xdc_runtime_Text_isLoaded__C                             
0     0008b648  _xdc_runtime_Text_nameEmpty__C                            
0     0008b64a  _xdc_runtime_Text_nameStatic__C                           
0     0008b64c  _xdc_runtime_Text_nameUnknown__C                          
0     0008afec  _xdc_runtime_Text_nodeTab__A                              
0     0008b64e  _xdc_runtime_Text_nodeTab__C                              
0     000876cf  _xdc_runtime_Text_printVisFxn__I                          
0     000867a5  _xdc_runtime_Text_putLab__E                               
0     00086c67  _xdc_runtime_Text_putMod__E                               
0     000860fa  _xdc_runtime_Text_putSite__E                              
0     0008b66f  _xdc_runtime_Text_registryModsLastId__C                   
0     00087b27  _xdc_runtime_Text_ropeText__E                             
0     0008b670  _xdc_runtime_Text_unnamedModsLastId__C                    
0     00086cda  _xdc_runtime_Text_visitRope2__I                           
0     0008b650  _xdc_runtime_Text_visitRopeFxn__C                         
0     000879b9  _xdc_runtime_Text_visitRope__I                            
0     000870ba  _xdc_runtime_Text_xprintf__I                              
0     00087d8c  binit                                                     
0     0008b674  cinit                                                     
abs   ffffffff  etext                                                     
abs   ffffffff  pinit                                                     


GLOBAL SYMBOLS: SORTED BY Symbol Address 

page  address   name                                                      
----  -------   ----                                                      
0     00000000  ___ISA__                                                  
0     00000013  ___TARG__                                                 
0     00000037  ___PLAT__                                                 
0     0000005d  ___TRDR__                                                 
0     00000084  ___ASM__                                                  
0     00000ce0  _Cla1SoftIntRegs                                          
0     00000d00  _EmuKey                                                   
0     00000d00  _PieVectTable                                             
0     00000d01  _EmuBMode                                                 
0     00008000  _InitFlash                                                
0     00008000  _RamfuncsRunStart                                         
0     00008029  _FlashOff                                                 
0     00008037  _F28x_usDelay                                             
0     0000803b  _SysCtlDelay                                              
0     0000803f  _RamfuncsRunEnd                                           
0     0000b000  _ti_catalog_c2800_initF2837x_Boot_initFlash               
0     00080000  _ti_catalog_c2800_initF2837x_Boot_entry                   
0     00080080  _RamfuncsLoadStart                                        
0     000800bf  _RamfuncsLoadEnd                                          
0     00080b74  ___TI_printfi                                             
0     00080c99  _buildCanMsg                                              
0     00080cca  _buildVarMsg                                              
0     00080cf5  _parsingCanMsg                                            
0     00080d01  _get_idxTxA                                               
0     00080d46  _get_idxTxB                                               
0     00080d70  _CanMsg_prnt                                              
0     00080d9d  _CANAIntHandler                                           
0     00080da7  _CanA_TxRx_Task                                           
0     00080fc5  _CANBIntHandler                                           
0     00080fcf  _CanB_TxRx_Task                                           
0     000811ed  _InitCanA                                                 
0     00081236  _InitCanB                                                 
0     0008127f  _CanA_EableTxRx                                           
0     0008136e  _CanB_EableTxRx                                           
0     0008148f  _Cmd_IntTmr                                               
0     000814b5  _Cmd_Can                                                  
0     00081561  _Cmd_CanRpt                                               
0     00081582  _Cmd_CanDebug                                             
0     000815c0  _Cmd_EMIF1_WR                                             
0     000815fb  _Cmd_EMIF1_RD                                             
0     00081637  _Cmd_IntAdcDebug                                          
0     0008168b  _Cmd_IntAdcDisplay                                        
0     000816b2  _Cmd_ExtAdcDebug                                          
0     000816d9  _Cmd_ExtAdcDisplay                                        
0     00081700  _Cmd_readGPIO                                             
0     00081750  _Cmd_readGPIOAll                                          
0     000817a7  _Cmd_writeGPIO                                            
0     00081816  _Cmd_EMIF1_ContiRD                                        
0     00081836  _Cmd_ExtIntDebug                                          
0     0008185d  _Cmd_ExtIntEnable                                         
0     00081869  _Cmd_TempDebug                                            
0     00081890  _Cmd_TempDisplay                                          
0     000818b7  _Cmd_Dac                                                  
0     000818f1  _Cmd_epwm_Duty                                            
0     00081974  _Cmd_epwm_Carrier                                         
0     000819e1  _Cmd_epwm_Info                                            
0     00081a21  _Cmd_epwm_Debug                                           
0     00081a69  _Cmd_help                                                 
0     00081a9b  _Cmd_Task                                                 
0     00081ad1  _UARTgetsNonblocking                                      
0     00081b28  _InitSysCtrl                                              
0     00081b65  _InitPeripheralClocks                                     
0     00081be9  _DisablePeripheralClocks                                  
0     00081c01  _SeizeFlashPump                                           
0     00081c10  _ReleaseFlashPump                                         
0     00081c1a  _ServiceDog                                               
0     00081c28  _DisableDog                                               
0     00081c36  _InitSysPll                                               
0     00081cfc  _InitAuxPll                                               
0     00081dc4  _CsmUnlock                                                
0     00081de5  _SysIntOsc1Sel                                            
0     00081def  _SysIntOsc2Sel                                            
0     00081df9  _SysXtalOscSel                                            
0     00081e05  _AuxIntOsc2Sel                                            
0     00081e0f  _AuxXtalOscSel                                            
0     00081e1b  _AuxAuxClkSel                                             
0     00081e25  _IDLE                                                     
0     00081e2e  _STANDBY                                                  
0     00081e39  _HALT                                                     
0     00081e52  _HIB                                                      
0     00081e6f  _ti_sysbios_heaps_HeapMem_allocUnprotected__E             
0     00081ff0  _ti_sysbios_BIOS_rtsLock__I                               
0     00082000  _ustrncpy                                                 
0     0008202d  _uvsnprintf                                               
0     0008223f  _usprintf                                                 
0     00082250  _usnprintf                                                
0     00082260  _ulocaltime                                               
0     00082340  _umktime                                                  
0     0008237d  _ustrtoul                                                 
0     00082409  _ustrtof                                                  
0     00082523  _ustrlen                                                  
0     00082533  _ustrstr                                                  
0     0008254d  _ustrncasecmp                                             
0     0008258c  _ustrcasecmp                                              
0     00082595  _ustrncmp                                                 
0     000825c0  _ustrcmp                                                  
0     000825c9  _usrand                                                   
0     000825d0  _urand                                                    
0     0008264b  _CANInit                                                  
0     000826f8  _CANEnable                                                
0     00082701  _CANDisable                                               
0     00082709  _CANClkSourceSelect                                       
0     00082730  _CANBitTimingGet                                          
0     0008275b  _CANBitRateSet                                            
0     000827ca  _CANBitTimingSet                                          
0     00082815  _CANIntRegister                                           
0     00082825  _CANIntUnregister                                         
0     00082832  _CANIntEnable                                             
0     00082840  _CANIntDisable                                            
0     00082850  _CANIntStatus                                             
0     0008286a  _CANIntClear                                              
0     00082893  _CANRetrySet                                              
0     000828a4  _CANRetryGet                                              
0     000828ae  _CANStatusGet                                             
0     000828d6  _CANErrCntrGet                                            
0     000828f1  _CANMessageSet                                            
0     000829e3  _CANMessageGet                                            
0     00082ab9  _CANMessageClear                                          
0     00082adf  _CANGlobalIntEnable                                       
0     00082ae8  _CANGlobalIntDisable                                      
0     00082af2  _CANGlobalIntClear                                        
0     00082afb  _CANGlobalIntstatusGet                                    
0     00082b08  _UARTParityModeSet                                        
0     00082b12  _UARTParityModeGet                                        
0     00082b1b  _UARTFIFOIntLevelSet                                      
0     00082b35  _UARTFIFOIntLevelGet                                      
0     00082b4b  _UARTFIFOLevelGet                                         
0     00082b63  _UARTConfigSetExpClk                                      
0     00082b92  _UARTConfigGetExpClk                                      
0     00082bb6  _UARTEnable                                               
0     00082bc0  _UARTDisable                                              
0     00082bd3  _UARTsetLoopBack                                          
0     00082be4  _UARTFIFOEnable                                           
0     00082bed  _UARTFIFODisable                                          
0     00082bf6  _UARTTxIntModeSet                                         
0     00082c06  _UARTTxIntModeGet                                         
0     00082c10  _UARTCharsAvail                                           
0     00082c36  _UARTSpaceAvail                                           
0     00082c47  _UARTCharGetNonBlocking                                   
0     00082c6c  _UARTCharGet                                              
0     00082c84  _UARTCharPutNonBlocking                                   
0     00082c97  _UARTCharPut                                              
0     00082ca4  _UARTBusy                                                 
0     00082cb5  _UARTRXIntRegister                                        
0     00082ccd  _UARTTXIntRegister                                        
0     00082ce5  _UARTRXIntUnregister                                      
0     00082cfb  _UARTTXIntUnregister                                      
0     00082d11  _UARTIntEnable                                            
0     00082d42  _UARTIntDisable                                           
0     00082d78  _UARTIntStatus                                            
0     00082da8  _UARTIntClear                                             
0     00082dd5  _UARTRxErrorGet                                           
0     00082ddb  _UARTRxErrorClear                                         
0     00082df1  _HOSTwrite                                                
0     00082e29  _HOSTunlink                                               
0     00082e4d  _HOSTtime64                                               
0     00082e92  _HOSTtime                                                 
0     00082ec8  _HOSTrename                                               
0     00082f06  _HOSTread                                                 
0     00082f45  _HOSTopen                                                 
0     00082f85  _HOSTlseek                                                
0     00082fe6  _HOSTgetenv                                               
0     0008300e  _HOSTclose                                                
0     00083037  _HOSTclock                                                
0     0008306d  _UARTStdioConfig                                          
0     0008309f  _UARTwrite                                                
0     000830c0  _UARTgets                                                 
0     0008310f  _UARTgetc                                                 
0     00083115  _UARTvprintf                                              
0     000832c9  _UARTprintf                                               
0     000832d4  _xdc_runtime_System_doPrint__I                            
0     00083533  _InitGpio                                                 
0     00083573  _GPIO_SetupPinMux                                         
0     000835ff  _GPIO_SetupPinOptions                                     
0     00083693  _GPIO_SetupLock                                           
0     000836bc  _GPIO_SetupXINT1Gpio                                      
0     000836c6  _GPIO_SetupXINT2Gpio                                      
0     000836d0  _GPIO_SetupXINT3Gpio                                      
0     000836da  _GPIO_SetupXINT4Gpio                                      
0     000836e4  _GPIO_SetupXINT5Gpio                                      
0     000836ee  _GPIO_EnableUnbondedIOPullupsFor176Pin                    
0     00083707  _GPIO_EnableUnbondedIOPullupsFor100Pin                    
0     0008372c  _GPIO_EnableUnbondedIOPullups                             
0     00083742  _GPIO_ReadPin                                             
0     00083759  _GPIO_WritePin                                            
0     00083777  _SysCtlPeripheralPresent                                  
0     00083796  _SysCtlPeripheralReady                                    
0     000837d0  _SysCtlPeripheralReset                                    
0     000837fc  _SysCtlPeripheralEnable                                   
0     00083816  _SysCtlPeripheralDisable                                  
0     00083831  _SysCtlReset                                              
0     0008383b  _SysCtlClockGet                                           
0     00083887  _SysCtlLowSpeedClockGet                                   
0     0008389e  _SysCtlClockSet                                           
0     0008393a  _SysCtlAuxClockSet                                        
0     000839b8  _SysCtlUSBPLLEnable                                       
0     000839b9  _SysCtlUSBPLLDisable                                      
0     000839ba  _ti_sysbios_knl_Event_pend__E                             
0     00083bec  _ti_sysbios_knl_Semaphore_pend__E                         
0     00083dd7  _IntMasterEnable                                          
0     00083ddf  _IntMasterDisable                                         
0     00083de7  _IntRegister                                              
0     00083dfa  _IntUnregister                                            
0     00083e0f  _IntEnable                                                
0     00083ea2  _IntDisable                                               
0     00083f22  _IntIFRClear                                              
0     00083fa1  _SpiA_Task                                                
0     00083fff  _ti_sysbios_BIOS_linkedWithIncorrectBootLibrary__E        
0     00084000  _ti_sysbios_heaps_HeapMem_freeUnprotected__E              
0     000841a1  _IntAdc_prnt                                              
0     000841c0  _Task_Control                                             
0     000842dd  _TickTmr_Isr                                              
0     000842e6  _ti_sysbios_knl_Task_sleep__E                             
0     0008441b  _xdc_runtime_System_printfExtend__I                       
0     00084525  _InitGpio_PMCU                                            
0     00084583  _Setup_GPIO_for_ExtInterrupt                              
0     000845c6  _XINT1_Isr                                                
0     000845d6  _XINT2_Isr                                                
0     000845e6  _XINT3_Isr                                                
0     000845f6  _GPIOXint_Debug_Task                                      
0     0008462d  LL$$DIV                                                   
0     00084669  LL$$MOD                                                   
0     000846a3  ULL$$DIV                                                  
0     000846d2  ULL$$MOD                                                  
0     00084734  _InitEPwmGpio                                             
0     0008474d  _InitEPwm1Gpio                                            
0     0008475f  _InitEPwm2Gpio                                            
0     00084771  _InitEPwm3Gpio                                            
0     00084785  _InitEPwm4Gpio                                            
0     00084799  _InitEPwm5Gpio                                            
0     000847ab  _InitEPwm6Gpio                                            
0     000847bd  _InitEPwm7Gpio                                            
0     000847d1  _InitEPwm8Gpio                                            
0     000847e5  _InitEPwm9Gpio                                            
0     000847f7  _InitEPwm10Gpio                                           
0     0008480a  _InitEPwm11Gpio                                           
0     0008481e  _InitEPwm12Gpio                                           
0     00084831  _ti_sysbios_heaps_HeapMem_Instance_init__E                
0     00084927  _AD7689_SPIB_Init                                         
0     0008492d  _AD7689_SPIB_Read_All_Raw                                 
0     000849ff  _ti_sysbios_family_c28_Hwi_clearInterrupt__E              
0     00084adf  _xdc_runtime_LoggerBuf_write8__E                          
0     00084bbe  _AdcSetMode                                               
0     00084c61  _CalAdcINL                                                
0     00084c9b  _InitAdcC                                                 
0     00084cab  _ConfigureAdcC                                            
0     00084cc6  _StartAdcCsoftware                                        
0     00084ccb  _SetupAdcC                                                
0     00084d5b  _AdcC1_Isr                                                
0     00084d73  _xdc_runtime_Core_createObject__I                         
0     00084e4a  _InitAdcD                                                 
0     00084e5a  _ConfigureAdcD                                            
0     00084e75  _StartAdcDsoftware                                        
0     00084e7a  _SetupAdcDsoftware                                        
0     00084f00  _AdcD1_Isr                                                
0     00084f62  _AD7689_SPI_SendByte                                      
0     00084f69  _AD7689_SPIB_ReadByte                                     
0     00084f6f  _AD7689_SPIB_SendWord                                     
0     00084f76  _AD7689_SPIB_ReadWord                                     
0     00084f7c  _AD7689_SPIB_CS_LOW                                       
0     00084f84  _AD7689_SPIB_CS_HIGH                                      
0     00084f8c  _Set_max_speed_for_SpiB                                   
0     00084fa6  _spiB_fifo_init                                           
0     00084fb5  _Enable_SpiB_for_AD7689                                   
0     00084fe2  _ti_sysbios_knl_Event_post__E                             
0     000850ac  _ti_sysbios_knl_Semaphore_post__E                         
0     000851b6  _AD5764_SPIC_SendByte                                     
0     000851bd  _AD5764_SPIC_ReadByte                                     
0     000851c3  _AD5764_SPIC_SendWord                                     
0     000851ca  _AD5764_SPIC_ReadWord                                     
0     000851d0  _Set_max_speed_for_SpiC                                   
0     000851ec  _spiC_fifo_init                                           
0     000851fb  _Enable_SpiC_for_AD5764                                   
0     0008522a  _ldexpl                                                   
0     0008522a  _scalbnl                                                  
0     000852e6  _read_Resolver1                                           
0     000852ee  _read_Resolver2                                           
0     000852f6  _reset_Resolver1                                          
0     000852fb  _reset_Resolver2                                          
0     00085300  _read_FaultGroup1                                         
0     0008530a  _read_FaultGroup2                                         
0     00085314  _read_FaultGroup3                                         
0     0008531e  _on_InvMagnCon                                            
0     00085328  _off_InvMagnCon                                           
0     00085332  _emif1_write_ushort                                       
0     0008533f  _emif1_read_ushort                                        
0     0008534b  _EMIF_Debug_Task                                          
0     00085397  _EMIF_Debug_Tick                                          
0     0008539e  _ti_sysbios_knl_Clock_workFunc__E                         
0     00085454  _InitAdcA                                                 
0     00085460  _ConfigureAdcA                                            
0     0008547b  _StartAdcAsoftware                                        
0     00085480  _SetupAdcA                                                
0     00085500  _AdcA1_Isr                                                
0     00085509  _InitAdcB                                                 
0     00085515  _ConfigureAdcB                                            
0     00085530  _StartAdcBsoftware                                        
0     00085535  _SetupAdcB                                                
0     000855b5  _AdcB1_Isr                                                
0     000855be  _ti_sysbios_knl_Swi_run__I                                
0     0008566d  _ti_sysbios_family_c28_Hwi_dispatchCore__I                
0     0008571b  _xdc_runtime_Error_policyDefault__E                       
0     000857c0  _xdc_runtime_Core_constructObject__I                      
0     00085862  _InitSpiGpio                                              
0     00085869  _InitSpiaGpio                                             
0     0008588f  _InitSpibGpio                                             
0     000858c5  _InitSpicGpio                                             
0     000858ff  FD$$ADD                                                   
0     0008599b  _ti_sysbios_family_c28_Hwi_dispatchTable                  
0     000859f8  _ti_sysbios_family_c28_Hwi_dispatchPie                    
0     00085a36  _xdc_runtime_LoggerBuf_write4__E                          
0     00085acb  _InitIPCwithCPU2                                          
0     00085ae4  _Test_memcpy                                              
0     00085b0b  _Send_Ipc2CPU2                                            
0     00085b38  _Ipc0_Isr                                                 
0     00085b4a  _Ipc1_Isr                                                 
0     00085b52  _IpcRx_Task                                               
0     00085b5f  _ti_sysbios_BIOS_nullFunc__I                              
0     00085b60  ___TI_writemsg                                            
0     00085bb3  C$$IO$$                                                   
0     00085bb8  ___TI_readmsg                                             
0     00085bf4  _ti_sysbios_family_c28_Hwi_enableInterrupt__E             
0     00085c82  FD$$DIV                                                   
0     00085d31  _SpiB_Task                                                
0     00085d8a  _TickExtAdc_Isr                                           
0     00085db3  _TMP123_SPIA_ReadByte                                     
0     00085db9  _TMP123_SPIA_ReadWord                                     
0     00085dbf  _Set_max_speed_for_SpiA                                   
0     00085dd9  _spiA_fifo_init                                           
0     00085de7  _Enable_SpiA_for_TMP123                                   
0     00085e14  FD$$MPY                                                   
0     00085e97  _ti_sysbios_family_c28_Hwi_disableInterrupt__E            
0     00085f18  _ti_sysbios_family_c28_Hwi_disablePIEIER__E               
0     00085f96  _ti_sysbios_family_c28_Timer_stopAndClear__I              
0     00085ffc  _ti_catalog_c2800_initF2837x_Boot_init                    
0     00086000  _ti_sysbios_family_c28_Hwi_enablePIEIER__E                
0     0008607d  _xdc_runtime_Startup_startMods__I                         
0     000860fa  _xdc_runtime_Text_putSite__E                              
0     00086175  _delay_loop                                               
0     00086180  _ConfigureUART                                            
0     000861ab  _myOutputFunc                                             
0     000861b3  _main                                                     
0     000861eb  _EPwm1Isr                                                 
0     000861fa  _EPwm2Isr                                                 
0     00086206  _EPwm4Isr                                                 
0     00086215  _EPwm5Isr                                                 
0     00086221  _InitEPwm                                                 
0     0008625e  _ti_sysbios_knl_Task_checkStacks__E                       
0     000862d1  _ti_sysbios_knl_Task_startCore__E                         
0     00086342  _ti_sysbios_gates_GateMutex_enter__E                      
0     000863b2  _ti_sysbios_knl_Task_schedule__I                          
0     00086438  _AD5764_SPIB_CS_LOW                                       
0     0008643d  _AD5764_SPIB_CS_HIGH                                      
0     00086442  _AD5764_SPIC_Init                                         
0     0008644d  _AD5764_SPIC_Write_DAC                                    
0     0008646e  _AD5764_SPIC_Read_DAC                                     
0     0008648d  _c_int00                                                  
0     000864f0  _ti_sysbios_knl_Swi_post__E                               
0     00086550  _ti_sysbios_knl_Task_blockI__E                            
0     000865b0  _frexpl                                                   
0     0008660a  _ti_sysbios_knl_Task_exit__E                              
0     00086661  _ti_sysbios_family_c28_Timer_setPeriodMicroSecs__E        
0     000866b5  _ti_sysbios_knl_Task_unblockI__E                          
0     00086706  _xdc_runtime_Core_deleteObject__I                         
0     00086757  _xdc_runtime_Memory_alloc__E                              
0     000867a5  _xdc_runtime_Text_putLab__E                               
0     000867f1  _ti_sysbios_heaps_HeapMem_alloc__E                        
0     0008683c  _ti_sysbios_knl_Task_postInit__I                          
0     00086887  _ti_sysbios_knl_Mailbox_post__E                           
0     000868d0  _CmdLineProcess                                           
0     00086919  _ti_sysbios_family_c28_Hwi_Module_startup__E              
0     00086960  _SpiC_Task                                                
0     000869a6  _copy_in                                                  
0     000869ec  _ti_sysbios_family_c28_Timer_postInit__I                  
0     00086a2f  _xdc_runtime_Error_setX__E                                
0     00086a72  _ti_sysbios_family_c28_Hwi_unPluggedInterrupt__I          
0     00086ab4  _xdc_runtime_Core_assignParams__I                         
0     00086af6  _xdc_runtime_System_formatNum__I                          
0     00086b36  _xdc_runtime_LoggerBuf_setFilterLevel__E                  
0     00086b75  _ti_sysbios_knl_Mailbox_pend__E                           
0     00086bb3  _ti_sysbios_knl_Swi_restoreHwi__E                         
0     00086bf1  _xdc_runtime_LoggerBuf_getFilterLevel__E                  
0     00086c2d  _ti_sysbios_family_c28_TaskSupport_start__E               
0     00086c67  _xdc_runtime_Text_putMod__E                               
0     00086ca1  _ti_sysbios_knl_Semaphore_Instance_init__E                
0     00086cda  _xdc_runtime_Text_visitRope2__I                           
0     00086d13  _xdc_runtime_LoggerBuf_Object__create__S                  
0     00086d4b  _Init_IntTmr                                              
0     00086d61  _Mgmt_Task                                                
0     00086d81  _ti_sysbios_knl_Clock_logTick__E                          
0     00086db7  _xdc_runtime_Error_print__E                               
0     00086ded  _xdc_runtime_Startup_exec__E                              
0     00086e22  _ti_sysbios_BIOS_rtsUnlock__I                             
0     00086e56  _ti_sysbios_knl_Task_Module_startup__E                    
0     00086e88  _xdc_runtime_Assert_raise__I                              
0     00086eba  _xdc_runtime_LoggerBuf_Instance_init__E                   
0     00086eec  _sprintf                                                  
0     00086f1e  _ti_sysbios_family_c28_Timer_getFreq__E                   
0     00086f4f  _atoi                                                     
0     00086f80  _ti_sysbios_knl_Swi_runLoop__I                            
0     00086fae  _ti_sysbios_knl_Swi_schedule__I                           
0     00086fdc  _ltoa                                                     
0     0008700a  _ti_sysbios_heaps_HeapMem_getStats__E                     
0     00087037  _ti_sysbios_family_c28_Hwi_getStackInfo__E                
0     00087063  _ti_sysbios_family_c28_Timer_start__E                     
0     0008708f  _ti_sysbios_knl_Mailbox_Module_startup__E                 
0     000870ba  _xdc_runtime_Text_xprintf__I                              
0     000870e4  FD$$CMP                                                   
0     0008710e  L$$DIV                                                    
0     0008711d  L$$MOD                                                    
0     0008712b  UL$$DIV                                                   
0     00087132  UL$$MOD                                                   
0     00087138  C$$EXIT                                                   
0     00087138  _abort                                                    
0     0008713a  _exit                                                     
0     00087161  _xdc_runtime_SysMin_flush__E                              
0     00087189  _ti_sysbios_heaps_HeapMem_free__E                         
0     000871b0  _ti_sysbios_heaps_HeapMem_init__I                         
0     000871d7  _ti_sysbios_family_c28_TaskSupport_buildTaskStack         
0     000871fc  _copysignl                                                
0     00087220  _xdc_runtime_System_processAtExit__E                      
0     00087243  I$$DIV                                                    
0     00087254  I$$MOD                                                    
0     00087265  _ti_sysbios_knl_Task_allBlockedFunction__I                
0     00087286  _xdc_runtime_System_atexit__E                             
0     000872a7  FD$$TOI                                                   
0     000872c8  _ti_sysbios_family_c28_Timer_setPrescale__E               
0     000872e8  _ti_sysbios_gates_GateHwi_Object__create__S               
0     00087307  _ti_sysbios_gates_GateMutex_Object__create__S             
0     00087326  _ti_sysbios_heaps_HeapMem_Object__create__S               
0     00087345  FD$$TOL                                                   
0     00087364  _xdc_runtime_SysMin_putch__E                              
0     00087382  LL$$CMP                                                   
0     00087394  ULL$$CMP                                                  
0     000873a0  _memcpy                                                   
0     000873be  _ti_sysbios_family_c28_TaskSupport_swap__E                
0     000873db  _xdc_runtime_LoggerBuf_filterOutEvent__I                  
0     000873f8  I$$TOFD                                                   
0     00087415  _ti_sysbios_hal_Hwi_checkStack                            
0     00087431  _IPC2_ISR                                                 
0     0008743f  _IPC3_ISR                                                 
0     0008744d  FS$$TOFD                                                  
0     00087469  L$$TOFD                                                   
0     00087485  _ti_sysbios_family_c28_Hwi_switchAndDispatch__I           
0     000874a0  _ti_sysbios_hal_Hwi_initStack                             
0     000874bb  _ti_sysbios_knl_Semaphore_construct                       
0     000874d6  _ti_sysbios_knl_Task_processVitalTaskFlag__I              
0     000874f1  _xdc_runtime_SysMin_output__I                             
0     0008750c  _ti_sysbios_knl_Clock_addI__E                             
0     00087526  _xdc_runtime_Core_assignLabel__I                          
0     00087540  _xdc_runtime_LoggerBuf_Module_startup__E                  
0     0008755a  _ddcopy                                                   
0     0008755a  _dpcopy                                                   
0     0008755a  _pdcopy                                                   
0     0008755a  _ppcopy                                                   
0     00087574  _ti_sysbios_family_c28_Hwi_Object__get__S                 
0     0008758d  _ti_sysbios_knl_Event_pendTimeout__I                      
0     000875a6  _ti_sysbios_knl_Mailbox_postInit__I                       
0     000875bf  _ti_sysbios_knl_Queue_Object__get__S                      
0     000875d8  _ti_sysbios_knl_Queue_construct                           
0     000875f1  _ti_sysbios_knl_Semaphore_pendTimeout__I                  
0     0008760a  _ti_sysbios_knl_Swi_restore__E                            
0     00087623  _xdc_runtime_Memory_valloc__E                             
0     0008763c  _xdc_runtime_System_aprintf_va__F                         
0     0008763c  _xdc_runtime_System_avprintf__E                           
0     00087655  _xdc_runtime_System_putchar__I                            
0     0008766e  __args_main                                               
0     00087687  _ti_sysbios_family_xxx_Hwi_switchAndRunFunc               
0     0008769f  _LoggerBuf_instanceStartup                                
0     0008769f  _xdc_runtime_LoggerBuf_reset__E                           
0     000876b7  _xdc_runtime_System_printf_va__F                          
0     000876b7  _xdc_runtime_System_vprintf__E                            
0     000876cf  _xdc_runtime_Text_printVisFxn__I                          
0     000876e7  LL$$AND                                                   
0     000876ef  LL$$OR                                                    
0     000876f7  LL$$XOR                                                   
0     000876ff  _ti_sysbios_BIOS_atExitFunc__I                            
0     00087716  _ti_sysbios_family_c28_Timer_startup__E                   
0     0008772d  _ti_sysbios_heaps_HeapMem_Object__get__S                  
0     00087744  _ti_sysbios_knl_Clock_doTick__I                           
0     0008775b  _ti_sysbios_knl_Mailbox_Object__get__S                    
0     00087772  _ti_sysbios_knl_Swi_Object__get__S                        
0     00087789  _ti_sysbios_knl_Task_Object__get__S                       
0     000877a0  _xdc_runtime_LoggerBuf_Object__get__S                     
0     000877b7  _xdc_runtime_SysMin_abort__E                              
0     000877ce  _ti_sysbios_family_c28_Timer_Module_startup__E            
0     000877e4  _ti_sysbios_knl_Task_restore__E                           
0     000877fa  _ti_sysbios_BIOS_startFunc__I                             
0     0008780f  _ti_sysbios_knl_Swi_Module_startup__E                     
0     00087824  _xdc_runtime_Text_cordText__E                             
0     00087839  _ti_sysbios_knl_Idle_run__E                               
0     0008784d  _ti_sysbios_knl_Semaphore_Instance_finalize__E            
0     00087861  _ti_sysbios_BIOS_errorRaiseHook__I                        
0     00087874  _ti_sysbios_family_c28_Timer_checkOverflow__I             
0     00087887  _ti_sysbios_gates_GateMutex_Object__delete__S             
0     0008789a  _ti_sysbios_knl_Event_checkEvents__I                      
0     000878ad  _ti_sysbios_family_c28_Hwi_disableIER__E                  
0     000878bf  _ti_sysbios_gates_GateHwi_Object__delete__S               
0     000878d1  _ti_sysbios_heaps_HeapMem_Object__delete__S               
0     000878e3  _ti_sysbios_knl_Clock_Module_startup__E                   
0     000878f5  _xdc_runtime_LoggerBuf_Object__delete__S                  
0     00087907  _ti_sysbios_gates_GateHwi_Handle__label__S                
0     00087918  _ti_sysbios_gates_GateMutex_Handle__label__S              
0     00087929  _ti_sysbios_heaps_HeapMem_Handle__label__S                
0     0008793a  _xdc_runtime_Error_raiseX__E                              
0     0008794b  _xdc_runtime_LoggerBuf_Handle__label__S                   
0     0008795c  _ti_sysbios_family_c28_Hwi_enableIER__E                   
0     0008796c  _ti_sysbios_family_c28_Timer_stop__E                      
0     0008797c  _ti_sysbios_knl_Task_restoreHwi__E                        
0     0008798c  _ti_sysbios_gates_GateMutex_Instance_init__E              
0     0008799b  _ti_sysbios_knl_Semaphore_Object__destruct__S             
0     000879aa  _xdc_runtime_LoggerBuf_write2__E                          
0     000879b9  _xdc_runtime_Text_visitRope__I                            
0     000879c8  _IntDefaultHandler                                        
0     000879d7  _ti_sysbios_family_c28_f2837x_TimestampProvider_get64__E  
0     000879e5  _ti_sysbios_knl_Queue_Object__destruct__S                 
0     00087a01  _xdc_runtime_Registry_findById__E                         
0     00087a0f  _xdc_runtime_SysMin_Module_startup__E                     
0     00087a1d  FD$$SUB                                                   
0     00087a2b  _ti_sysbios_BIOS_registerRTSLock__I                       
0     00087a38  _ti_sysbios_BIOS_removeRTSLock__I                         
0     00087a45  _ti_sysbios_family_c28_Hwi_dispatchC__I                   
0     00087a52  _ti_sysbios_family_c28_Hwi_restoreIER__E                  
0     00087a5f  _ti_sysbios_knl_Task_SupportProxy_start__E                
0     00087a6c  _ti_sysbios_knl_Task_enter__I                             
0     00087a79  _ti_sysbios_knl_Task_sleepTimeout__I                      
0     00087a86  _xdc_runtime_Error_check__E                               
0     00087a93  _xdc_runtime_LoggerBuf_write1__E                          
0     00087aa0  _xdc_runtime_Memory_HeapProxy_alloc__E                    
0     00087aad  _xdc_runtime_System_abort__E                              
0     00087aba  _memccpy                                                  
0     00087ac7  _ti_sysbios_BIOS_exitFunc__I                              
0     00087ad3  _ti_sysbios_gates_GateMutex_leave__E                      
0     00087adf  _ti_sysbios_knl_Queue_get__E                              
0     00087aeb  _ti_sysbios_knl_Queue_put__E                              
0     00087af7  _ti_sysbios_knl_Task_enabled__E                           
0     00087b03  _xdc_runtime_Memory_free__E                               
0     00087b0f  _xdc_runtime_System_aprintf__E                            
0     00087b1b  _xdc_runtime_System_printf__E                             
0     00087b27  _xdc_runtime_Text_ropeText__E                             
0     00087b33  _memset                                                   
0     00087b3f  _strchr                                                   
0     00087b4b  _ti_sysbios_family_c28_Hwi_Module__startupDone__F         
0     00087b56  _ti_sysbios_family_c28_Timer_Module__startupDone__F       
0     00087b61  _ti_sysbios_knl_Task_unblock__E                           
0     00087b6c  _xdc_runtime_LoggerBuf_Instance_finalize__E               
0     00087b77  _xdc_runtime_LoggerBuf_write0__E                          
0     00087b82  _xdc_runtime_Startup_exec__I                              
0     00087b8d  _xdc_runtime_SysMin_exit__E                               
0     00087b98  _xdc_runtime_System_exit__E                               
0     00087ba3  U$$DIV                                                    
0     00087ba8  U$$MOD                                                    
0     00087bb8  _strcmp                                                   
0     00087bc2  _ti_sysbios_family_c28_TaskSupport_checkStack__E          
0     00087bcb  _ti_sysbios_family_c28_TaskSupport_glue                   
0     00087bd4  _ti_sysbios_hal_Hwi_Module_startup__E                     
0     00087bdd  _ti_sysbios_hal_Timer_Module_startup__E                   
0     00087be6  _xdc_runtime_System_snprintf_va__F                        
0     00087be6  _xdc_runtime_System_vsnprintf__E                          
0     00087bef  __register_unlock                                         
0     00087bf3  __register_lock                                           
0     00087bf7  __nop                                                     
0     00087bf8  FD$$NEG                                                   
0     00087c01  _ti_catalog_c2800_initF2837x_Boot_initSharedRAMs          
0     00087c09  _ti_sysbios_BIOS_setThreadType__E                         
0     00087c11  _ti_sysbios_gates_GateMutex_Instance_finalize__E          
0     00087c21  _xdc_runtime_Memory_HeapProxy_free__E                     
0     00087c29  _xdc_runtime_Memory_calloc__E                             
0     00087c31  _xdc_runtime_SysMin_ready__E                              
0     00087c39  _strlen                                                   
0     00087c41  _ti_catalog_c2800_initF2837x_Boot_initStartup             
0     00087c48  _ti_sysbios_BIOS_RtsGateProxy_leave__E                    
0     00087c4f  _ti_sysbios_hal_Hwi_HwiProxy_getStackInfo__E              
0     00087c56  _ti_sysbios_heaps_HeapMem_Module_GateProxy_leave__E       
0     00087c5d  _ti_sysbios_knl_Event_sync__E                             
0     00087c64  _ti_sysbios_knl_Queue_empty__E                            
0     00087c6b  _ti_sysbios_knl_Task_SupportProxy_checkStack__E           
0     00087c72  _ti_sysbios_knl_Task_SupportProxy_swap__E                 
0     00087c79  _xdc_runtime_Error_init__E                                
0     00087c80  _xdc_runtime_LoggerBuf_Module_GateProxy_leave__E          
0     00087c87  _xdc_runtime_System_Module_GateProxy_leave__E             
0     00087c8e  _ti_sysbios_BIOS_RtsGateProxy_enter__E                    
0     00087c94  _ti_sysbios_BIOS_start__E                                 
0     00087c9a  _ti_sysbios_family_c28_IntrinsicsSupport_maxbit__E        
0     00087ca0  _ti_sysbios_heaps_HeapMem_Module_GateProxy_enter__E       
0     00087ca6  _ti_sysbios_heaps_HeapMem_Module_GateProxy_query__E       
0     00087cac  _ti_sysbios_knl_Clock_TimerProxy_getMaxTicks__E           
0     00087cb2  _ti_sysbios_knl_Queue_destruct                            
0     00087cb8  _ti_sysbios_knl_Semaphore_destruct                        
0     00087cbe  _ti_sysbios_knl_Swi_disable__E                            
0     00087cc4  _ti_sysbios_knl_Task_disable__E                           
0     00087cca  _xdc_runtime_Gate_enterSystem__E                          
0     00087cd0  _xdc_runtime_Gate_leaveSystem__E                          
0     00087cd6  _xdc_runtime_LoggerBuf_Module_GateProxy_enter__E          
0     00087cdc  _xdc_runtime_LoggerBuf_TimestampProxy_get64__E            
0     00087ce2  _xdc_runtime_System_Module_GateProxy_enter__E             
0     00087ce8  _xdc_runtime_System_SupportProxy_abort__E                 
0     00087cee  _xdc_runtime_System_SupportProxy_exit__E                  
0     00087cf4  _xdc_runtime_System_SupportProxy_putch__E                 
0     00087cfa  _ti_sysbios_family_c28_Hwi_switchFromBootStack__E         
0     00087cff  _ti_sysbios_gates_GateHwi_enter__E                        
0     00087d09  _xdc_runtime_LoggerBuf_enable__E                          
0     00087d0e  _strcpy                                                   
0     00087d13  _ti_sysbios_family_c28_Hwi_startup__E                     
0     00087d17  _ti_sysbios_heaps_HeapMem_isBlocking__E                   
0     00087d1b  _ti_sysbios_knl_Swi_startup__E                            
0     00087d1f  _xdc_runtime_LoggerBuf_disable__E                         
0     00087d23  _xdc_runtime_Memory_getMaxDefaultTypeAlign__E             
0     00087d27  _xdc_runtime_Startup_rtsDone__E                           
0     00087d2b  ___xdc__init                                              
0     00087d2e  _ti_sysbios_family_c28_Hwi_Module__startupDone__S         
0     00087d31  _ti_sysbios_family_c28_Timer_Module__startupDone__S       
0     00087d34  _ti_sysbios_gates_GateHwi_leave__E                        
0     00087d37  _ti_sysbios_hal_Hwi_HwiProxy_Module__startupDone__S       
0     00087d3a  _ti_sysbios_hal_Hwi_HwiProxy_startup__E                   
0     00087d3d  _ti_sysbios_hal_Hwi_HwiProxy_switchFromBootStack__E       
0     00087d40  _ti_sysbios_hal_Hwi_startup__E                            
0     00087d43  _ti_sysbios_hal_Timer_TimerProxy_Module__startupDone__S   
0     00087d46  _ti_sysbios_knl_Clock_TimerProxy_Module__startupDone__S   
0     00087d49  _ti_sysbios_knl_Idle_loop__E                              
0     00087d4c  _ti_sysbios_knl_Queue_Instance_init__E                    
0     00087d4f  _ti_sysbios_knl_Task_SupportProxy_Module__startupDone__S  
0     00087d52  _ti_sysbios_knl_Task_startup__E                           
0     00087d55  _xdc_runtime_Startup_reset__I                             
0     00087d58  _xdc_runtime_System_Module_startup__E                     
0     00087d5b  _xdc_runtime_System_SupportProxy_ready__E                 
0     00087d5e  _xdc_runtime_System_abortStd__E                           
0     00087d61  _xdc_runtime_System_exitStd__E                            
0     00087d64  _ti_sysbios_family_c28_TaskSupport_Module__startupDone__S 
0     00087d66  _ti_sysbios_family_c28_Timer_getMaxTicks__E               
0     00087d68  _ti_sysbios_gates_GateHwi_query__E                        
0     00087d6a  _ti_sysbios_gates_GateMutex_query__E                      
0     00087d6c  _xdc_runtime_Error_getSite__E                             
0     00087d6e  _ti_sysbios_family_c28_Hwi_interruptReturn__I             
0     00087d6f  _ti_sysbios_gates_GateHwi_Instance_init__E                
0     00087d8c  __TI_table_binit                                          
0     00087d8c  ___binit__                                                
0     00087d8c  binit                                                     
0     00088000  _xdc_runtime_Text_charTab__A                              
0     0008a5c5  _ti_sysbios_family_c28_Hwi_Module__id__C                  
0     0008a80e  _ti_sysbios_family_c28_Hwi_vectors                        
0     0008ab57  __ctypes_                                                 
0     0008ad0b  _ti_sysbios_family_c28_Hwi_Module__loggerDefined__C       
0     0008adab  _ti_sysbios_family_c28_Hwi_NUM_INTERRUPTS_ALL__C          
0     0008aebd  _ti_sysbios_family_c28_Hwi_Object__count__C               
0     0008af29  _ti_sysbios_family_c28_TaskSupport_Module__id__C          
0     0008af91  _ti_sysbios_family_c28_Timer_Module__id__C                
0     0008afec  _xdc_runtime_Text_nodeTab__A                              
0     0008b09e  _Ext1Hwi                                                  
0     0008b0a0  _Ext2Hwi                                                  
0     0008b0a2  _Ipc0Hwi                                                  
0     0008b0a4  _Ipc0Mbx                                                  
0     0008b0a6  _GPIOXint_Debug                                           
0     0008b0a8  _EmifEvent                                                
0     0008b0aa  _Ext3Hwi                                                  
0     0008b0ac  _ExtIntEvent                                              
0     0008b0ae  _IntAppEvent                                              
0     0008b0b0  _IntAppMbx                                                
0     0008b0b2  _AdcCHwi                                                  
0     0008b0b4  _AdcDHwi                                                  
0     0008b0b6  _ePwmEvent                                                
0     0008b0b8  _EpwmMbx                                                  
0     0008b0ba  _ePwm1Hwi                                                 
0     0008b0bc  _ePwm4Hwi                                                 
0     0008b0be  _CanATxRxTask                                             
0     0008b0c0  _CanBTxRxTask                                             
0     0008b0c2  _MgmtEvent                                                
0     0008b0c4  _MgmtMbx                                                  
0     0008b0c6  _ControlTaskHd                                            
0     0008b0c8  _TickforTmr                                               
0     0008b0ca  _CMDtaskHd                                                
0     0008b0cc  _MgmtTaskHd                                               
0     0008b0ce  _CanAHwi                                                  
0     0008b0d0  _CanBHwi                                                  
0     0008b0d2  _EmifMbx                                                  
0     0008b0d4  _EMIF_Debug                                               
0     0008b0d6  _CanBEvent                                                
0     0008b0d8  _CanBRxMbx                                                
0     0008b0da  _CanAEvent                                                
0     0008b0dc  _CanARxMbx                                                
0     0008b0de  _SpiBTaskHandle                                           
0     0008b0e0  _ExtDacEvent                                              
0     0008b0e2  _ExtAdcEvent                                              
0     0008b0e4  _SpiBMbx                                                  
0     0008b0e6  _AdcAHwi                                                  
0     0008b0e8  _AdcBHwi                                                  
0     0008b0ea  _SpiCMbx                                                  
0     0008b0ec  _SpiCTaskHandle                                           
0     0008b0ee  _SpiAMbx                                                  
0     0008b0f0  _SpiATaskHandle                                           
0     0008b0f2  _adcResultSem                                             
0     0008b21b  _ti_sysbios_family_c28_Timer_startupNeeded__C             
0     0008b263  _ti_sysbios_gates_GateMutex_Module__id__C                 
0     0008b2a7  _ti_sysbios_hal_Hwi_Module__id__C                         
0     0008b31a  _xdc_runtime_LoggerBuf_Module__FXNS__C                    
0     0008b3a0  _xdc_runtime_Startup_sfxnTab__A                           
0     0008b3ca  _ti_sysbios_heaps_HeapMem_Module__FXNS__C                 
0     0008b3de  _ti_sysbios_gates_GateHwi_Module__FXNS__C                 
0     0008b3f0  _ti_sysbios_gates_GateMutex_Module__FXNS__C               
0     0008b402  _ti_sysbios_heaps_HeapMem_Object__PARAMS__C               
0     0008b414  _xdc_runtime_LoggerBuf_Object__PARAMS__C                  
0     0008b437  _ti_sysbios_heaps_HeapMem_Module__id__C                   
0     0008b438  _ti_sysbios_gates_GateHwi_Object__DESC__C                 
0     0008b448  _ti_sysbios_gates_GateMutex_Object__DESC__C               
0     0008b458  _ti_sysbios_heaps_HeapMem_Object__DESC__C                 
0     0008b468  _ti_sysbios_knl_Queue_Object__DESC__C                     
0     0008b478  _ti_sysbios_knl_Semaphore_Object__DESC__C                 
0     0008b488  _ti_sysbios_knl_Semaphore_Object__PARAMS__C               
0     0008b498  _xdc_runtime_LoggerBuf_Object__DESC__C                    
0     0008b4b4  _ti_sysbios_gates_GateHwi_Object__PARAMS__C               
0     0008b4c0  _ti_sysbios_gates_GateMutex_Object__PARAMS__C             
0     0008b4cc  _ti_sysbios_knl_Queue_Object__PARAMS__C                   
0     0008b4d8  _xdc_runtime_Startup_sfxnRts__A                           
0     0008b503  _ti_sysbios_heaps_HeapMem_Object__count__C                
0     0008b50a  _xdc_runtime_Startup_firstFxns__A                         
0     0008b515  _ti_sysbios_knl_Clock_Module__id__C                       
0     0008b516  _ti_sysbios_knl_Idle_funcList__C                          
0     0008b51a  _xdc_runtime_Startup_firstFxns__C                         
0     0008b51e  _xdc_runtime_Startup_lastFxns__C                          
0     0008b522  _ti_sysbios_BIOS_installedErrorHook__C                    
0     0008b524  _ti_sysbios_family_c28_Hwi_A_badIntNum__C                 
0     0008b526  _ti_sysbios_family_c28_Hwi_A_invalidArg__C                
0     0008b528  _ti_sysbios_family_c28_Hwi_E_unpluggedInterrupt__C        
0     0008b52a  _ti_sysbios_family_c28_Hwi_LD_end__C                      
0     0008b52c  _ti_sysbios_family_c28_Hwi_LM_begin__C                    
0     0008b52e  _ti_sysbios_family_c28_Hwi_Module__diagsEnabled__C        
0     0008b530  _ti_sysbios_family_c28_Hwi_Module__diagsIncluded__C       
0     0008b532  _ti_sysbios_family_c28_Hwi_Module__diagsMask__C           
0     0008b534  _ti_sysbios_family_c28_Hwi_Module__loggerFxn1__C          
0     0008b536  _ti_sysbios_family_c28_Hwi_Module__loggerFxn8__C          
0     0008b538  _ti_sysbios_family_c28_Hwi_Module__loggerObj__C           
0     0008b53a  _ti_sysbios_family_c28_Hwi_Object__table__C               
0     0008b53c  _ti_sysbios_family_c28_TaskSupport_E_invalidStack__C      
0     0008b53e  _ti_sysbios_family_c28_Timer_Module__diagsEnabled__C      
0     0008b540  _ti_sysbios_family_c28_Timer_Module__diagsIncluded__C     
0     0008b542  _ti_sysbios_family_c28_Timer_Module__diagsMask__C         
0     0008b544  _ti_sysbios_gates_GateMutex_A_badContext__C               
0     0008b546  _ti_sysbios_gates_GateMutex_Instance_State_sem__O         
0     0008b548  _ti_sysbios_gates_GateMutex_Module__diagsEnabled__C       
0     0008b54a  _ti_sysbios_gates_GateMutex_Module__diagsIncluded__C      
0     0008b54c  _ti_sysbios_gates_GateMutex_Module__diagsMask__C          
0     0008b54e  _ti_sysbios_hal_Hwi_E_stackOverflow__C                    
0     0008b550  _ti_sysbios_heaps_HeapMem_A_align__C                      
0     0008b552  _ti_sysbios_heaps_HeapMem_A_heapSize__C                   
0     0008b554  _ti_sysbios_heaps_HeapMem_A_invalidFree__C                
0     0008b556  _ti_sysbios_heaps_HeapMem_A_zeroBlock__C                  
0     0008b558  _ti_sysbios_heaps_HeapMem_E_memory__C                     
0     0008b55a  _ti_sysbios_heaps_HeapMem_Module__diagsEnabled__C         
0     0008b55c  _ti_sysbios_heaps_HeapMem_Module__diagsIncluded__C        
0     0008b55e  _ti_sysbios_heaps_HeapMem_Module__diagsMask__C            
0     0008b560  _ti_sysbios_heaps_HeapMem_Module__gateObj__C              
0     0008b562  _ti_sysbios_heaps_HeapMem_Object__table__C                
0     0008b564  _ti_sysbios_heaps_HeapMem_reqAlign__C                     
0     0008b566  _ti_sysbios_knl_Clock_LM_begin__C                         
0     0008b568  _ti_sysbios_knl_Clock_LM_tick__C                          
0     0008b56a  _ti_sysbios_knl_Clock_LW_delayed__C                       
0     0008b56c  _ti_sysbios_knl_Clock_Module_State_clockQ__O              
0     0008b56e  _ti_sysbios_knl_Clock_Module__diagsEnabled__C             
0     0008b570  _ti_sysbios_knl_Clock_Module__diagsIncluded__C            
0     0008b572  _ti_sysbios_knl_Clock_Module__diagsMask__C                
0     0008b574  _ti_sysbios_knl_Clock_Module__loggerFxn1__C               
0     0008b576  _ti_sysbios_knl_Clock_Module__loggerFxn2__C               
0     0008b578  _ti_sysbios_knl_Clock_Module__loggerObj__C                
0     0008b57a  _ti_sysbios_knl_Event_A_badContext__C                     
0     0008b57c  _ti_sysbios_knl_Event_A_eventInUse__C                     
0     0008b57e  _ti_sysbios_knl_Event_A_nullEventId__C                    
0     0008b580  _ti_sysbios_knl_Event_A_nullEventMasks__C                 
0     0008b582  _ti_sysbios_knl_Event_A_pendTaskDisabled__C               
0     0008b584  _ti_sysbios_knl_Event_Instance_State_pendQ__O             
0     0008b586  _ti_sysbios_knl_Event_LM_pend__C                          
0     0008b588  _ti_sysbios_knl_Event_LM_post__C                          
0     0008b58a  _ti_sysbios_knl_Event_Module__diagsEnabled__C             
0     0008b58c  _ti_sysbios_knl_Event_Module__diagsIncluded__C            
0     0008b58e  _ti_sysbios_knl_Event_Module__diagsMask__C                
0     0008b590  _ti_sysbios_knl_Event_Module__loggerFxn4__C               
0     0008b592  _ti_sysbios_knl_Event_Module__loggerFxn8__C               
0     0008b594  _ti_sysbios_knl_Event_Module__loggerObj__C                
0     0008b596  _ti_sysbios_knl_Idle_funcList__A                          
0     0008b598  _ti_sysbios_knl_Mailbox_Instance_State_dataQue__O         
0     0008b59a  _ti_sysbios_knl_Mailbox_Instance_State_dataSem__O         
0     0008b59c  _ti_sysbios_knl_Mailbox_Instance_State_freeQue__O         
0     0008b59e  _ti_sysbios_knl_Mailbox_Instance_State_freeSem__O         
0     0008b5a0  _ti_sysbios_knl_Mailbox_Object__table__C                  
0     0008b5a2  _ti_sysbios_knl_Queue_Object__table__C                    
0     0008b5a4  _ti_sysbios_knl_Semaphore_A_badContext__C                 
0     0008b5a6  _ti_sysbios_knl_Semaphore_A_overflow__C                   
0     0008b5a8  _ti_sysbios_knl_Semaphore_A_pendTaskDisabled__C           
0     0008b5aa  _ti_sysbios_knl_Semaphore_Instance_State_pendQ__O         
0     0008b5ac  _ti_sysbios_knl_Semaphore_LM_pend__C                      
0     0008b5ae  _ti_sysbios_knl_Semaphore_LM_post__C                      
0     0008b5b0  _ti_sysbios_knl_Semaphore_Module__diagsEnabled__C         
0     0008b5b2  _ti_sysbios_knl_Semaphore_Module__diagsIncluded__C        
0     0008b5b4  _ti_sysbios_knl_Semaphore_Module__diagsMask__C            
0     0008b5b6  _ti_sysbios_knl_Semaphore_Module__loggerFxn2__C           
0     0008b5b8  _ti_sysbios_knl_Semaphore_Module__loggerFxn4__C           
0     0008b5ba  _ti_sysbios_knl_Semaphore_Module__loggerObj__C            
0     0008b5bc  _ti_sysbios_knl_Semaphore_eventPost__C                    
0     0008b5be  _ti_sysbios_knl_Semaphore_eventSync__C                    
0     0008b5c0  _ti_sysbios_knl_Swi_LD_end__C                             
0     0008b5c2  _ti_sysbios_knl_Swi_LM_begin__C                           
0     0008b5c4  _ti_sysbios_knl_Swi_LM_post__C                            
0     0008b5c6  _ti_sysbios_knl_Swi_Module__diagsEnabled__C               
0     0008b5c8  _ti_sysbios_knl_Swi_Module__diagsIncluded__C              
0     0008b5ca  _ti_sysbios_knl_Swi_Module__diagsMask__C                  
0     0008b5cc  _ti_sysbios_knl_Swi_Module__loggerFxn1__C                 
0     0008b5ce  _ti_sysbios_knl_Swi_Module__loggerFxn4__C                 
0     0008b5d0  _ti_sysbios_knl_Swi_Module__loggerObj__C                  
0     0008b5d2  _ti_sysbios_knl_Swi_Object__table__C                      
0     0008b5d4  _ti_sysbios_knl_Task_A_badTimeout__C                      
0     0008b5d6  _ti_sysbios_knl_Task_A_sleepTaskDisabled__C               
0     0008b5d8  _ti_sysbios_knl_Task_E_spOutOfBounds__C                   
0     0008b5da  _ti_sysbios_knl_Task_E_stackOverflow__C                   
0     0008b5dc  _ti_sysbios_knl_Task_LD_block__C                          
0     0008b5de  _ti_sysbios_knl_Task_LD_exit__C                           
0     0008b5e0  _ti_sysbios_knl_Task_LD_ready__C                          
0     0008b5e2  _ti_sysbios_knl_Task_LM_sleep__C                          
0     0008b5e4  _ti_sysbios_knl_Task_LM_switch__C                         
0     0008b5e6  _ti_sysbios_knl_Task_Module_State_inactiveQ__O            
0     0008b5e8  _ti_sysbios_knl_Task_Module__diagsEnabled__C              
0     0008b5ea  _ti_sysbios_knl_Task_Module__diagsIncluded__C             
0     0008b5ec  _ti_sysbios_knl_Task_Module__diagsMask__C                 
0     0008b5ee  _ti_sysbios_knl_Task_Module__loggerFxn2__C                
0     0008b5f0  _ti_sysbios_knl_Task_Module__loggerFxn4__C                
0     0008b5f2  _ti_sysbios_knl_Task_Module__loggerObj__C                 
0     0008b5f4  _ti_sysbios_knl_Task_Object__table__C                     
0     0008b5f6  _ti_sysbios_knl_Task_allBlockedFunc__C                    
0     0008b5fc  _xdc_runtime_Assert_E_assertFailed__C                     
0     0008b5fe  _xdc_runtime_Core_A_initializedParams__C                  
0     0008b600  _xdc_runtime_Core_Module__diagsEnabled__C                 
0     0008b602  _xdc_runtime_Core_Module__diagsIncluded__C                
0     0008b604  _xdc_runtime_Core_Module__diagsMask__C                    
0     0008b606  _xdc_runtime_Error_E_memory__C                            
0     0008b608  _xdc_runtime_Error_Module__diagsEnabled__C                
0     0008b60a  _xdc_runtime_Error_Module__diagsIncluded__C               
0     0008b60c  _xdc_runtime_Error_Module__diagsMask__C                   
0     0008b60e  _xdc_runtime_Error_Module__loggerFxn8__C                  
0     0008b610  _xdc_runtime_Error_Module__loggerObj__C                   
0     0008b612  _xdc_runtime_Error_policyFxn__C                           
0     0008b614  _xdc_runtime_Error_raiseHook__C                           
0     0008b616  _xdc_runtime_IFilterLogger_Interface__BASE__C             
0     0008b618  _xdc_runtime_IGateProvider_Interface__BASE__C             
0     0008b61a  _xdc_runtime_IHeap_Interface__BASE__C                     
0     0008b61c  _xdc_runtime_ILogger_Interface__BASE__C                   
0     0008b61e  _xdc_runtime_IModule_Interface__BASE__C                   
0     0008b620  _xdc_runtime_Log_L_error__C                               
0     0008b622  _xdc_runtime_LoggerBuf_E_badLevel__C                      
0     0008b624  _xdc_runtime_LoggerBuf_Module__gateObj__C                 
0     0008b626  _xdc_runtime_LoggerBuf_Object__table__C                   
0     0008b628  _xdc_runtime_LoggerBuf_statusLogger__C                    
0     0008b62a  _xdc_runtime_Main_Module__diagsEnabled__C                 
0     0008b62c  _xdc_runtime_Main_Module__diagsIncluded__C                
0     0008b62e  _xdc_runtime_Main_Module__diagsMask__C                    
0     0008b630  _xdc_runtime_Memory_defaultHeapInstance__C                
0     0008b632  _xdc_runtime_Startup_execImpl__C                          
0     0008b634  _xdc_runtime_Startup_sfxnRts__C                           
0     0008b636  _xdc_runtime_Startup_sfxnTab__C                           
0     0008b638  _xdc_runtime_Startup_startModsFxn__C                      
0     0008b63a  _xdc_runtime_SysMin_bufSize__C                            
0     0008b63c  _xdc_runtime_SysMin_outputFunc__C                         
0     0008b63e  _xdc_runtime_System_Module__gateObj__C                    
0     0008b640  _xdc_runtime_System_abortFxn__C                           
0     0008b642  _xdc_runtime_System_exitFxn__C                            
0     0008b644  _xdc_runtime_System_extendFxn__C                          
0     0008b646  _xdc_runtime_Text_charTab__C                              
0     0008b648  _xdc_runtime_Text_nameEmpty__C                            
0     0008b64a  _xdc_runtime_Text_nameStatic__C                           
0     0008b64c  _xdc_runtime_Text_nameUnknown__C                          
0     0008b64e  _xdc_runtime_Text_nodeTab__C                              
0     0008b650  _xdc_runtime_Text_visitRopeFxn__C                         
0     0008b652  _ti_sysbios_knl_Clock_Module__loggerDefined__C            
0     0008b653  _ti_sysbios_knl_Event_Module__id__C                       
0     0008b654  _ti_sysbios_knl_Event_Module__loggerDefined__C            
0     0008b655  _ti_sysbios_knl_Mailbox_Object__count__C                  
0     0008b656  _ti_sysbios_knl_Mailbox_maxTypeAlign__C                   
0     0008b657  _ti_sysbios_knl_Queue_Object__count__C                    
0     0008b658  _ti_sysbios_knl_Semaphore_Module__id__C                   
0     0008b659  _ti_sysbios_knl_Semaphore_Module__loggerDefined__C        
0     0008b65a  _ti_sysbios_knl_Swi_Module__id__C                         
0     0008b65b  _ti_sysbios_knl_Swi_Module__loggerDefined__C              
0     0008b65c  _ti_sysbios_knl_Swi_Object__count__C                      
0     0008b65d  _ti_sysbios_knl_Task_Module__id__C                        
0     0008b65e  _ti_sysbios_knl_Task_Module__loggerDefined__C             
0     0008b65f  _ti_sysbios_knl_Task_Object__count__C                     
0     0008b660  _ti_sysbios_knl_Task_numConstructedTasks__C               
0     0008b661  _xdc_runtime_Core_Module__id__C                           
0     0008b662  _xdc_runtime_Error_Module__loggerDefined__C               
0     0008b663  _xdc_runtime_Error_maxDepth__C                            
0     0008b664  _xdc_runtime_Error_policy__C                              
0     0008b665  _xdc_runtime_LoggerBuf_Module__id__C                      
0     0008b666  _xdc_runtime_LoggerBuf_Object__count__C                   
0     0008b667  _xdc_runtime_LoggerBuf_filterByLevel__C                   
0     0008b668  _xdc_runtime_Main_Module__id__C                           
0     0008b669  _xdc_runtime_Memory_Module__id__C                         
0     0008b66a  _xdc_runtime_Startup_maxPasses__C                         
0     0008b66b  _xdc_runtime_SysMin_flushAtExit__C                        
0     0008b66c  _xdc_runtime_System_maxAtexitHandlers__C                  
0     0008b66d  _xdc_runtime_Text_charCnt__C                              
0     0008b66e  _xdc_runtime_Text_isLoaded__C                             
0     0008b66f  _xdc_runtime_Text_registryModsLastId__C                   
0     0008b670  _xdc_runtime_Text_unnamedModsLastId__C                    
0     0008b674  ___cinit__                                                
0     0008b674  cinit                                                     
1     00000122  __stack                                                   
1     00000322  __STACK_END                                               
1     00000b00  _AdcaResultRegs                                           
1     00000b20  _AdcbResultRegs                                           
1     00000b40  _AdccResultRegs                                           
1     00000b60  _AdcdResultRegs                                           
1     00000c00  _CpuTimer0Regs                                            
1     00000c08  _CpuTimer1Regs                                            
1     00000c10  _CpuTimer2Regs                                            
1     00000ce0  _PieCtrlRegs                                              
1     00001000  _DmaRegs                                                  
1     00001400  _Cla1Regs                                                 
1     00004000  _EPwm1Regs                                                
1     00004100  _EPwm2Regs                                                
1     00004200  _EPwm3Regs                                                
1     00004300  _EPwm4Regs                                                
1     00004400  _EPwm5Regs                                                
1     00004500  _EPwm6Regs                                                
1     00004600  _EPwm7Regs                                                
1     00004700  _EPwm8Regs                                                
1     00004800  _EPwm9Regs                                                
1     00004900  _EPwm10Regs                                               
1     00004a00  _EPwm11Regs                                               
1     00004b00  _EPwm12Regs                                               
1     00005000  _ECap1Regs                                                
1     00005020  _ECap2Regs                                                
1     00005040  _ECap3Regs                                                
1     00005060  _ECap4Regs                                                
1     00005080  _ECap5Regs                                                
1     000050a0  _ECap6Regs                                                
1     00005100  _EQep1Regs                                                
1     00005140  _EQep2Regs                                                
1     00005180  _EQep3Regs                                                
1     00005c00  _DacaRegs                                                 
1     00005c10  _DacbRegs                                                 
1     00005c20  _DaccRegs                                                 
1     00005c80  _Cmpss1Regs                                               
1     00005ca0  _Cmpss2Regs                                               
1     00005cc0  _Cmpss3Regs                                               
1     00005ce0  _Cmpss4Regs                                               
1     00005d00  _Cmpss5Regs                                               
1     00005d20  _Cmpss6Regs                                               
1     00005d40  _Cmpss7Regs                                               
1     00005d60  _Cmpss8Regs                                               
1     00005e00  _Sdfm1Regs                                                
1     00005e80  _Sdfm2Regs                                                
1     00006000  _McbspaRegs                                               
1     00006040  _McbspbRegs                                               
1     00006100  _SpiaRegs                                                 
1     00006110  _SpibRegs                                                 
1     00006120  _SpicRegs                                                 
1     00006200  _UppRegs                                                  
1     00007000  _WdRegs                                                   
1     00007060  _NmiIntruptRegs                                           
1     00007070  _XintRegs                                                 
1     00007200  _SciaRegs                                                 
1     00007210  _ScibRegs                                                 
1     00007220  _ScicRegs                                                 
1     00007230  _ScidRegs                                                 
1     00007300  _I2caRegs                                                 
1     00007340  _I2cbRegs                                                 
1     00007400  _AdcaRegs                                                 
1     00007480  _AdcbRegs                                                 
1     00007500  _AdccRegs                                                 
1     00007580  _AdcdRegs                                                 
1     00007900  _InputXbarRegs                                            
1     00007920  _XbarRegs                                                 
1     00007940  _SyncSocRegs                                              
1     00007980  _DmaClaSrcSelRegs                                         
1     00007a00  _EPwmXbarRegs                                             
1     00007a80  _OutputXbarRegs                                           
1     00007c00  _GpioCtrlRegs                                             
1     00007f00  _GpioDataRegs                                             
1     00008040  __CIOBUF_                                                 
1     0000c000  _ti_sysbios_knl_Task_Instance_State_6_stack__A            
1     0000c100  _ti_sysbios_knl_Task_Instance_State_5_stack__A            
1     0000c200  _ti_sysbios_knl_Task_Instance_State_10_stack__A           
1     0000c300  _ti_sysbios_knl_Task_Instance_State_8_stack__A            
1     0000c400  _ti_sysbios_knl_Task_Instance_State_1_stack__A            
1     0000c600  _ti_sysbios_knl_Task_Instance_State_3_stack__A            
1     0000c800  _ti_sysbios_knl_Task_Instance_State_2_stack__A            
1     0000ca00  _ti_sysbios_knl_Task_Instance_State_4_stack__A            
1     0000cc00  _ti_sysbios_knl_Task_Instance_State_9_stack__A            
1     0000d000  _ti_sysbios_knl_Task_Instance_State_0_stack__A            
1     0000d600  _ti_sysbios_knl_Task_Instance_State_7_stack__A            
1     0000de00  _ti_sysbios_heaps_HeapMem_Instance_State_0_buf__A         
1     0000ee03  _ExtDAC_DebugOn                                           
1     0000ee04  _threshold_t_value                                        
1     0000ee06  _threshold_m_value                                        
1     0000ee08  _m_rpm                                                    
1     0000ee0a  _T1_delta                                                 
1     0000ee0c  _t1_rpm                                                   
1     0000ee0e  _motor4_rpm                                               
1     0000ee10  _t1_sec                                                   
1     0000ee12  _t1_hz                                                    
1     0000ee14  _motor_dir                                                
1     0000ee16  _M_old                                                    
1     0000ee18  _qep_tcnt                                                 
1     0000ee1a  _T_ov                                                     
1     0000ee1c  _m_sec                                                    
1     0000ee1e  _m_hz                                                     
1     0000ee20  _M_new                                                    
1     0000ee22  _M_delta                                                  
1     0000ee24  _UT_PRD                                                   
1     0000ee26  _Extcnt                                                   
1     0000ee27  _ExtADC_DebugOn                                           
1     0000ee28  _ExtADC_Display_Interval                                  
1     0000ee29  _recv_data                                                
1     0000ee3f  _errno                                                    
1     0000ee40  _TorqueIndex                                              
1     0000ee41  _SpeedIndex                                               
1     0000ee42  _MFluxIndex                                               
1     0000ee44  _deltaMFlux                                               
1     0000ee46  _deltaTorque                                              
1     0000ee48  _iddd                                                     
1     0000ee4a  _iqqq                                                     
1     0000ee4c  _MagFlux                                                  
1     0000ee4e  _iRefC                                                    
1     0000ee50  _torqCmd                                                  
1     0000ee52  _iRefTMax                                                 
1     0000ee54  _deltaRpm                                                 
1     0000ee56  _tableY2                                                  
1     0000ee58  _tableX1                                                  
1     0000ee5a  _tableMin                                                 
1     0000ee5c  _tableMax                                                 
1     0000ee5e  _tableY1                                                  
1     0000ee60  _tableX2                                                  
1     0000ee80  _MFluxTable                                               
1     0000eec0  _rpmTable                                                 
1     0000ef00  _torqueTable                                              
1     0000ef80  _IqTable_Mot                                              
1     0000f900  _IdTable_Mot                                              
1     00010272  _Ecnt                                                     
1     00010273  _i                                                        
1     00010274  _Emif_DebugOn                                             
1     00010275  _ErrCount                                                 
1     00010276  _EMIF_Display_Interval                                    
1     00010278  _EMIF_Read_OffAddr                                        
1     0001027a  _TEST_STATUS                                              
1     0001027e  _g_ui32Base                                               
1     00010280  _xdc_runtime_Error_Module__state__V                       
1     00010282  _ti_sysbios_knl_Task_Module_State_0_idleTask__A           
1     00010284  ___xdc__init__addr                                        
1     00010286  _xdc_runtime_Memory_Module__state__V                      
1     00010288  _ti_sysbios_gates_GateHwi_Object__table__V                
1     0001028a  _xdc_runtime_LoggerBuf_Module__state__V                   
1     0001028e  _ti_sysbios_knl_Queue_Module__root__V                     
1     00010292  _ti_sysbios_knl_Event_Module__root__V                     
1     00010296  _ti_sysbios_hal_Hwi_Module__root__V                       
1     0001029a  _xdc_runtime_Registry_Module__state__V                    
1     0001029e  _ti_sysbios_knl_Swi_Module__root__V                       
1     000102a2  _ti_sysbios_knl_Clock_Module__root__V                     
1     000102a6  _xdc_runtime_Text_Module__state__V                        
1     000102aa  _ti_sysbios_knl_Semaphore_Module__root__V                 
1     000102ae  _ti_sysbios_knl_Mailbox_Module__root__V                   
1     000102b2  _ti_sysbios_gates_GateHwi_Module__root__V                 
1     000102b6  _xdc_runtime_LoggerBuf_Module__root__V                    
1     000102ba  _ti_sysbios_knl_Task_Module__root__V                      
1     000102c0  _ti_sysbios_gates_GateMutex_Module__root__V               
1     000102c4  _ti_sysbios_family_c28_Hwi_Module__root__V                
1     000102c8  _ti_sysbios_family_c28_Timer_Module__root__V              
1     000102cc  _xdc_runtime_SysMin_Module__state__V                      
1     000102d0  _xdc_runtime_System_Module__state__V                      
1     000102d4  _xdc_runtime_Startup_Module__state__V                     
1     000102d8  _ti_sysbios_hal_Timer_Module__root__V                     
1     000102dc  _ti_sysbios_heaps_HeapMem_Module__root__V                 
1     000102e0  _ti_sysbios_family_c28_Timer_Module__state__V             
1     000102e8  _xdc_runtime_System_Module_State_0_atexitHandlers__A      
1     000102f0  _ti_sysbios_knl_Semaphore_Object__table__V                
1     00010300  _ti_sysbios_knl_Swi_Module__state__V                      
1     0001030c  _ti_sysbios_heaps_HeapMem_Object__table__V                
1     00010318  _ti_sysbios_family_c28_Hwi_Module__state__V               
1     00010328  _ti_sysbios_knl_Mailbox_Instance_State_4_allocBuf__A      
1     00010340  _ti_sysbios_knl_Mailbox_Instance_State_9_allocBuf__A      
1     00010352  _xdc_runtime_LoggerBuf_Object__table__V                   
1     00010364  _ti_sysbios_knl_Mailbox_Instance_State_3_allocBuf__A      
1     00010380  _ti_sysbios_BIOS_Module__state__V                         
1     00010392  _ti_sysbios_knl_Swi_Object__table__V                      
1     000103a6  _ti_sysbios_knl_Clock_Module__state__V                    
1     000103c0  _ti_sysbios_gates_GateMutex_Object__table__V              
1     000103dc  _ti_sysbios_knl_Task_Module__state__V                     
1     00010400  _ti_sysbios_knl_Mailbox_Instance_State_2_allocBuf__A      
1     00010440  _ti_sysbios_knl_Mailbox_Instance_State_6_allocBuf__A      
1     00010480  _ti_sysbios_family_c28_Timer_Object__table__V             
1     000104c0  _ti_sysbios_knl_Mailbox_Instance_State_5_allocBuf__A      
1     00010500  _ti_sysbios_knl_Event_Object__table__V                    
1     00010540  _ti_sysbios_knl_Mailbox_Instance_State_1_allocBuf__A      
1     00010580  _ti_sysbios_knl_Mailbox_Instance_State_0_allocBuf__A      
1     000105c0  _ti_sysbios_knl_Swi_Module_State_0_readyQ__A              
1     00010600  _ti_sysbios_knl_Task_Module_State_0_readyQ__A             
1     00010640  _ti_sysbios_family_c28_Hwi_Object__table__V               
1     00010740  _ti_sysbios_knl_Mailbox_Instance_State_8_allocBuf__A      
1     00010880  _ti_sysbios_knl_Mailbox_Instance_State_7_allocBuf__A      
1     000109c0  _ti_sysbios_knl_Task_Object__table__V                     
1     00010b40  _ti_sysbios_knl_Mailbox_Object__table__V                  
1     00010d00  _ti_sysbios_family_c28_Hwi_Module_State_0_dispatchTable__A
1     00010ec0  _xdc_runtime_LoggerBuf_Instance_State_0_entryArr__A       
1     000110c0  _xdc_runtime_SysMin_Module_State_0_outbuf__A              
1     000112c0  _CANA_Err_Int_Enable                                      
1     000112c1  _Aerror_message                                           
1     000112c2  _Berror_message                                           
1     000112c3  _CAN_DebugOn                                              
1     000112c4  _CANB_Err_Int_Enable                                      
1     000112c6  _g_ulRxMsgCount                                           
1     000112c8  _u32CanAErrorStatus                                       
1     000112ca  _g_bErrFlag                                               
1     000112cc  _u32CntTXMsgData                                          
1     000112ce  _g_ulTxMsgCount                                           
1     000112d0  _ucTXMsgDataB                                             
1     000112d8  _g_ulRxMsgCountPMSM                                       
1     000112e0  _ucRXMsgDataB                                             
1     000112e8  _g_ulTxMsgCountPMSMB                                      
1     000112f0  _ucRXMsgDataA                                             
1     000112f8  _ucTXMsgDataA                                             
1     00011300  _sTXCANMessageA                                           
1     0001130a  _sRXCANMessageA                                           
1     00011314  _sTXCANMessageB                                           
1     0001131e  _sRXCANMessageB                                           
1     00011328  _g_ulTxMsgCountPMSM                                       
1     00011340  _g_ulRxMsgCountPMSMB                                      
1     0001134e  _ucRXMsgDataPMSM                                          
1     00011380  _ucTXMsgDataPMSMB                                         
1     000113c0  _sRXCANMessagePMSM                                        
1     00011400  _sTXCANMessagePMSMB                                       
1     00011440  _ucRXMsgDataPMSMB                                         
1     00011480  _ucTXMsgDataPMSM                                          
1     000114c0  _sTXCANMessagePMSM                                        
1     00011540  _sRXCANMessagePMSMB                                       
1     0001158e  ___TI_enable_exit_profile_output                          
1     00011590  ___TI_cleanup_ptr                                         
1     00011592  ___TI_dtors_ptr                                           
1     00011596  _TempReadInterval                                         
1     00011597  _Temp_DebugOn                                             
1     00011598  __lock                                                    
1     0001159a  __unlock                                                  
1     000115c2  _g_sFresultStrings                                        
1     00011640  _string_display                                           
1     000116c0  _g_psCmdTable                                             
1     00011780  _ExtInt_DebugOn                                           
1     000117c0  _GPIO_Conf_InitVal                                        
1     00011840  _Ccnt                                                     
1     00011841  _Bcnt                                                     
1     00011842  _BackTicker                                               
1     00011843  _Acnt                                                     
1     00011844  _ADC_Display_Interval                                     
1     00011845  _Dcnt                                                     
1     00011846  _IsrTicker4                                               
1     00011847  _TickCNT500ms                                             
1     00011848  _TickCNT100ms                                             
1     00011849  _TickCNT1000ms                                            
1     0001184a  _ADC_DebugOn                                              
1     0001184b  _TickCNT10ms                                              
1     0001184c  _IsrTicker1                                               
1     0001184e  _PwmCarrier                                               
1     00011850  _CurrentRisingEdgeDelay                                   
1     00011852  _CurrentCarrier2                                          
1     00011854  _PwmDuty                                                  
1     00011856  _PwmCarrier2                                              
1     00011858  _PwmDuty2                                                 
1     0001185a  _CurrentFallingEdgeDelay2                                 
1     0001185c  _CurrentRisingEdgeDelay2                                  
1     0001185e  _CurrentCarrier                                           
1     00011860  _CurrentFallingEdgeDelay                                  
1     00011862  _CurrentDuty2                                             
1     00011864  _CurrentDuty                                              
1     00011866  _AdcA_Cur                                                 
1     0001186c  _AdcD_Cur                                                 
1     00011872  _AdcB_Cur                                                 
1     00011878  _AdcC_Cur                                                 
1     00047000  _Emif1Regs                                                
1     00047800  _Emif2Regs                                                
1     00050000  _IpcRegs                                                  
1     00050024  _FlashPumpSemaphoreRegs                                   
1     0005d000  _DevCfgRegs                                               
1     0005d180  _AnalogSubsysRegs                                         
1     0005d200  _ClkCfgRegs                                               
1     0005d300  _CpuSysRegs                                               
1     0005e608  _RomPrefetchRegs                                          
1     0005f000  _DcsmZ1Regs                                               
1     0005f040  _DcsmZ2Regs                                               
1     0005f070  _DcsmCommonRegs                                           
1     0005f400  _MemCfgRegs                                               
1     0005f480  _Emif1ConfigRegs                                          
1     0005f4a0  _Emif2ConfigRegs                                          
1     0005f4c0  _AccessProtectionRegs                                     
1     0005f500  _MemoryErrorRegs                                          
1     0005f540  _RomWaitStateRegs                                         
1     0005f800  _Flash0CtrlRegs                                           
1     0005fb00  _Flash0EccRegs                                            
1     00078000  _DcsmZ1Otp                                                
1     00078200  _DcsmZ2Otp                                                
abs   00000001  _xdc_runtime_Startup__EXECFXN__C                          
abs   00000001  _xdc_runtime_Startup__RESETFXN__C                         
abs   0000003f  _RamfuncsLoadSize                                         
abs   0000003f  _RamfuncsRunSize                                          
abs   00000200  __STACK_SIZE                                              
abs   ffffffff  .text                                                     
abs   ffffffff  ___TI_pprof_out_hndl                                      
abs   ffffffff  ___TI_prof_data_size                                      
abs   ffffffff  ___TI_prof_data_start                                     
abs   ffffffff  ___c_args__                                               
abs   ffffffff  ___etext__                                                
abs   ffffffff  ___pinit__                                                
abs   ffffffff  ___text__                                                 
abs   ffffffff  etext                                                     
abs   ffffffff  pinit                                                     

[1208 symbols]
